:020000040000FA
:10000000000204000000000044A0000044A0000022
:1000100044A0000044A0000044A0000044A0000050
:1000200044A0000044A0000044A0000044A0000040
:1000300044A0000044A0000044A0000044A0000030
:1000400044A0000044A0000044A0000044A0000020
:1000500044A00000E07200000673000044A000000D
:1000600044A0000044A0000044A0000044A0000000
:1000700044A0000044A0000044A0000044A00000F0
:1000800044A0000044A0000044A0000044A00000E0
:1000900044A0000044A0000044A0000044A00000D0
:1000A00044A0000044A0000044A0000044A00000C0
:1000B00044A0000044A0000044A0000044A00000B0
:1000C00044A0000044A0000044A0000044A00000A0
:1000D00044A0000044A0000044A0000044A0000090
:1000E00044A0000044A0000044A0000044A0000080
:1000F00044A0000044A0000044A0000044A0000070
:1001000044A0000044A0000044A0000044A000005F
:1001100044A0000044A0000044A0000044A000004F
:1001200044A0000044A0000044A0000044A000003F
:1001300044A0000044A0000044A0000044A000002F
:1001400044A0000044A0000044A0000044A000001F
:1001500044A0000044A0000044A0000044A000000F
:1001600044A0000044A0000044A0000044A00000FF
:1001700044A0000044A0000044A0000044A00000EF
:1001800044A0000044A0000044A0000044A00000DF
:1001900044A0000044A0000044A0000044A00000CF
:1001A00044A0000044A0000044A0000044A00000BF
:1001B00044A0000044A0000044A0000044A00000AF
:1001C00044A0000044A0000044A0000044A000009F
:1001D00044A0000044A0000044A0000044A000008F
:1001E00044A0000044A0000044A0000044A000007F
:1001F00044A0000044A0000044A0000044A000006F
:10020000FFFFFF00FFFFFF0044A0000044A000002C
:1002100044A0000044A0000044A0000044A000004E
:1002200044A0000044A0000044A0000044A000003E
:1002300044A0000044A0000044A0000044A000002E
:1002400044A0000044A0000044A0000044A000001E
:1002500044A00000E07200000673000044A000000B
:1002600044A0000044A0000044A0000044A00000FE
:1002700044A0000044A0000044A0000044A00000EE
:1002800044A0000044A0000044A0000044A00000DE
:1002900044A0000044A0000044A0000044A00000CE
:1002A00044A0000044A0000044A0000044A00000BE
:1002B00044A0000044A0000044A0000044A00000AE
:1002C00044A0000044A0000044A0000044A000009E
:1002D00044A0000044A0000044A0000044A000008E
:1002E00044A0000044A0000044A0000044A000007E
:1002F00044A0000044A0000044A0000044A000006E
:1003000044A0000044A0000044A0000044A000005D
:1003100044A0000044A0000044A0000044A000004D
:1003200044A0000044A0000044A0000044A000003D
:1003300044A0000044A0000044A0000044A000002D
:1003400044A0000044A0000044A0000044A000001D
:1003500044A0000044A0000044A0000044A000000D
:1003600044A0000044A0000044A0000044A00000FD
:1003700044A0000044A0000044A0000044A00000ED
:1003800044A0000044A0000044A0000044A00000DD
:1003900044A0000044A0000044A0000044A00000CD
:1003A00044A0000044A0000044A0000044A00000BD
:1003B00044A0000044A0000044A0000044A00000AD
:1003C00044A0000044A0000044A0000044A000009D
:1003D00044A0000044A0000044A0000044A000008D
:1003E00044A0000044A0000044A0000044A000007D
:1003F00044A0000044A0000044A0000044A000006D
:100400008F272200007F22000001880000000000EA
:100410000C000700601929000100200011000700EE
:10042000000020000000E000020032000000020096
:1004300000000000C69F0200000000000040DA003B
:100440000000FE004440A900002F20000000E00052
:100450000300320000002000A00188004440A800F2
:100460000000060091018800800078000000EB0089
:1004700015003700E280400032A0B4009101BA00BC
:10048000E280400032A0B4009102BA00E280400055
:1004900032A0B4000002EB00472BDE00F507B200EB
:1004A000602CE10004003A000059EB008301E900F0
:1004B000FDFF3E00040037006128E100010032002A
:1004C0000082EB00040007001101BA000200E00006
:1004D000E8FF3A00000006003159BA008301E90044
:1004E0000C0032002159BA008301E90008003200F3
:1004F0000400E00003003A00E280400032A0B400B3
:10050000F5FF370011D9BA008301E900FAFF3A007C
:100510008100E800E180400032A0B4000000060045
:1005200000000000000000000000000000000000CB
:1005300000000000000000000000000000000000BB
:1005400000000000000000000000000000000000AB
:10055000000000000000000000000000000000009B
:1007E0000000000000000000889FBE008A9FBE003D
:1007F000010578000100E0000400350008003C001D
:100800000000E0002000320005003700600010000A
:10081000E080180002003B0001F02C001A003700B5
:100820000004BE006011B8006B0920000982CF00EF
:10083000020039000882CF000441B0006942520032
:100840000E00320008003B008281710061016400EB
:100850008904D1000884D3008B05E8000442E80035
:10086000F9FF3A00050037000804440089844C0071
:100870008B05E9000442E900FBFF3A002C01070068
:100880000AF0A70001F0A0004F05BE004F04BE0013
:1008900000000600F4FF2F004B0137001400200079
:1008A00049013700889FBE008A9FBE008C1F7800D8
:1008B000600107006701330003866C006450E100AB
:1008C0002E0032006420E100330032006150E1006C
:1008D0002F0032006120E100310032008585550093
:1008E000EB07B000090020000804200005003700D5
:1008F0000804440089844C000A00310006034300C8
:1009000087834B000001530081815B00F8FF3300B7
:100910000203BE000800A0000804440089844C00C3
:10092000F6FF3900C639DD00830173000100320093
:10093000130020008904D1000884D3000998A30083
:10094000050032000800A7000300A0008904D100C0
:100950000884D3008B05E8008904D1000884D30003
:100960000001EB000281D200F100070001F0A100BC
:100970000CF0A70001F0A0003F0137006420E10067
:10098000410132000801BE000200BE00F7FF37003F
:100990006120E1003C0132006000B800F3FF370045
:1009A0000000200001F82700F0FF370003F0A2004C
:1009B000889FBE008A9FBE008C1F78001D01070023
:1009C000240133006450E1004F0032006420E10054
:1009D0005200320003826C0007003B000905D00082
:1009E0000306D000820F54000C065D00020039009F
:1009F00002003200890178000306780085825500E4
:100A000004003D000003FD008103FD008502EA00B3
:100A10008B854200840F720002003B0060001000D2
:100A2000E08018006011B8000005EB007A28E100B2
:100A30000A00390006007800C75DDD00F707B20044
:100A4000878075002D003700828171000A017800CF
:100A5000610560008180D1000080D3008502E9003B
:100A6000F9FF3B00060440008784480002003B0079
:100A700060041400E0841C000988A3000700320011
:100A80008A81710082817100610164008904D10052
:100A90000884D3008B05E800170037000978A3000D
:100AA00013003A000B00E000130034008B05E9004E
:100AB0000804440089844C000A4474000978A300A7
:100AC0000D003A000B00E000070034008B05E90040
:100AD0000804440089844C0001003A000B00200007
:100AE0000978A300F7FF32000001EB000200370095
:100AF000828171000A0178008D0007000CF0A700C8
:100B000001F0A000DC0037006420E10002003A00A0
:100B1000838F6C00DC0033000801BE000200BE00C1
:100B2000D5003700889FBE008A9FBE008C1F7800CA
:100B3000C0000700C700330003866C006450E1006A
:100B4000240032006420E100270032006150E100FF
:100B5000220032006120E100210032008B8542003A
:100B6000EB07B1000134B800003AB80008044200B5
:100B700089844A00013AB8000030B80088804000FB
:100B800009014A0004003300000040008180480051
:100B9000020149008B05E900C909DD0083017000ED
:100BA0000100320013002000C814DE004814DD00EC
:100BB0004709DE001200B200C808DE000884700099
:100BC0005B00070001F0A1000CF0A70001F0A000FD
:100BD000A90037006120E100AB0032000801BE002F
:100BE0000200BE00F7FF37006150E100FCFF3A0051
:100BF000A50037000001BE00A60007000470A70092
:100C000003F0A10003F8A30013003A006509B10046
:100C100010003200090035006928E10002003500AB
:100C2000010028000000050000004000818048000D
:100C30008502E900FCFF3A0000000600F88F420040
:100C4000050035008100D1000080D3008502E80056
:100C5000FCFF3A00000006008000EB0000000500E9
:100C60006022B800060220000000D0008180D2007F
:100C70000482D2008582D2000000A000020252004D
:100C800083825A00030031000202420083824A003C
:100C90000000A1000603E900F3FF3A00000006008F
:100CA000EFFF07000400BE00000006000001BE00C8
:100CB000780007000470A70003F0A1006509B100E7
:100CC000160032000D0035006828E10006003500EE
:100CD000F0FF2F00F1FF27000300E00013003B00AE
:100CE000010028000000050000004000818048004D
:100CF0008502E900FCFF3A0008003700F88F420047
:100D000002003C008000EB00000005008100D100E3
:100D10000080D3008502E800FCFF3A000300E000F9
:100D200002003B0060001000E08018000000060098
:100D300081002000618055000B003D000B00200069
:100D400061FE2F000100E1001D003400828171006E
:100D5000610164008904D1000884D3000000E80028
:100D6000FAFF3A0071002000610064000300700087
:100D7000020060000900320061044400E0844C007D
:100D80000988A500050032008B05E8006808E1002D
:100D900002003A008904D1000884D300F20F200039
:100DA0000258E10005003D00C75DDD00F907B20013
:100DB0008980750008007800000006000BF8270005
:100DC0008B00780000000500889FBE008A9FBE004F
:100DD000841F7800170007004F00780011003300CF
:100DE000F0FF2F00838F6C0006003B0004056500B8
:100DF0000A00A7000800370009F0A6001000200034
:100E000008003700820F5400838F5C000300390014
:100E10001000200001003E000000200009F0A700A3
:100E20000000EA004F05BE004F04BE000000E000D5
:100E3000000006000004BE00160007000003BE000C
:100E40000405BE000200BE0012000700844F7500BA
:100E5000000006000200BE006450E10005003600FC
:100E60006420E100020036000968A30001003A0096
:100E70000800BE000160A0004F0678004F05BE00CC
:100E80004F04BE0000000600F0FF2F00F1FF270016
:100E9000F9FF3700C70ADE00F107B200F50FB20014
:100EA00008003200E1CF4200020032000170A000D1
:100EB00024000500810F70000100320004080500C5
:100EC00044000500810F700002003A001400050084
:100ED0008502E9000000400081C04800FCFF3B00A3
:100EE0000170A00024000500005E0000BCE20000CC
:100EF000613F0000DD830000C29C00007E200000F6
:100F0000A3FD00001F4100009DC30000217F0000E1
:100F1000FCA20000401E00005F010000E3BD0000D5
:100F20003E60000082DC0000237D00009FC10000C5
:100F3000421C0000FEA00000E1BF00005D030000B5
:100F400080DE00003C620000BEE00000025C0000A9
:100F5000DF810000633D00007C220000C09E000095
:100F60001D430000A1FF000046180000FAA4000085
:100F7000277900009BC5000084DA00003866000075
:100F8000E5BB000059070000DB8500006739000061
:100F9000BAE400000658000019470000A5FB000055
:100FA00078260000C49A0000653B0000D987000045
:100FB000045A0000B8E60000A7F900001B45000035
:100FC000C69800007A240000F8A60000441A000029
:100FD00099C70000257B00003A64000086D8000015
:100FE0005B050000E7B900008CD20000306E000005
:100FF000EDB30000510F00004E100000F2AC0000F5
:101000002F71000093CD0000114F0000ADF30000E0
:10101000702E0000CC920000D38D00006F310000D4
:10102000B2EC00000E500000AFF10000134D0000C4
:10103000CE900000722C00006D330000D18F0000B4
:101040000C520000B0EE0000326C00008ED00000A8
:10105000530D0000EFB10000F0AE00004C12000094
:1010600091CF00002D730000CA9400007628000084
:10107000ABF500001749000008560000B4EA000074
:1010800069370000D58B000057090000EBB5000060
:10109000366800008AD4000095CB00002977000054
:1010A000F4AA000048160000E9B70000550B000044
:1010B00088D60000346A00002B75000097C9000034
:1010C0004A140000F6A80000742A0000C896000028
:1010D000154B0000A9F70000B6E800000A54000014
:1010E000D78900006B3500004C450000540000001B
:1010F0004946000000540000484500004E00000032
:10110000454C000053450000004700004F540000CC
:101110004F000000474F0000535500004200000000
:101120005245000054550000524E0000005200008D
:10113000454D000000500000524900004E54000090
:10114000004900004E5000005554000000460000C9
:101150004F520000005400004F0000004E450000B8
:1011600058540000005200004541000044000000B7
:10117000444100005441000000530000544100006D
:10118000525400000053000054410000525400002B
:1011900052000000535400004F5000000053000064
:1011A000544F00005052000000530000454E000014
:1011B000440000005245000043450000495600002D
:1011C00045000000434C00004B000000444100007B
:1011D0005400000042490000545200004541000004
:1011E000440000004144000043000000415500005D
:1011F00058000000505300005500000050550000FA
:101200004C4C0000555000000041000055580000B3
:10121000504900004E0000004652000045510000B9
:1012200000440000555400005900000044450000EF
:101230004C410000590000004D41000043520000A5
:101240004F000000454E0000440000000052000026
:10125000554E0000004C00004953000054000000AF
:101260004558000049540000004400004542000079
:1012700055470000004E00004557000000000000E8
:101280003E200000000800002008000000000000D0
:10129000203D00002000000056520000454700009D
:1012A000207400006F6F0000206C00006F7700005A
:1012B0002C200000697300002074000068650000A5
:1012C000726500002061000020730000686F00005C
:1012D000727400003F0000002E2000003C0000005F
:1012E0003E0000002E200000000D00000A28000033
:1012F000002900003E20000000420000757300003D
:101300002050000069720000617400006520000038
:10131000763100006100000046690000726D000037
:10132000776100007265000020760000352E000015
:1013300038200000287200003530000034290000F9
:1013400020000000202800000041000033000000C1
:101350004234000000420000350000004238000026
:10136000005500004E4B000000290000004900001D
:10137000090000004F0900000048000009000000BB
:101380004C090000004500006E740000657200000A
:10139000207200006177000020760000616C000080
:1013A00075650000206600006F720000204200009A
:1013B00052470000000000003062000000300000D2
:1013C000303000002C000000303000000030000001
:1013D0003132000033340000353600003738000069
:1013E00039410000424300004445000046300000FF
:1013F00078000000436F0000756C0000646E000010
:1014000027740000206B000065650000702000005C
:1014100075700000000000005350000049310000CA
:10142000000000000029000000200000570000001C
:10143000205200000049000032430000310000004B
:101440003A200000000000002E000000315700008C
:10145000303100000000000008080000080800000B
:101460000800000000000000204800007A00000092
:101470000000000000410000525400003100000054
:1014800042420000494F000031000000524100007C
:101490005731000000000000314100004C530000B3
:1014A000000000004F430000443100000000000035
:1014B0000000000000000000290000000000000003
:1014C00000000000000000001C00FA000000EB001B
:1014D000200F98000000EB00506988000000EB002E
:1014E000406988000000EB00A04088000000EB008D
:1014F000606988000000EB00100798000000EB0016
:1015000040079800140037000000EB002007980007
:101510000B0037004E009000AE0090004500DD004B
:1015200081004000E0D22000808040000040EB00BD
:10153000804878002E0090000000E8002007980006
:101540002E009000FF0F5000F2FF34004E0090007C
:101550000000E800400798004E009000E40F5000A3
:10156000E9FF34000000EB00706E8800A1408000AD
:10157000E00220000088B900610220008080400065
:10158000E0932000008040002C6E0200000000006C
:10159000D140800000202000008060000000E000BA
:1015A0000400320071002000C0592000D89B0200C6
:1015B00000000000009428002C6E020000000000D3
:1015C000F6003700706E80000000E000630032001B
:1015D000706E80000000E900706E88000000EB0073
:1015E000200798001E00370042698000706E80005E
:1015F000AE0090004500DD0081004000E0D22000F8
:10160000008040009040780080C22000000041002F
:1016100001487800706E8000AE0090004500DD004B
:1016200081004000E0D2200000804000104078009F
:101630008872020000000000406980000000E8009D
:10164000406988002E0090000000E8002007980004
:1016500041698000F00F2000008060004069880030
:10166000706E8000AE0090004500DD0081004000FB
:10167000E0D2200000804000104078000004E0002C
:10168000D9FF3A000000EB00706E8800330037008D
:1016900080B8200010407800624060000004E00044
:1016A0002E003200A1408000E00220000088B90036
:1016B000FA004000E0932000008040001000780015
:1016C000000001000000E00024003200A140800082
:1016D000E00220000088B900610220008080400004
:1016E000E0932000008040002C6E0200000000000B
:1016F000009428002C6E0200000000005169800058
:1017000040698000808F50001400320050698000D2
:10171000200798000D003700AE00900080C2200026
:101720000080400010407800887202000000000035
:10173000AE009000F00F20000080600020079800AD
:101740002E0090000000E80020079800AE009000F6
:1017500040698000808F5000EFFF3A006A720200FB
:10176000000000000004E000C9FF320022C2BF00F8
:10177000624060000004E0000500320010118000AB
:10178000D1FF2F0001006000101188008300370096
:101790007672020000000000604798006E409000E2
:1017A0000080FB00300F98003E089000E80F5000CA
:1017B00011003200BE089000E88F500007003C0086
:1017C0003E0990000200E0003C003200BE0990009B
:1017D000E28F5100440032004B0037003E08900079
:1017E000EA0F500013003200BE089000ED8F500049
:1017F00010003200440037004169800050698000C9
:10180000808F500065003200406980000000E900D0
:101810004069880041698000F00F2000008060006E
:1018200040698800309428002C6E020000000000FF
:101830005A00370010002000200F980040698000F7
:101840008000E800F00F2000808060005069800078
:10185000808F50000D0032004169800080C220005E
:10186000808040000040EB008048780040698000A4
:101870000000E8004069880041698000F00F200006
:1018800000806000406988000800370070C0B30025
:1018900088720200000000004169800080C22000C0
:1018A000808040000040EB00804878007094280061
:1018B000586E020000000000380037001E00900043
:1018C0000000E800100798001E009000F40F500080
:1018D00032003A00E6780200000000000000EB0051
:1018E000100798002D0037001E009000E40F5000F4
:1018F0002A00340086880200000000000000EB008F
:101900001007980025003700406980008000E8003B
:10191000F00F20008080600050698000808F5000B0
:10192000160032006E409000FF4F50001B00360042
:101930006E4090000004E000180035006E409000FA
:101940008872020000000000416980006E41900032
:1019500080C220000080400002487800406980007A
:101960000000E8004069880041698000F00F200015
:1019700000806000406988000800370070C0B30034
:1019800088720200000000004169800080C22000CF
:10199000808040000040EB00804878002E089000D6
:1019A0000000E00007FF320040698000000F98004F
:1019B00050698000700798000000EB00200F98002D
:1019C0000000EB00100F98000000EB006069880039
:1019D000D140800000202000008060000000E00076
:1019E000E6043200DC30020000000000510020005C
:1019F000305A2000629C020000000000100020000D
:101A0000100F9800DD0437005169800080C220006B
:101A10000080400010407800604798006E409000C1
:101A20000080FB006101B900420F9800530F98003D
:101A3000D0072000010020004E099000DE09900030
:101A4000800F5100818F59009E043E004E08900087
:101A5000DE089000006001009C0437009904370004
:101A60009804370097043700960437009504370030
:101A70009404370093043700920437009104370030
:101A8000920437008F0437008E0437008F0437002C
:101A90008C0437008B0437008A0437008904370030
:101AA0008804370087043700860437008504370030
:101AB0008404370083043700820437008104370030
:101AC000800437007F0437007E0437007D04370030
:101AD0007C0437007B0437007C043700590437004E
:101AE0009B023700EE003700FB003700AA013700E9
:101AF0009801370073043700720237007104370011
:101B00007004370071043700700437000504370093
:101B10001E043700E90337001403370013033700AE
:101B20001203370011033700100337000F0337008B
:101B30000E0337000D0337000C0337000B0337008B
:101B4000600437005F043700B301370095003700A9
:101B50005C043700460037000D013700FF003700F6
:101B6000580437006B003700770137005504370001
:101B7000540437005304370052043700510437002F
:101B8000500437004F0437006C0037004D04370015
:101B90004C0437004B0437004A043700490437002F
:101BA00048043700910137004604370045043700E8
:101BB000440437000C013700420437004104370069
:101BC00040043700C5023700C9033700D50237008B
:101BD000FD033700E00337003A043700D200370036
:101BE0002E00370041003700490137003504370027
:101BF0003000370032003700150037001F00370073
:101C0000300437002F043700590037002100370017
:101C10002C043700230037002A043700290437003A
:101C20004D0337006D0137002604370025043700C7
:101C30001E0037002201370022043700210437003C
:101C400020043700AE02370073003700BE023700B1
:101C5000D90607000000E0001C043A00506980002B
:101C60007007980040698000000F98001704370043
:101C7000789C020000000000140437002E080700C2
:101C8000A04080000000E000100432008C08070033
:101C90000E043700400607000C043700B2090700A5
:101CA0000A0437008A09070008043700FE08070005
:101CB000060437003A7602000000000003043700F3
:101CC000A04080000000E00005003A00D1012000A3
:101CD000305D2000629C020000000000FB03370022
:101CE0009E74020000000000F803370080B8200056
:101CF000104078000000A10081B8200080487800E2
:101D000061012000805A2000629C02000000000057
:101D1000EE03370080B82000104078000000A000DB
:101D200081B820008048780051012000E05B20004D
:101D3000629C020000000000E403370080B820002D
:101D4000104078000020A00081B820008048780072
:101D5000C1012000B07E2000D89B020000000000DE
:101D600070942800586E020000000000D70337006E
:101D700080B82000104078000020A10081B8200029
:101D800080487800B1012000007D2000D89B02002F
:101D90000000000070942800586E0200000000004F
:101DA000CA033700506980000000E80050698800CD
:101DB00051698000F00F20000080600050698800A9
:101DC000E3050700F7030700200798002E009000A6
:101DD0002671020000000000809428002C6E020092
:101DE000000000002E009000C470020000000000FF
:101DF000809428002C6E0200000000002E0090004D
:101E00008C6E02000000000070942800586E0200E2
:101E100000000000AD033700506980000000E800BA
:101E20005069880051698000F00F20000080600038
:101E300050698800C6050700DA03070020079800EC
:101E40002E0090000080FB009C9902000000000022
:101E5000200798002E00900026710200000000006C
:101E6000809428002C6E0200000000002E009000DC
:101E7000C470020000000000809428002C6E020054
:101E8000000000002E0090008C6E02000000000098
:101E900070942800586E0200000000008B03370089
:101EA000089D0200000000000000E00087033200EF
:101EB0005100200030632000629C020000000000FE
:101EC00023C2BF00614060000004E000FCFF32005C
:101ED0000000FE007D033700089D020000000000A6
:101EE0000000E00079033200A100200080632000A0
:101EF000629C020000000000400620003A990200A7
:101F0000000000008C9702000000000023C2BF0008
:101F1000614060000004E000FCFF320081BF2A0045
:101F20000140010069033700430507000000E80095
:101F30004007980002003700787702000000000098
:101F40004E0090000000E900400798004E0090000D
:101F50000000E000F8FF3A005C0337003605070098
:101F60000000E800400798000200370056770200A2
:101F7000000000004E0090000000E90040079800BB
:101F80004E0090000000E000F8FF3A004F033700D9
:101F9000290507000000E800400798000B00370003
:101FA0006101200020642000D89B02000000000096
:101FB0009A77020000000000166E02000000000088
:101FC00070942800586E0200000000004E0090003F
:101FD0000000E900400798004E0090000000E0007B
:101FE000EFFF3A0039033700A04080000000E00016
:101FF00005003A00D1012000305D2000629C020003
:102000000000000031033700C082A900C282A8008E
:10201000C8A2A900CAA2A80021E3A80020002000AD
:102020003A99020000000000A0C0B300DC97020053
:102030000000000080007800001B2000808F50000E
:102040000F00360090C0B300DC97020000000000D3
:1020500080007800702B2000808F50000800360030
:102060001101200080652000D89B020000000000C4
:1020700070942800586E0200000000000E00370027
:10208000C082A900C282A900C8A2A900CAA2A90050
:10209000C0942800586E02000000000021012000BA
:1020A00090662000D89B0200000000007094280079
:1020B000586E02000000000021E3A900030337006E
:1020C000A04080000000E00005003A00D10120009F
:1020D000305D2000629C020000000000FB0237001F
:1020E000C082A900C282A900C8A2A900CAA2A900F0
:1020F0002101200090662000D89B02000000000013
:1021000070942800586E020000000000EF023700B3
:10211000F1002000A0392000D89B02000000000040
:10212000F69702000000000011002000903A200005
:10213000D89B02000000000070942800586E020036
:1021400000000000E10237000898020000000000D3
:10215000DE023700B8040700400798006100200045
:1021600070682000D89B0200000000004E00900024
:10217000667002000000000021002000D0682000EE
:10218000629C0200000000004E0090006699020070
:1021900000000000CD023700A704070040079800A8
:1021A0006100200070682000D89B02000000000041
:1021B0004E00900066700200000000002100200028
:1021C00090EC2000629C0200000000004E00900095
:1021D0003A99020000000000BC023700D0408000A5
:1021E0000090A000D0408800B8023700A0408000D6
:1021F0000000E00005003A00D1012000305D200021
:10220000629C020000000000B0023700CE7702009E
:1022100000000000AD023700100020006069880057
:10222000100020002007980010003700516980003E
:102230002E00900080804000F00F20008080600021
:1022400080C220000080400090407800E0C3B300CE
:1022500080CF500002003A000000EB006069880067
:102260002E0090000000E8002007980051698000CF
:102270002E00900080804000F00F200080806000E1
:1022800080C2200000804000104078000004E00080
:10229000E6FF3A00AE00900020022000808F500040
:1022A000020034001000200060698800606980002E
:1022B0000000E00085023A00506980000000E8005C
:1022C0005069880051698000F00F20000080600094
:1022D00050698800B3020700200798005169800008
:1022E000F00F20008080600080C22000008040004D
:1022F00090407800D0C3B30080CF500044003A0033
:102300002E0090000000E0003E0034002E009000FF
:10231000E50F50003B003C00506980000000E800E1
:102320005069880051698000F00F20000080600033
:10233000506988002E0090000000E90020079800F6
:102340000000EB00400798000B0037002E009000C3
:10235000CE0090004500DD0081004000E0D220006A
:10236000808040000040EB00804878004E009000E4
:102370000000E800400798004E009000FF0F50005A
:10238000F2FF34000000EB00400798001500370012
:10239000AE0190004E0290005169800080C2200082
:1023A00000804000104178004518DD0084004000A6
:1023B000E0D2200000804000024878004E009000EB
:1023C0000000E80040079800506980000000E80025
:1023D0005069880051698000F00F20000080600083
:1023E000506988005169800080C220000080400050
:1023F00090407800E0C3B30080CF5000E4FF3A0083
:102400003202370010002000606988002F02370078
:102410002E0090000000E0001B003A000000EB00DE
:1024200040079800140037004E0090000040E8007C
:10243000C470020000000000C09628002C6E02004C
:10244000000000004E0090004500DD008000780094
:10245000E0D22000008040002C6E0200000000004E
:1024600000972800586E0200000000004E00900007
:102470000000E800400798004E009000E40F500074
:10248000E9FF3400110237002E0090000000E00048
:10249000090034002E009000E50F500006003C00BB
:1024A00070942800586E020000000000AE009000FA
:1024B000716E8800050237001000200060698800F6
:1024C00002023700506980000000E800506988006F
:1024D00051698000F00F2000008060005069880082
:1024E0003002070060079800190407005169800056
:1024F000F00F20008080600080C22000008040003B
:102500009040780090C2B30080CF50000D003A0098
:10251000A1408000E00220000088B900FC004000DB
:10252000E093200000804000900078006E00900052
:102530000100010070942800586E020000000000A5
:10254000E20137001000200060698800DF013700D9
:10255000100020006069880010002000200798000B
:1025600010003700516980002E00900080804000EC
:10257000F00F20008080600080C2200000804000BA
:102580009040780020C2B30080CF500002003A0093
:102590000000EB00606988002E0090000000E80059
:1025A00020079800516980002E0090008080400034
:1025B000F00F20008080600080C22000008040007A
:1025C000104078000004E000E6FF3A0060698000F7
:1025D0000000E000BD013A0071002000F06820001A
:1025E000D89B02000000000020C2B30088720200E5
:1025F000000000002200370051698000F00F200029
:1026000000806000506988005169800080C220000D
:102610000080400010407800887202000000000036
:102620005169800080C22000008040001040780086
:102630000000FB006007980080B820001040780080
:10264000644060000004E000040032006E0090006E
:102650009C9902000000000060079800A1408000E3
:10266000E00220000088B900E8004000E09320006C
:1026700000804000900078006E0090000100010092
:10268000506980000000E8005069880051698000AE
:10269000F00F20008080600080C220000080400099
:1026A0009040780020C2B30080CF5000D2FF3A00A3
:1026B00050698000F10F200001006000506988001F
:1026C00020C2B3008872020000000000709428004D
:1026D000586E0200000000007C013700A14080001D
:1026E000E00220000088B90080007800E09320001C
:1026F00000804000100078000000010073013700E6
:10270000A1408000E00220000088B9008080E8003D
:10271000E0932000008040001000780000000100DD
:102720006A013700A1408000E00220000088B90063
:10273000E4004000E093200000804000100078009A
:102740000000010061013700A1408000E00220008C
:102750000088B900E6004000E093200000804000BF
:1027600010007800000001005801370071002000BF
:10277000F0682000D89B02000000000089010700DB
:1027800060079800506980000000E90050698800E7
:1027900051698000F00F20000080600050698800BF
:1027A000250307000000E8004007980045030700E4
:1027B000000F78001E00E0005D0032001E0078006F
:1027C0008040780070B72000014878008200200027
:1027D0009E0F11000600340080B8200010407800E1
:1027E0000040A00081B820008048780050003700E9
:1027F00080B82000104078000040A10081B820007F
:10280000804878004A0037006E00900094980200DB
:102810000000000080B82000104078007040600088
:102820000004E00004003A0070B720001040780077
:10283000E84F500009003A0080B8200010407800AE
:10284000704060000004E0000B00320070B7200010
:1028500010407800F04F500007003200B0C3B300C2
:10286000887202000000000070B72000104078005D
:10287000C47002000000000080B820001040780002
:10288000644060000004E000040032006E0090002C
:102890009C9902000000000060079800A1408000A1
:1028A000E00220000088B900E8004000E09320002A
:1028B00000804000900078006E0090000100010050
:1028C0005007980000C2B3008872020000000000A8
:1028D00080B82000104078000042B2000004E00000
:1028E000130032006100200060692000D89B0200C4
:1028F0000000000080B820001040780064406000B4
:102900000004E000040032005E0090009C99020088
:1029100000000000500798005E00900094980200AC
:102920000000000000C2B300887202000000000036
:102930004E0090000000E900400798004E00900013
:102940000000E000B0FF3A0070942800586E0200CA
:1029500000000000DD0037006100200060692000F9
:10296000D89B020000000000B30207000000E8004E
:1029700040079800D3020700000F78001E00E00017
:10298000440032001E0078008040780070B72000BC
:1029900001487800830020009E8F1100060034005B
:1029A00080B82000104078000040A00081B82000CE
:1029B000804878003700370080B820001040780049
:1029C0000040A10081B82000804878003100370025
:1029D000A1408000E00220000088B900EA00400029
:1029E000E09320000080400010007800000001000B
:1029F0005007980080B820001040780064406000C4
:102A00000004E000040032005E0090009C99020087
:102A100000000000500798005E00900094980200AB
:102A20000000000080B82000104078007040600076
:102A30000004E00004003A0070B720001040780065
:102A4000E84F500009003A0080B82000104078009C
:102A5000704060000004E0000B00320070B72000FE
:102A600010407800F04F500007003200B0C3B300B0
:102A7000887202000000000070B72000104078004B
:102A8000C47002000000000000C2B300887202009F
:102A9000000000004E0090000000E9004007980090
:102AA0004E0090000000E000C9FF3A00709428003A
:102AB000586E0200000000008400370081002000F2
:102AC000C0692000629C020000000000A14080005C
:102AD000E00220000088B900EC004000E0932000F4
:102AE00000804000100078000000010077003700EF
:102AF00081002000406A2000629C0200000000006B
:102B0000A1408000E00220000088B900EE004000F3
:102B1000E0932000008040001000780000000100D9
:102B20006A003700E1002000C06A2000629C0200B9
:102B300000000000A1408000E00220000088B900F1
:102B4000F0004000E093200000804000100078007A
:102B5000000001005D003700E1002000A06B2000B4
:102B6000629C020000000000A1408000E002200002
:102B70000088B900F2004000E0932000008040008F
:102B8000100078000000010050003700C100200054
:102B9000B0672000D89B020000000000A140800028
:102BA000E00220000088B900F4004000E09320001B
:102BB000008040001000780000000100166E020046
:102BC00000000000410037001B020700400798008A
:102BD000D1002000806D2000D89B02000000000082
:102BE0004E00900094980200000000004E009000FB
:102BF0000000E8004007980008003700A14080006E
:102C0000E00220000088B900F6004000E0932000B8
:102C10000080400010007800000001004E0090008D
:102C20000000E900400798004E0090000000E0001E
:102C3000F2FF3A0070942800586E02000000000075
:102C400022003700FC0107000000E8004007980060
:102C5000A1002000506E2000D89B02000000000060
:102C60000D003700A1408000E00220000088B9007C
:102C7000F8004000E0932000008040001000780041
:102C800000000100166E02000000000000C2B30048
:102C900088720200000000004E0090000000E90071
:102CA000400798004E0090000000E000EDFF3A0061
:102CB00001012000806C2000629C020000000000E6
:102CC0000200370010002000606988005069800011
:102CD0000000E8005069880051698000F00F200072
:102CE0000080600050698800606980000000E0009A
:102CF0001C00320051012000F06E2000D89B020021
:102D000000000000FE00900050698000808F50009D
:102D10000700310050698000804078007E009000FC
:102D200000C05000C4700200000000000600370020
:102D300050698000804078007E00900000C0500004
:102D4000C4700200000000000000EB006069880011
:102D500010002000100F980070942800586E020098
:102D6000000000005169800040698000808F5000A1
:102D700002003A0010002000100F98001E0890007A
:102D80000000E00020FB32000E089000506988002F
:102D90000E089000406988000000EB00200F9800AA
:102DA000F2F937000600FA000000EB001007980067
:102DB0000000EB00000F7800516980001E009000B9
:102DC00080804000F00F20008080600080C22000E2
:102DD000008040009040780000C3B30080CF5000D6
:102DE00043003400516980001E0090008080400044
:102DF000F00F20008080600080C220000080400032
:102E00009040780090C3B30080CF500038003C0061
:102E1000516980001E00900080804000F00F20006B
:102E20008080600080C22000008040001040780058
:102E30008000FB0000FD2F00008F40001E0090006E
:102E40000000E80010079800120037001E0078000C
:102E50006A00B900000F7800516980001E009000E0
:102E600080804000F00F20008080600080C2200041
:102E700000804000104078000000FB009E004000F1
:102E800000FD2F00008F40001E0090000000E800B1
:102E900010079800516980001E009000808040005B
:102EA000F00F20008080600080C220000080400081
:102EB00090407800F0C2B30080CF50005101340040
:102EC000516980001E00900080804000F00F2000BB
:102ED0008080600080C22000008040009040780028
:102EE00090C3B30080CF5000D8FF340045013700B5
:102EF000516980001E00900080804000F00F20008B
:102F00008080600080C220000080400090407800F7
:102F100000C3B30080CF500035013A001E0090007E
:102F20000000E80010079800516980001E00900022
:102F300080804000F00F20008080600080C2200070
:102F4000008040009040780020C6B30080CF500041
:102F50000B003200516980001E009000808040000C
:102F6000F00F20008080600080C2200000804000C0
:102F70009040780020C4B30080CF50002D003A006C
:102F80001E0090000000E8001007980012003700B3
:102F90001E00780000004000000F7800516980009A
:102FA0001E00900080804000F00F200080806000B4
:102FB00080C2200000804000104078000000FB002C
:102FC0009E00400000FD2F00008F40001E0090007A
:102FD0000000E80010079800516980001E00900072
:102FE00080804000F00F20008080600080C22000C0
:102FF000008040009040780010C3B30080CF5000A4
:10300000E3FF3200516980001E0090008080400084
:10301000F00F20008080600080C22000008040000F
:103020009040780000C3B30080CF5000D8FF32003A
:10303000F4003700516980001E009000808040003D
:10304000F00F20008080600080C2200000804000DF
:103050009040780080C7B30080CF50000B00320052
:10306000516980001E00900080804000F00F200019
:103070008080600080C22000008040009040780086
:1030800080C5B30080CF50008E003A001E00900033
:103090000000E80010079800470037001E00780085
:1030A0004400DD00000F7800516980001E00900090
:1030B00080804000F00F20008080600080C22000EF
:1030C0000080400090407800F0C2B30080CF5000F4
:1030D00018003400516980001E009000808040007C
:1030E000F00F20008080600080C22000008040003F
:1030F0009040780090C3B30080CF50000D003C009A
:10310000516980001E00900080804000F00F200078
:103110008080600080C22000008040001040780065
:103120000000FB009E00400000FD2F00008F4000CB
:103130001E003700516980001E0090008080400012
:10314000F00F200000816000516980001E00900097
:1031500080804000F00F20008080600080C220004E
:10316000008040009040780000C2B30080C0700032
:1031700080C22000000041000148780051698000B1
:103180001E00900080804000F00F200080806000D2
:1031900080C2200000804000104078000000FB004A
:1031A0009E00400090FA2F00008F40001E0090000B
:1031B0000000E80010079800516980001E00900090
:1031C00080804000F00F20008080600080C22000DE
:1031D0000080400090407800F0C2B30080CF5000E3
:1031E0000B003400516980001E0090008080400078
:1031F000F00F20008080600080C22000008040002E
:103200009040780090C3B30080CF5000A3FF3400FB
:10321000516980001E00900080804000F00F200067
:103220008080600080C220000080400090407800D4
:1032300000C4B30080CF50000B00340051698000FF
:103240001E00900080804000F00F20008080600011
:1032500080C22000008040009040780060C4B3002D
:1032600080CF50008DFF3400516980001E00900017
:1032700080804000F00F20008080600080C220002D
:10328000008040009040780000C6B30080CF50001E
:103290005C003400516980001E0090008080400076
:1032A000F00F20008080600080C22000008040007D
:1032B0009040780060C6B30080CF500077FF3400A4
:1032C00050003700516980001E009000808040004F
:1032D000F00F20008080600080C22000008040004D
:1032E00090407800F0C2B30080CF50004500340019
:1032F000516980001E00900080804000F00F200087
:103300008080600080C220000080400090407800F3
:1033100090C3B30080CF50003A003C005169800058
:103320001E00900080804000F00F20008080600030
:1033300080C2200000804000104078008000FB0028
:1033400000FD2F00008F4000120037001E007800A3
:103350006A00B900000F7800516980001E009000DB
:1033600080804000F00F20008080600080C220003C
:1033700000804000104078000000FB009E004000EC
:1033800000FD2F00008F40001E0090000000E800AC
:1033900010079800516980001E0090008080400056
:1033A000F00F20008080600080C22000008040007C
:1033B00090407800F0C2B30080CF5000110034007C
:1033C000516980001E00900080804000F00F2000B6
:1033D0008080600080C22000008040009040780023
:1033E00090C3B30080CF5000D8FF340005003700F1
:1033F00010002000606988000000EB0020079800A2
:103400000A003700516980001E00900000804000D3
:103410005069880051698000F00F20000080600032
:10342000506988001E007800200798002E00900048
:103430000080FA00000006000400FA0050698000D5
:103440008000E800F00F20008080600080C2200033
:103450000080400090407800A0C3B30080CF5000AF
:1034600013003A00506980000080E800506988002D
:1034700051698000F00F20000080600050698800D2
:1034800048FE0700000F7800506980000000E90046
:103490005069880051698000F00F200000806000B2
:1034A000506988001E00780010079800020037005D
:1034B00010002000100798001E0090000080FA0005
:1034C000000006000400FA00506980008000E80057
:1034D000F00F20008080600080C22000008040004B
:1034E00090407800B0C3B30080CF500013003A0082
:1034F000506980000080E8005069880051698000B0
:10350000F00F2000008060005069880025FE070051
:10351000000F7800506980000000E90050698800C1
:1035200051698000F00F2000008060005069880021
:103530001E00780010079800020037000000EB0022
:10354000100798001E0090000080FA00000006009E
:103550000000FA0007003700506980000000E80012
:103560005069880051698000F00F200000806000E1
:10357000506988005169800080C2200000804000AE
:103580009040780000C2B30080CF5000F2FF3200BC
:103590000080FA00000006000400FA000000EB00C2
:1035A000000F7800506980000000E8005069880032
:1035B00051698000F00F2000008060005069880091
:1035C000E3FF0700F7FD0700000F78001E00E00092
:1035D0004D003A000000EB00100798001300370080
:1035E0001E0090000040E800C470020000000000CF
:1035F000209728002C6E0200000000009E00900022
:10360000E00220000088B9006102200080804000B4
:10361000E093200000804000586E0200000000008F
:103620001E0090000000E800100798001E009000A7
:10363000E80F5000EAFF34007101200040702000C4
:10364000629C0200000000000000EB00606988003E
:103650001300200092002000110020001000200024
:10366000F6000700000FE900E0FF2F009E0F10009A
:10367000030032000080EB009E0F100005003A00AE
:10368000E1002000B0712000629C020000000000F8
:1036900042003700A1408000E00220000088B9000D
:1036A0000102200080804000E09320000080400064
:1036B00010007800000001008C970200000000005C
:1036C0001E007800A0408800A1408000E002200099
:1036D0000088B900FE004000E09320000080400018
:1036E00010007800000001001E00E0000100320020
:1036F000CA82A80051002000305A2000629C0200BB
:1037000000000000250037001E0FE90080002000A7
:103710009E0F10001D003C00A1408000E002200030
:103720000088B9000102200080804000E093200062
:103730000080400010007800000001008C9702001B
:10374000000000001E007800A0408800A14080001A
:10375000E00220000088B900FE004000E093200055
:103760000080400010007800000001001E00E00012
:1037700001003200CA82A80051002000305A200007
:10378000629C02000000000004003700510120008C
:1037900090722000629C02000000000040698000DE
:1037A0008000E900F00F2000008060005069880070
:1037B0000080FA00000006002600FA001000200039
:1037C00020079800506980000000E9001007980069
:1037D0009E009000F00F200000806000100798000D
:1037E000430037009E00900080C22000008040000F
:1037F000104078000004E00036003A001E009000FF
:103800008000E800F00F20008080600080C220006F
:1038100000804000104078000004E0002D003200DD
:103820002E009000C47002000000000020972800C5
:103830002C6E02000000000010002000000F780035
:103840000A0037001E0090009E004000F00F20008C
:103850008080600080C2200000804000104078001E
:1038600088720200000000001E0FE8001E00900099
:103870009E004000F00F20008080600080C2200089
:1038800000804000104078000004E000EDFF3A00A6
:10389000AE0190001E0090008000E800F00F2000B4
:1038A00000816000E60047000380410002B078001C
:1038B0002E0090000000E800200798002E009000E5
:1038C000EF0F50000E00320070942800586E020076
:1038D000000000001E0090000000E90010079800A2
:1038E0009E009000F00F20000080600010079800FC
:1038F0009E00900050698000808F5000B9FF3A0010
:1039000071002000E0732000629C020000000000B3
:10391000130020002E019000110020000000EB0099
:1039200046000700100798001E009000E10F4000BD
:1039300003003A0010002000201798003C003700D8
:103940000000EB0020079800160037004169800056
:103950002E00900080804000F00F20000081600069
:103960001E009000E600470000004000E080780064
:103970002E00900080804000F00F200080806000CA
:1039800080C22000008040009040780080C220006B
:1039900000004100014878002E0090000000E8007F
:1039A000200798001E009000E6004700000040003D
:1039B000E08078002E00900080804000F00F200012
:1039C0008080600080C220000080400010407800AD
:1039D0000004E000DDFF3A00406980008000E9005B
:1039E000F00F20000080600050698800516980005D
:1039F0002E009000008040008080E800F00F200042
:103A00000080600040698800406980008000E90013
:103A1000F00F20008080600080C220008080400085
:103A20000040EB00804878000000EB002017980071
:103A30002E1090000080FA00000006001E00FA0020
:103A4000100F9800210F9800320F9800430F980034
:103A50000000EB00400798000000EB0020079800F2
:103A60000000EB00100798000000EB00000F78004A
:103A7000509728002C6E0200000000001E089000E5
:103A8000C470020000000000909728002C6E020015
:103A9000000000006700370076720200000000009E
:103AA000204F98002E4890000000FB00600F980007
:103AB0006E089000ED0F500029003200EE089000D3
:103AC000ED8F500007003C006E099000E80F510098
:103AD0000D0032006E089000EA0F50002000320006
:103AE00035003700D0022000EE089000808F500093
:103AF0001E003200800720006E099000800F5100E8
:103B0000270032002C0037004E0090000000E0003B
:103B1000070032004E0090000000E90040079800C6
:103B2000309428002C6E0200000000004100370095
:103B30001E00E000060032000000EB00000F7800DD
:103B4000309428002C6E020000000000390037007D
:103B500070C0B3008872020000000000350037001A
:103B60001000200020079800320037004E0090001F
:103B70000000E00006003A00D0C2B30088720200E4
:103B80000000000010002000000F7800290037001E
:103B900070C0B300887202000000000025003700EA
:103BA0004E0890000000E000030032000080EB00AF
:103BB000500F98005D003700AE489000F0C2B3008F
:103BC00080CF500018003400AE48900090C3B3007E
:103BD00080CF500014003C004E009000E30F5000D6
:103BE0000600340070C0B3008872020000000000BC
:103BF00040002000400798000E0037002E4890003B
:103C00008872020000000000CE0090006B004700A8
:103C10002E499000827078004E0090000000E8006D
:103C2000400798000300370070C0B300887202009C
:103C3000000000002E0090000000E00096FF32001F
:103C400070942800586E0200000000004E009000A2
:103C50000000E00003003A001E089000500F98009A
:103C6000320037000000EB00100798004E00900073
:103C70000000E90040079800CE009000310798004E
:103C8000110037001E0090006A00B900100798006C
:103C9000BE0090004E009000808050006B004700F6
:103CA000614078008000FB001E0090008080400092
:103CB00000FD2F0000804000100798004E0090008B
:103CC0000000E900400798004E0090000000E0006E
:103CD000ECFF3D009E0090002E089000808F500069
:103CE0000D0035009E0090003E089000808F50002F
:103CF00009003C001E00E000040032001E0090009D
:103D00000000EA00500F9800080037001E019000E4
:103D1000520F980005003700B1012000E0EA2000B2
:103D2000629C02000000000049FF37005E0890001E
:103D30000080FA00000006000400FA00D097280076
:103D4000586E020000000000C09828002C6E02008F
:103D500000000000D100200070802000D89B0200ED
:103D600000000000A1BF2A000000EB00E273020087
:103D700000000000000F78001E0078004800DE0000
:103D8000C470020000000000E0C2B30088720200AC
:103D9000000000001E007800C47002000000000057
:103DA00070942800586E020000000000610020009E
:103DB00000762000D89B020000000000B040800088
:103DC0007E710200000000007100200070EA2000F7
:103DD000D89B020000000000C04080007E710200FD
:103DE00000000000209A28002C6E02000000000055
:103DF000C040800010079800200423009E0090001F
:103E0000808F500016003200200423009E00900096
:103E1000808F500005003E00300023009E0090007F
:103E2000808F50000A003200190037003004230050
:103E30009E009000808F50000D003200600423002F
:103E40009E009000808F50000D003200100037005F
:103E5000509A28002C6E0200000000000F0037006E
:103E6000809A28002C6E0200000000000B00370032
:103E7000B09A28002C6E02000000000007003700F6
:103E8000E09A28002C6E02000000000003003700BA
:103E9000109B28002C6E020000000000509B2800A0
:103EA000586E020000000000E10120006076200052
:103EB000629C0200000000000080FA000000060082
:103EC0000000FA005100200020922000D89B020040
:103ED00000000000C1BF2A000000EB00E2730200F6
:103EE000000000007E710200000000006100200060
:103EF00070922000D89B020000000000E1BF2A0061
:103F00000000EB00E2730200000000007E7102007E
:103F10000000000070942800586E020000000000AD
:103F2000C100200040782000629C020000000000D8
:103F30005D000700CAC2BF000042B2000004E000FA
:103F4000050032001101200080652000D89B02008E
:103F500000000000040037002101200090662000CE
:103F6000D89B020000000000C0C2B30088720200AB
:103F70000000000000C2B3008872020000000000D0
:103F800080B8200010407800684060000004E00025
:103F9000050032002102200000792000629C02000E
:103FA0000000000004003700E1012000207B200019
:103FB000629C02000000000080B8200010407800E1
:103FC000644060000004E00005003A00B1012000F8
:103FD000007D2000D89B0200000000000400370094
:103FE000C1012000B07E2000D89B0200000000002C
:103FF000C0C2B300887202000000000000C2B3001B
:104000008872020000000000B1012000C0202100E1
:10401000D89B02000000000070B72000104078001C
:10402000C47002000000000070942800586E020066
:104030000000000080B8200010407800614060005F
:104040000004E0000500320051012000E05B200088
:10405000629C0200000000000400370061012000A3
:10406000805A2000629C020000000000A1408000F5
:10407000E00220000088B90041022000808040005A
:10408000E093200000804000100078000000010054
:10409000C100200040782000629C02000000000067
:1040A0000080FA00000006000000FA00A1002000D5
:1040B000A0052100629C02000000000061042000B5
:1040C000200B2100629C020000000000A1012000E2
:1040D00040062100D89B020000000000A1408000A3
:1040E000E00220000088B90021022000808040000A
:1040F000E0932000008040001000780000000100E4
:10410000A1002000E0072100D89B02000000000071
:104110000040200050000700001020004E00070063
:10412000002020004C000700000420004A00070087
:10413000000820004800070070942800586E020014
:104140000000000041002000800F2100D89B0200E9
:104150000000000021E3A800A0C0B300DC9702002B
:1041600000000000C87102000000000011002000E3
:10417000903A2000D89B02000000000090C0B300DD
:10418000887202000000000090C0B300DC970200BB
:1041900000000000C87102000000000011002000B3
:1041A000903A2000D89B02000000000090C0B300AD
:1041B0008872020000000000C0C0B300DC9702005B
:1041C00000000000C8710200000000001100200083
:1041D000903A2000D89B02000000000090C0B3007D
:1041E0008872020000000000B0C0B300DC9702003B
:1041F00000000000C8710200000000001100200053
:10420000903A2000D89B02000000000090C0B3004C
:10421000887202000000000021E3A9000040200095
:104220001C000700001020001A00070000202000DA
:1042300018000700000420001600070000082000F6
:104240001400070070942800586E0200000000005F
:104250000080FA00000006000200FA00000F78005B
:10426000401680001E0060000000E00004003200E4
:10427000709B28002C6E0200000000000300370035
:10428000A09B28002C6E0200000000000080FA00B5
:10429000000006000200FA00000F780050168000AF
:1042A0001E0060000000E00004003200D09B2800E7
:1042B0002C6E02000000000003003700009C280064
:1042C0002C6E0200000000000080FA0000000600D2
:1042D0000200FA00506980000000E8005069880080
:1042E00051698000F00F2000008060005069880054
:1042F00097FC0700ABFA0700000F78001E00E000F3
:1043000006003400400020009E0F100003003C0017
:104310001E00E900904088000D0037000000EB000F
:10432000606988002102200040812000629C020018
:10433000000000008001EB0042002000110020007E
:1043400010002000BDFD07000000E900904088003B
:104350002101200060832000629C02000000000018
:104360000080FA00000006000200FA005069800098
:104370000000E8005069880051698000F00F2000BB
:10438000008060005069880071FC070085FA070012
:10439000104798001E4090000004E0000900320021
:1043A0001E409000EA4F500006003E001E40900064
:1043B0000040E9008040780000812000014878003A
:1043C0000F0037000000EB0060698800D108200072
:1043D00030872000629C0200000000008001EB009A
:1043E000A2002000110020009000200093FD070093
:1043F0000040E900804078000081200001487800FA
:104400000081200010407800E94F500010003A0071
:104410004FFC070063FA0700004F78001E04E0001D
:104420000B003A000000EB0060698800309C280017
:10443000586E0200000000008001EB00F2FF270030
:104440008000EB00200220007CFD0700004F780078
:104450004101200000902000629C0200000000004A
:1044600011012000B01F2100629C0200000000002A
:1044700023C2BF00614060000004E000FCFF320086
:104480000081200010407800E94F500003003A00FE
:104490001E407800A672020000000000669802002C
:1044A00000000000000037006A72020000000000F7
:1044B0000004E000FCFF3200767202000000000001
:1044C0008040780000C2B30080CF5000010032006D
:1044D000F5FF37000080FA00000006000000FA0037
:1044E0004173800000E72000008040009040780089
:1044F00030C8B30080CF50000E003A0040738000F7
:104500000000E8004073880003003700407380001B
:104510000000E800407388004173800000E720003D
:10452000008040009040780000CEB30080CF500063
:10453000F6FF36000080FA00000006000A00FA00CC
:10454000300798000000EB0020079800AE009000B4
:1045500000E72000008040009040780000CEB300CB
:1045600080CF500003003E000080EB004007980021
:1045700023003700AE00900000E7200000804000DC
:10458000104078008080FB0000F22F000080400087
:10459000100798002E0090008000E80000E720003F
:1045A00000804000104078000080FB004801DD00E2
:1045B0002E0090008080E80000E72000008040008E
:1045C000104078000080FB00000F41009E00780042
:1045D0003E009000808F500003003A002E009000B3
:1045E00040079800060037009E0090002E009000C3
:1045F000008040006300400020079800D3FF370090
:104600004E0090000080FA00000006000600FA004C
:10461000881F78000000EB00000F780041738000D5
:1046200000E72000008040009040780080C2B30086
:1046300080CF500010003A00407380000000E80076
:10464000407388001D010700000F7800417380004F
:1046500000E72000008040009040780090C2B30046
:1046600080CF5000AA003A00407380000000E800AC
:1046700040738800A60037004173800000E72000E7
:10468000008040009040780000C4B30080CF50000C
:10469000160036004173800000E7200000804000D3
:1046A00090407800A0C5B30080CF50000F003E00BE
:1046B0004273800000E720000000410010407800B5
:1046C0008080FB00F0FB2F00008040008000400055
:1046D00080E0200000804000100078002007980053
:1046E0000200E800407388008B00370041738000AF
:1046F00000E72000008040009040780000C8B30030
:1047000080CF5000740036004173800000E7200025
:1047100000804000104078000080FB0010079800E7
:104720000100E80040738800700920009E0090009E
:10473000808F500041003200700920009E009000E0
:10474000808F50000D003C00400920009E0090002A
:10475000808F500016003200600920009E009000FB
:10476000808F50002B003200300920009E00900006
:10477000808F50001800320046003700900920005A
:104780009E009000808F50001E0032009009200093
:104790009E009000808F500039003500A009200055
:1047A0009E009000808F50002E00320039003700AC
:1047B000A1408000E00220000088B900EA0040002B
:1047C000E09320000080400010007800000001000D
:1047D000000F78004E003700A1408000E00220006A
:1047E0000088B900E8004000E0932000008040000D
:1047F000100478008200070008000100000F780014
:10480000430037009A77020000000000000F780094
:104810003F003700A1408000E00220000088B9007E
:10482000F4004000E0932000008040001000780079
:1048300000000100000F780035003700A140800023
:10484000E00220000088B900F8004000E09320005A
:10485000008040001000780000000100000F780088
:104860002B003700CAC2BF000080FB004500DE00FD
:10487000614060000080FB00000F780024003700DA
:10488000C0C0B300DC97020000000000000F7800F9
:104890001F0037000000EB00000F78001C003700FD
:1048A0001E0078006A00B900000F78004173800094
:1048B00000E7200000804000104078000080FB00EE
:1048C0009E00400000FD2F00008F400040738000DC
:1048D0000000E800407388004173800000E720007A
:1048E0000080400090407800F0C2B30080CF5000BC
:1048F000070036004173800000E720000080400080
:104900009040780090C3B30080CF5000E4FF3600A1
:104910001E007800200798002E0090004F047800B9
:104920000080FA00000006000600FA0037FF0700CA
:10493000000F7800000037004173800000E720007E
:104940000080400090407800A0C2B30080CF5000AB
:104950000A0032004173800000E720000080400020
:1049600090407800F0C2B30080CF500003003200C6
:104970001E007800200798001E0037004173800059
:1049800000E7200000804000104078000080FB001D
:10499000100798000100E80040738800A002200082
:1049A0009E009000808F500005003200F002200031
:1049B0009E009000808F500007003200DEFF37001D
:1049C00012FF0700800078001E0078000180B90007
:1049D000000F7800D8FF37000CFF070000017800B7
:1049E0001E007800110009000200D800000F7800B6
:1049F000D1FF37002E0090000080FA000000060072
:104A00000600FA00C8FF0700000F7800000037001A
:104A10004173800000E72000008040009040780053
:104A2000D0C2B30080CF50000A0032004173800032
:104A300000E720000080400090407800B0C2B30042
:104A400080CF5000030032001E007800200798003D
:104A5000170037004173800000E72000008040000D
:104A6000104078000080FB00100798000100E8006B
:104A700040738800B00220009E009000808F50009C
:104A800008003200D00220009E009000808F50006D
:104A900001003200DEFF3700A3FF07001E0F1000E9
:104AA000DBFF3700A0FF07001E0F4000D8FF3700D4
:104AB0002E0090000080FA00000006000C00FA00B2
:104AC0004273800000E720000000410010407800A1
:104AD0008080FB00F0FB2F00008040008000400041
:104AE00080E02000008040009000780021079800BE
:104AF0000200E800407388000000EB00000F78001F
:104B00000B0037009E0178004273800000E7200010
:104B100000004100104078008040780066004700A7
:104B2000817178000200E800407388001E0FE800E1
:104B30004173800000E72000008040009040780032
:104B400000C4B30080CF50000700360041738000DE
:104B500000E720000080400090407800A0C5B3002E
:104B600080CF50000E0036004173800000E7200027
:104B70000080400090407800F0C2B30080CF500029
:104B8000E0FF36004173800000E720000080400015
:104B90009040780090C3B30080CF5000D9FF3E0012
:104BA00097FF070010079800660047001040780044
:104BB0000000FB0050079800C0032000DE009000BA
:104BC000808F500032003200C0032000DE009000D1
:104BD000808F500005003C0010022000DE00900095
:104BE000808F5000410032004E003700D00320007B
:104BF000DE009000808F500005003200E0032000AE
:104C0000DE009000808F50000A003200450037001F
:104C10000000EB0040079800AE0090001E009000DE
:104C2000808F500041003A00110020004107980099
:104C30003E0037006600470090409000D0C3B300AC
:104C400080CF500009003A000000EB0040079800B8
:104C5000AE0090001E009000808F500033003500A1
:104C60001100200041079800300037000000EB00E1
:104C700040079800AE0090001E009000808F50000A
:104C80002A00340011002000410798002700370057
:104C90006600470090409000D0C3B30080CF500022
:104CA00009003A000000EB0040079800AE009000B9
:104CB0001E009000808F50001C003C00110020005E
:104CC00041079800190037000000EB0040079800EA
:104CD000AE0090001E009000808F500013003D0039
:104CE00011002000410798001000370066004700BF
:104CF00090409000D0C3B30080CF500009003A002C
:104D00000000EB0040079800AE0090001E009000ED
:104D1000808F5000050032001100200041079800EC
:104D2000020037000000EB00400798004E009000A2
:104D30000080FA00000006001C00FA00881F7800BE
:104D40000000EB00407388000000EB003007980083
:104D50000000EB00200798000000EB00100798000F
:104D60000000EB00507388000000EB0060738800C7
:104D70000000EB00707388000000EB005007980003
:104D8000D04080000080A000D04088000000EB00F0
:104D900040079800090037004E0090008000400056
:104DA00080E02000808040000000EB008008780058
:104DB0004E0090000000E800400798004E00900070
:104DC000F90F5000F4FF3400330437001E00900048
:104DD0000000E00021003A004173800000E720005D
:104DE0000080400090407800F0CDB30080CF5000AC
:104DF00003003E00200020003007980029043700FF
:104E00004173800000E720000080400010407800DF
:104E10008080FB0000F22F000080400060079800B7
:104E2000407380008000E80000E720000080400020
:104E3000104078000080FB004801DD0040738000D6
:104E40008080E80000E720000080400010407800EB
:104E50000080FB0000007100500798000000EB008C
:104E60001007980040738000E300400000E7200036
:104E700000804000104078000080FB006101B90014
:104E800000F82F00F1FF2F0002014000838148004D
:104E9000420F9800530F98001002200001002000DC
:104EA0004E099000DE099000800F5100818F59005B
:104EB000ED033E004E089000DE0890000060010007
:104EC0002100370035003700E7033700E6033700DD
:104ED0007100370081003700A3003700B7003700AA
:104EE000BE0037003B01370088013700DE03370082
:104EF000EE0137003502370099023700A002370073
:104F0000AE023700BC023700CA023700D8023700B1
:104F1000D50337007A0337005E033700D20337002A
:104F2000D1033700E2023700F0023700A103370057
:104F3000AC03370000033700140337003403370095
:104F4000B4033700C5033700100020002007980085
:104F5000407380006600400040738800407380000A
:104F60008080E90000E720000080400010407800C9
:104F70008080FB00F0FB2F0000844000A0FE0700B3
:104F8000000178008800440080E02000008040009C
:104F90000208780051FD0700B5033700100020001B
:104FA0002007980040738000640040004073880030
:104FB000C2FE07000000E0001C00320041738000C8
:104FC000310F980000E720003E09900000004100EA
:104FD000904078008041EB004357980020C8B30010
:104FE00080CF500002003A0010C0B3004057980034
:104FF000BE0890000100E800407388004E51900008
:105000000204E0009A03320010002000100798000C
:1050100040738000630050004073880094033700A1
:10502000407380000000E8004073880041738000F6
:1050300000E72000008040009040780030C8B300B6
:1050400080CF5000070032004173800000E720004D
:10505000008040009040780000CEB30080CF500028
:10506000EFFF36004173800000E720000080400021
:105070009040780030C8B30080CF50007C033A00E5
:105080001000200010079800407380000080E900A5
:105090004073880076033700100020002007980036
:1050A00040738000640040004073880054FE070095
:1050B00022FD0700000F78008081EB009E8F110019
:1050C000030032001E007800407388006803370038
:1050D00060002000300798006503370010002000B2
:1050E00020079800407380006400400040738800EF
:1050F00060738000E90F500018003C00627380006C
:10510000417380006E009000008040008001E90043
:1051100082004100C0E320000080400003087800C6
:10512000607380000000E8006073880034FE0700B0
:1051300002FD0700000F78008080EB009E8F1000BA
:10514000030032001E0178004273880048033700D4
:1051500060002000300798004503370070002000F1
:105160003007980042033700008928002C6E0200A7
:1051700000000000100020002007980060738000ED
:105180000000E0000A003200607380000000E900C7
:10519000607388006073800080004000C0E32000DE
:1051A0000080400010007800407388003003370012
:1051B00080002000300798002D03370010002000E9
:1051C00020079800417380006E009000008040002E
:1051D0006300400040738800250337001000200062
:1051E00020079800407380006400400040738800EE
:1051F000570037004173800000E720000080400026
:105200009040780020C2B30080CF50001F003A00C9
:10521000407380000000E8004073880010003700F1
:10522000D04080000080A100D04088004173800001
:1052300000E7200000804000104078000041780026
:105240000100E80040738800024078008872020084
:1052500000000000D04080000080A000D040880006
:105260004173800000E720000080400090407800FB
:1052700020C2B30080CF5000E9FF3A0040738000A5
:105280000000E8004073880031003700417380005F
:1052900000E72000008040009040780000C4B30088
:1052A00080CF5000070036004173800000E72000E7
:1052B0000080400090407800A0C5B30080CF50002F
:1052C0000D0036004173800000E7200000804000A0
:1052D000104078000004E00013003D00417380009E
:1052E00000E720000080400090407800F0CDB3003F
:1052F00080CF50000C003E00C1FD0700000F780079
:10530000D04080000080A100D04088001E007800BE
:105310006670020000000000D04080000080A00005
:10532000D04088000A0037004173800000E7200069
:105330000080400090407800B0C3B30080CF5000A0
:1053400003003A00407380000000E80040738800CA
:105350004173800000E7200000804000904078000A
:10536000F0CDB30080CF500007003E0041738000B5
:1053700000E72000008040009040780030C8B30073
:1053800080CF50009BFF3A00407380008000E9000E
:1053900000E720000080400090407800B0C3B300D8
:1053A00080CF500009003200D04080000080A10072
:1053B000D040880060922800586E02000000000073
:1053C000D04080000080A000D040880043FC07004F
:1053D000A70237001000200020079800D04080006E
:1053E0000080A100D040880040738000640040002D
:1053F000407388004173800000E720000080400077
:105400009040780020C2B30080CF500018003A00CE
:10541000407380000000E800407388000A003700F5
:105420004173800000E720000080400010407800B9
:10543000004178000100E8004073880002407800D5
:1054400088720200000000004173800000E7200025
:10545000008040009040780020C2B30080CF500010
:10546000EFFF3A00407380000000E80040738800BE
:105470004173800000E720000080400090407800E9
:10548000C0C2B30080CF500004003A0040738000D7
:105490000000E80040738800020037003000200060
:1054A000300798004173800000E720000080400032
:1054B000104078008080FB00F0FB2F00008440004B
:1054C0008001EB00F2FF27008000EB000000EB0002
:1054D0001E1D02000000000000017800880044004A
:1054E00080E02000008040000208780040738000C7
:1054F0000000E80040738800F8FB0700D0408000FF
:105500000080A000D0408800590237001000200021
:1055100020079800407380006400400040738800BA
:1055200050738000E30F500004003C005073800073
:105530000000E8005073880002003700400020009F
:1055400030079800527380004373800000E720000A
:1055500000804100104078008080FB0000FC2F009C
:10556000008240006610B9008080E80000E520005D
:1055700000804000040878000300E80040738800C1
:105580004173800000E720000080400090407800D8
:10559000D0C3B30080CF500011003A0040738000A8
:1055A0000000E80040738800507380006600B90076
:1055B0008080E80000E520000080400010007800B6
:1055C0000004E9000EFD0700000178008800440097
:1055D00080E02000008040000208780002003700D0
:1055E000300020003007980043738000130F9800AC
:1055F00000E720009E089000008040009040780066
:105600000041EB0002579800B0C8B30080CF5000B3
:1056100002003A0013C0B300035798009E089000A0
:105620000100E800407388000E5190000204E00081
:105630000900320058738000F1FC07000001780077
:105640006640B900E400400000E520000080400012
:105650000208780002003700300020003007980070
:105660004173800000E720000080400090407800F7
:10567000F0CDB30080CF500008003600507380009A
:10568000427380006600B9008000780000E52000C9
:10569000008040000208780002003700300020003F
:1056A000300798008DFB0700F10137001000200043
:1056B0002007980040738000640040004073880019
:1056C0004273800000E72000000041001040780095
:1056D0008080FB0000FC2F00008F40000200E800EB
:1056E0004073880050002000300798000000EB0055
:1056F000400798002F0037004E0090006600B90068
:105700008080E80000E52000008040001000780064
:105710009E0F500024003A001E00E9008000400067
:1057200080E0200000804000100178004E009000D2
:105730006600B900E400400000E520000080400061
:1057400010007800800F510012003D009E00E9001B
:105750000181400080E0200000004100100078003E
:105760000001E8008180400080E0200000804000CF
:10577000020878004E0090006600B90080007800B2
:1057800000E5200000804000100078004073880091
:1057900003003700507380000000E9005073880058
:1057A0000000EB00300798004E0090000000E80079
:1057B00040079800517380004E009000810F500008
:1057C000CDFF340045FB0700A90137001000200081
:1057D00020079800407380006400400040738800F8
:1057E000707380000000E00027003A000000EB002A
:1057F000400798000A003700CE00900000E7200024
:1058000000804000104078008080FB004E00900037
:105810008080400030F22F00008040004007980058
:105820004E009000E300400000E7200000804000B0
:1058300090407800E0C8B30080CF500006003200EE
:10584000CE00900000E7200000804000104078006B
:105850000004E000E8FF3A00CE00900000E72000DE
:1058600000804000104078000004E0000400320096
:105870004E00900064004000707388000200370002
:10588000900020003007980043738000030F7800D9
:1058900070738000407388009E00780000E720004D
:1058A00000804000104078008080FB00F0FB2F005B
:1058B0000084400055FB0700000178008800440088
:1058C00080E02000008040000208780040738000E3
:1058D000707388001E00E8004073880071738000B8
:1058E00000E720000080400090407800C0C2B30074
:1058F00080CF500003003A00707380000000E80081
:10590000707388007173800000E720000080400001
:105910009040780000CEB30080CF50000E003600DB
:1059200070738000E300400000E72000008040002A
:1059300090407800E0C8B30080CF500003003200F0
:105940000000EB0070738800030037007073800064
:105950006400400070738800E0FA070044013700DB
:105960001000200020079800417380006E00900016
:105970000080400063004000407388003C01370015
:105980001000200020079800407380006400400051
:1059900040738800A1408000E00220000088B90028
:1059A00080007800E0932000008040001000780024
:1059B00000000100C9FA07002D0137001000200087
:1059C0002007980040738000640040004073880006
:1059D000A1408000E00220000088B9008080E8003B
:1059E000E0932000008040001000780000000100DB
:1059F000BAFA07001E0137001000200020079800A7
:105A0000407380006400400040738800A140800023
:105A1000E00220000088B900E4004000E09320008C
:105A2000008040001000780000000100ABFA070081
:105A30000F013700100020002007980040738000FD
:105A40006400400040738800A1408000E002200014
:105A50000088B900E6004000E0932000008040008C
:105A600010007800000001009CFA070000013700D8
:105A70001000200020079800407380006400400060
:105A800040738800A1408000E00220000088B90037
:105A9000E8004000E09320000080400010047800FF
:105AA000D7FB0700080001008CFA0700F000370060
:105AB0001000200020079800407380006400400020
:105AC00040738800CEFB07000000E00003003200B6
:105AD00056770200000000000200370078770200CD
:105AE000000000007DFA0700E100370010002000F0
:105AF00020079800407380006400400040738800D5
:105B0000BFFB07000000E00005003200C082A900D2
:105B1000C282A800C8A2A900CAA2A8000400370037
:105B2000C082A900C282A900C8A2A900CAA2A90075
:105B30006AFA0700CE003700100020002007980006
:105B4000407380006400400040738800ACFB070095
:105B50000000E0000600320080B82000104078000D
:105B60000000A00081B820008048780005003700C0
:105B700080B82000104078000000A00081B820000C
:105B80008048780055FA0700B9003700100020005F
:105B90002007980040738000640040004073880034
:105BA00097FB070020618800206180000000E00072
:105BB00002003D000000EB002061880021618000B0
:105BC00000FA2000808F50000200340000FA20000C
:105BD0002061880030618000E10F500002003C002D
:105BE00020002000306188003161800030062000F4
:105BF000808F5000020034003006200030618800A1
:105C0000FC7302000000000034FA0700980037001F
:105C100010002000200798004073800064004000BE
:105C20004073880076FB07003061880020618000A7
:105C30000000E00002003D000000EB002061880051
:105C40002161800000FA2000808F500002003400A3
:105C500000FA20002061880030618000E10F5000D0
:105C600002003C002000200030618800316180008B
:105C700030062000808F50000200340030062000E3
:105C800030618800FC7302000000000013FA070076
:105C90007700370010002000200798004073800034
:105CA000640040004073880055FB07000000E000DE
:105CB00009003200A1408000E00220000088B90005
:105CC000F0004000E09320000080400010007800C9
:105CD0000000010008003700A1408000E002200021
:105CE0000088B900F2004000E093200000804000EE
:105CF0001000780000000100F8F907005C00370090
:105D000010002000200798004073800064004000CD
:105D1000407388003AFB0700700798007E009000EF
:105D2000E10F500010003200FE009000E28F5000A2
:105D3000160032007E0190000200E00001003200F7
:105D40001A003700A1408000E00220000088B9005E
:105D5000EE004000E093200000804000100078003A
:105D60000000010011003700A1408000E002200087
:105D70000088B900EC004000E09320000080400063
:105D8000100078000000010008003700A1408000EA
:105D9000E00220000088B900F6004000E0932000F7
:105DA000008040001000780000000100CBF90700DF
:105DB0002F0037001000200020079800407380005B
:105DC0006400400040738800417380006E009000C2
:105DD000008040000000E90040738800BFF9070020
:105DE0002300370010002000200798004073800037
:105DF000640040004073880001FB0700000F78003A
:105E00001E0078003A99020000000000B3F9070074
:105E10001700370010002000200798004073800012
:105E20006400400040738800F5FA0700000F780016
:105E3000A1408000E00220000088B900FC00400082
:105E4000E093200000804000900078001E00780061
:105E500001000100A1F90700050037001000200033
:105E6000300798000200370030002000300798000B
:105E70002E0090000000E00005003A004173800011
:105E80006E00900000804000630040004073880076
:105E90000000EB00200798003E0090000000E000AA
:105EA000CAFB3200D04080000080A100D0408800B2
:105EB0003E009000E10F5000180032006100200009
:105EC000A03A2000D89B0200000000003E00900095
:105ED000667002000000000081002000003B2000EE
:105EE000D89B0200000000005E0090006670020077
:105EF00000000000B1002000803B2000D89B020081
:105F00000000000040738000667002000000000086
:105F100060922800586E0200000000004F047800D4
:105F20000080FA00000006000200FA00000F78006E
:105F300000C2B30088720200000000001E0078005A
:105F40002C6E02000000000000C2B3008872020044
:105F5000000000000080FA00000006000400FA00C3
:105F60000000EB00407388003F0037004173800061
:105F700000E7200000804000904078002147980012
:105F80002E4090000004E000040035002E409000F8
:105F9000887202000000000030003700AE40900020
:105FA00000CEB30080CF50001C0036006092280065
:105FB000586E020000000000407380008000E8007E
:105FC00000E7200000804000104078000080FB00C7
:105FD0004801DD00407380008080E80000E7200079
:105FE00000804000104078000080FB00000041006D
:105FF000000F7800407380000080E8004073880044
:106000001E007800667002000000000000C2B300AD
:1060100088720200000000001000370000C2B300C8
:1060200088720200000000002E4090008080FB007B
:1060300000F82F00008040008000400020B32000C6
:1060400000804000100078002C6E0200000000006C
:1060500000C2B3008872020000000000407380009C
:106060000000E800407388004173800000E72000D2
:1060700000804000104078000004E000BBFF3A00C0
:1060800060922800586E02000000000040738000FB
:106090000000E900667002000000000071002000AE
:1060A000303C2000629C0200000000000080FA00EA
:1060B000000006000600FA001007980050698000F2
:1060C000000F7800170037001E0090001041780084
:1060D0005169800080C2200000804000104078009C
:1060E000804F5100050032001E0078005069880082
:1060F0000000EB0020079800100037005069800076
:106100000000E8005069880051698000F00F20000D
:1061100000806000506988001E0090000000E800C8
:10612000100798001E009000104078000004E00066
:10613000E5FF3A0010002000200798002E00900094
:106140000080FA00000006000400FA000000EB00E6
:10615000000F7800100037001E007800800040001B
:1061600020B320000080400010007800D1FF07001D
:106170000000E000070032001E0078008040780038
:1061800000C8B30000C040000080FB00100798006A
:10619000060037001E0FE800000220009E0F1000CE
:1061A000EDFF34000000EB00100798001E00900087
:1061B0000080FA00000006003600FA0050698000F6
:1061C000000F98001F0037008E08900080C220004A
:1061D000008040009040780000C6B30080CF50009F
:1061E000110034008E08900080C220000080400022
:1061F00090407800A0C7B30080CF50000A003C0058
:106200000E0990008E08900080C22000008040009F
:1062100090407800F0CDB30080C0600080C22000C4
:1062200000004100014878000E0890000000E800DE
:10623000000F98008E089000F00F20000080600092
:10624000000F98008E08900040698000808F5000F9
:10625000DDFF3A000000EB00000F9800516980005C
:1062600080C220000080400090407800F0C2B3005F
:1062700080CF50002C0134005169800080C2200082
:10628000008040009040780090C3B30080CF500061
:1062900025013C000000EB00000F980007003700CC
:1062A0000E099000F20047000040EB0000F178007A
:1062B0000E0890000000E800000F98008E08900083
:1062C00020022000808F5000F5FF3400D21602001B
:1062D00000000000600798006E0090004880DE001B
:1062E0008040780072004700114098006E009000D6
:1062F0008040780000C0EB0080C060007200470062
:10630000214098006E0090008CF80700500798001C
:106310005E009000E10F40002B003200DE00900094
:1063200000E7200000804000104078008080FB00E3
:1063300030F22F0000804000300798005E0090008F
:10634000000F98000D0037000E0990008E08900095
:106350003E0090008080400000E720000080400068
:106360009040780000E720000000410001487800DC
:106370000E0890000000E800000F98000140200087
:106380003E009000808050000E089000808F5000EA
:10639000EDFF3C00080037008E08900000E7200069
:1063A000808040000040EB00804878000E0890009C
:1063B0000000E800000F98008E089000F03F2000D9
:1063C000808F5000F4FF340030002000000F980050
:1063D0000000EB0020079800A81A0200000000004F
:1063E000420037002E0090000000E00002003A005A
:1063F000A81A0200000000002E0090000000E0003B
:1064000004003A0050FF07000080FB00600798007E
:10641000020037000000EB00600798006E0090005B
:106420000000E0000C0032000E0990006E009000A9
:10643000804078007200470001717800EE00900003
:1064400070082000808F50001C003A0010002000CF
:1064500020079800190037005169800080C2200091
:10646000008040009040780020C2B30080CF5000F0
:1064700003003A002E0090000000A20020079800C0
:106480000E0990005169800080C220000080400009
:106490001040780080407800720047000171780059
:1064A000506980000000E800506988005169800050
:1064B000F00F200000806000506988000E089000F6
:1064C0000000E800000F98008E08900030022000C5
:1064D000808F50000500340091002000A03C200077
:1064E000629C020000000000D20037005169800069
:1064F00040698000808F5000BAFF3A000E0890007B
:10650000E30F5000CB0032000E089000E40F500063
:10651000C80032000E08900080407800C0CDB30063
:1065200000C04000804078007200470001487800B9
:106530000000EB00000F98000000EB0040079800FF
:106540000000EB0050079800460037008E089000CE
:1065500000E72000008040009040780000CEB300AB
:1065600080CF50002E0036008E08900000E72000FB
:1065700000804000104078008080FB0000F22F0077
:1065800000804000300798000E0890008000E8006E
:1065900000E7200000804000104078000080FB00F1
:1065A0004801DD000E0890008080E80000E7200030
:1065B00000804000104078000080FB000000410097
:1065C0001007980072004700104090000080FB0008
:1065D000C800DD0072004700204090000080FB00F2
:1065E00000804000000F78001E0090009E0F5000B9
:1065F000050031008E0890003E00900000804000B1
:106600006300400050079800BE0090000E08900004
:106610000080400063004000000F98000200370037
:106620000E089000400798000E0890008000E800D7
:1066300000E7200000804000104078000080FB0050
:106640004801DD000E0890008080E80000E720008F
:1066500000804000104078000080FB0000004100F6
:10666000600798004E0090000000E000B7FF320085
:1066700072004700104078008080FB0030F22F004D
:1066800000804000600798004E009000000F9800C6
:106690000D0037008E0890006E00900000814000D1
:1066A0008E08900000E720000080400090407800B5
:1066B00000E7200000004100014878000E0890002B
:1066C0000000E900000F98008E0890005E00900026
:1066D000808F5000EFFF3D000000EB00000F98009E
:1066E0000C003700DE0090000E0890000081400092
:1066F0008E08900072004700E140780000E720001B
:1067000000004100014878000E0890000000E800F9
:10671000000F98008E0890006E009000808F50004F
:10672000F0FF3500430037007092280061FE07003B
:106730000000E000050032007FF9070060922800A9
:10674000586E0200000000003A003700B0922800A6
:1067500058FE07000000E00002003200FFFD0700C5
:10676000340037000093280052FE07000000E000CC
:1067700004003200D04080000090A100D04088008A
:106780002C003700509328004AFE07000000E0006C
:10679000200032000000EB00000F980018003700C6
:1067A0000000EB00700798000F0037008E08900083
:1067B0007E0090008080400000E7200000804000C4
:1067C000104078000080FB002671020000000000ED
:1067D00000C2B30088720200000000007E0090003A
:1067E0000000E800700798007E009000EF0F500056
:1067F000EEFF34000E08900070004000000F98007B
:106800008E089000F03F2000808F5000E4FF34009D
:1068100008003700B093280026FE07000000E000C3
:1068200004003A00C1002000303D2000629C0200BC
:10683000000000000080FA00000006000200FA00DC
:106840000000EB00000F7800060037009E00780083
:1068500000E72000808040000040EB008048780086
:106860001E0FE800F03F20009E0F1000F7FF3400DD
:1068700011CEB30000E720000148780080C0EB0093
:1068800010E720000148780080C0EB0020E72000DE
:106890000148780011CAB30030E7200001487800B1
:1068A0000080FA00000006005752490054452000BD
:1068B000424954003A2020002A6E65007874200076
:1068C000636C6F00636B2000285E290020776900ED
:1068D0006C6C20007573650020746800697320007B
:1068E00076616C0075653100574952004520720091
:1068F0006F757400696E65007320280043292000BD
:106900003230300030204D006963680061656C00F2
:106910002050650061726300652047004E552000DD
:1069200047504C004E6F2000646576006963650037
:106930002C2074007279200028414C0041524D00F7
:106940002920530045415200434820006D616300F7
:10695000726F2000666972007374410044445200F3
:1069600045535300204D410043524F00202030003A
:106970002E4D610063726F00206D65006E754D00D5
:10698000616372006F2020002020200031574900F1
:10699000524520006164640072657300730D0A0043
:1069A000202020002A3157004952450020524F0034
:1069B0004D2043004F4D4D00414E4400204D4100BD
:1069C00043524F00733A0D000A203500312E520019
:1069D0004541440020524F004D20280030783300BC
:1069E000332920002A666F0072207300696E6700E9
:1069F0006C6520006465760069636500206275003F
:106A0000730D0A00203835002E4D410054434800D4
:106A100020524F004D2028003078350035292000C5
:106A20002A666F006C6C6F007765640020627900E5
:106A3000203634006269740020616400647265006D
:106A400073730D000A20320030342E00534B49007E
:106A5000502052004F4D2000283078004343290039
:106A6000202A66006F6C6C006F77650064206200FE
:106A7000792063006F6D6D00616E64000D0A200067
:106A8000323336002E414C0041524D002053450018
:106A900041524300482028003078450043290D002A
:106AA0000A20320034302E00534541005243480042
:106AB00020524F004D2028003078460030294100F8
:106AC0004C4152004D2053004541520043482000A4
:106AD000283078004543290053454100524348007F
:106AE000202830007846300029446500766963002C
:106AF00065204900447320006172650020617600C2
:106B000061696C0061626C006520620079204D0053
:106B1000414352004F2C200073656500202830004F
:106B2000292E52004541440020524F004D2028009C
:106B30003078330033293A00204D41005443480057
:106B400020524F004D202800307835003529530061
:106B50004B49500020524F004D2028003078430010
:106B6000432955006E6B6E006F776E00206D6100DB
:106B700063726F002C207400727920003F206F0038
:106B80007220280030292000666F7200206865009E
:106B90006C7042005553200052455300455420006C
:106BA000576172006E696E00673A20002A536800D0
:106BB0006F727400206F7200206E6F00207075007D
:106BC0006C6C2D00757020002A4E6F0020646500EB
:106BD0007669630065206400657465006374650010
:106BE000642044005331380053323000204869009B
:106BF00067682000507265007320440069672000B8
:106C000054686500726D44005331380042323000E0
:106C1000205072006F6720005265730020446900A5
:106C200067205400686572006D44530031383200AB
:106C300032204500636F6E002044690067205400D5
:106C4000686572006D4453003234300034204500D2
:106C5000636F6E0072616D00207469006D652000C5
:106C600043686900704453003234330031203100EE
:106C70004B204500455052004F4D55006E6B6E0045
:106C80006F776E0020646500766963006550570079
:106C90004D20640069736100626C650064314B00D3
:106CA000487A2D00342C300030304B00487A2000D8
:106CB00050574D0046726500717565006E6379002E
:106CC00020696E00204B48007A20500072657300E6
:106CD00063616C00653A500052323A0044757400AA
:106CE0007920630079636C00652069006E202500BF
:106CF000205057004D20610063746900766545009F
:106D000052524F00523A200050574D00206163000C
:106D100074697600652C2000672074006F20640081
:106D200069736100626C650041555800204672002D
:106D300065717500656E6300793A20004155580011
:106D400020494E00505554002F4849002D5A41000B
:106D500055582000484947004841550058204C00EC
:106D60004F5756004F4C54004D455400455220009B
:106D70004D4F440045564F004C54410047452000BC
:106D800050524F0042453A002056450072726F0043
:106D90007228290020406C00696E65003A2040008E
:106DA00070676D007370610063653A00206279005E
:106DB000746573002E546F006F206C006F6E670057
:106DC000215379006E7461007820650072726F0043
:106DD000724E6F002045450050524F004D457200E5
:106DE000617369006E6764006F6E650053617600C1
:106DF000696E670020746F0020736C006F74200050
:106E0000496E7600616C6900642073006C6F7400D9
:106E10004C6F610064696E0067206600726F6D00E0
:106E200020736C006F742000455252004F523A009C
:106E300020636F006D6D61006E64200068617300F7
:106E4000206E6F0020656600666563007420680030
:106E50006572650041434B004E4143004B4932008F
:106E600043205300544152005420420049544900E9
:106E70003243200053544F005020420049544900EF
:106E8000324320006D6F6400653A0D000A20310026
:106E90002E2053006F66740077617200650D0A0042
:106EA00020322E0020486100726477006172650014
:106EB0005365740020737000656564003A0D0A0024
:106EC00020312E00207E35004B487A000D0A20002C
:106ED000322E20007E3530004B487A000D0A20000B
:106EE000332E20007E313000304B48007A0D0A00EE
:106EF00020342E00207E340030304B00487A57007A
:106F000041524E00494E47003A2048004152440049
:106F10005741520045204900324320006973200048
:106F200062726F006B656E00206F6E0020746800E7
:106F30006973200050494300212028005245560023
:106F4000204133002953650074207300706565008B
:106F5000643A0D000A2031002E20310030304B0001
:106F6000487A0D000A2032002E20340030304B00C9
:106F7000487A0D000A2033002E2031004D487A0057
:106F80004932430020286D006F6420007370640054
:106F9000293D2800202030002E4D610063726F00D3
:106FA000206D65006E750D000A2031002E376200DD
:106FB000697420006164640072657300732073005B
:106FC0006561720063680D000A2032002E493200AC
:106FD000432073006E696600666572005365610048
:106FE00072636800696E67002049320043206100C7
:106FF00064647200657373002073700061636500E0
:107000002E2046006F756E0064206400657669006E
:1070100063657300206174003A536E006966660010
:1070200065722800424153004943290052656100BE
:10703000647961002F412F00402063006F6E74005F
:10704000726F6C00732041005558200070696E000B
:10705000612F41002F402000636F6E0074726F003B
:107060006C7320004353200070696E00436F6D0005
:107070006D616E0064206E006F7420007573650092
:10708000642069006E20740068697300206D6F00D1
:1070900064655000756C6C002D7570002072650081
:1070A00073697300746F720073204F00464650007E
:1070B000756C6C002D75700020726500736973002B
:1070C000746F720073204F004E5365006C662D0084
:1070D00074657300742069006E204800695A2000AE
:1070E0006D6F640065206F006E6C7900524553002F
:1070F000455442004F4F54004C4F4100444552000C
:107100004155580020494E00505554002F48490021
:107110002D5A2C002052450041443A0020506F0067
:10712000776572002073750070706C00696573007C
:10713000204F4E00506F770065722000737570000D
:10714000706C6900657320004F464600444154004E
:107150004120530054415400453A200044454C001E
:10716000415920007573570052495400453A200098
:1071700052454100443A2000434C4F00434B2C0001
:10718000203143004C4F43004B2C20003044410041
:10719000544120004F555400505554002C203100CC
:1071A0004441540041204F005554500055542C0088
:1071B000203020002A7069006E20690073206E0064
:1071C0006F77200048695A00434C4F00434B200022
:1071D000544943004B533A0020524500414420009B
:1071E000424954003A205300796E740061782000BF
:1071F000657272006F722000617420006368610024
:10720000722078002E206500786974002877690064
:1072100074686F0075742000636861006E676500B4
:10722000296E6F00206D6F00646520006368610047
:107230006E6765004E6F6E00657869007374650057
:107240006E74200070726F00746F63006F6C2100A9
:10725000782E200065786900740D0A00496E76006A
:10726000616C690064206300686F690063652C00CD
:107270002074720079206100676169006E444500E6
:10728000564944003A68740074703A002F2F640025
:10729000616E670065726F0075737000726F7400C5
:1072A0006F747900706573002E636F006D2A2D0076
:1072B0002D2D2D002D2D2D002D2D2D002A4F700050
:1072C000656E200064726100696E20006F75740045
:1072D0007075740073202800483D4800692D5A00DD
:1072E0002C204C003D474E0044294E006F726D002B
:1072F000616C20006F757400707574007320280035
:10730000483D33002E3376002C204C003D474E0084
:1073100044294D0053422000736574003A204D000B
:107320004F53540020736900672062006974200085
:107330006669720073744C005342200073657400D8
:107340003A204C00454153005420730069672000E7
:1073500062697400206669007273740020426F00D5
:107360006F746C006F6164006572200076203100DC
:107370002E20480045580D000A2032002E204400DF
:1073800045430D000A2033002E204200494E0D00D7
:107390000A2034002E2052004157440069737000C7
:1073A0006C61790020666F00726D6100742073005B
:1073B000657456006F6C740061676500206D6F0026
:1073C0006E6974006F7273003A203500563A2000DF
:1073D000207C2000332E3300563A2000207C2000F1
:1073E000565055004C4C5500503A200053657400DF
:1073F00020736500726961006C2070006F72740008
:1074000020737000656564003A2028006270730084
:10741000290D0A0020312E0020333000300D0A00E3
:1074200020322E002031320030300D000A2033008F
:107430002E203200343030000D0A2000342E20007F
:1074400034383000300D0A0020352E002039360047
:1074500030300D000A2036002E2031003932300045
:10746000300D0A0020372E00203338003430300031
:107470000D0A2000382E20003537360030300D0040
:107480000A2039002E2031003135320030300D0015
:107490000A3130002E2042005247200072617700EE
:1074A000207661006C75650041646A007573740034
:1074B00020796F0075722000746572006D696E002E
:1074C000616C410072652000796F75002073750052
:1074D00072653F002043460047313A002043460092
:1074E00047323A00285C2D002F5F5C002D292800D0
:1074F0005C5F2F002D295300656C650063742000CC
:107500006F757400707574002074790070653A00AE
:107510000D0A2000312E20004F7065006E2064009F
:10752000726169006E202800483D4800692D5A00AC
:107530002C204C003D474E0044290D000A2032000B
:107540002E204E006F726D00616C200028483D00B7
:10755000332E3300562C20004C3D47004E4429006A
:1075600052325700202873007064200068697A0046
:10757000293D2800202030002E4D610063726F00ED
:10758000206D65006E750D000A2031002E495300F4
:107590004F37380031362D003320410054520D0052
:1075A0000A2032002E4953004F37380031362D0063
:1075B000332070006172730065206F006E6C79007B
:1075C00049534F002037380031362D003320410019
:1075D000545220002852450053455400206F6E003D
:1075E00020435300290D0A00524553004554200002
:1075F00048494700482C2000434C4F00434B200093
:10760000544943004B2C2000524553004554200060
:107610004C4F570049534F002037380031362D006A
:107620003320720065706C00792028007573650046
:107630007320630075727200656E7400204C5300F5
:107640004220730065747400696E6700293A200057
:1076500050726F00746F63006F6C3A0020736500A6
:10766000726961006C332000776972006532200016
:10767000776972006552460055756E006B6E6F003B
:10768000776E5200656164002074790070653A007D
:1076900020746F0020656E0064766100726961007D
:1076A000626C6500206C65006E6774006844610060
:1076B00074612000756E690074733A00206E6F006B
:1076C00020696E0064696300617469006F6E440034
:1076D0006174610020756E00697420006C656E0035
:1076E000677468002028620069747300293A2000DA
:1076F00043532000454E4100424C45004443530053
:1077000020444900534142004C4544005233570045
:10771000202873007064200063736C002068690087
:107720007A293D00282029000D0A4400697363006E
:107730006F6E6E006563740020616E0079206400D6
:1077400065766900636573000D0A43006F6E6E0015
:10775000656374002028560070752000746F200047
:107760002B355600292061006E642000284144001A
:10777000432074006F202B00332E33005629430022
:1077800074726C00415558004D4F440045204C0028
:1077900045445000554C4C00555020004850550071
:1077A0004C4C55005020480056524500474144007B
:1077B000432061006E64200073757000706C790066
:1077C00035565600505533002E3356004144430081
:1077D0004275730020686900676842007573200075
:1077E00048692D005A203000427573002048690016
:1077F0002D5A2000314D4F0044452000616E640039
:1078000020565200454720004C4544007320730029
:10781000686F75006C642000626520006F6E210047
:10782000466F75006E64200020657200726F7200F2
:10783000732E4D004F534900434C4B004D495300AC
:107840004F435300204F4B0020464100494C53000A
:10785000657420007370650065643A000D0A2000AD
:10786000312E200033304B00487A0D000A203200C0
:107870002E20310032354B00487A0D000A203300AB
:107880002E20320035304B00487A0D000A2034009B
:107890002E2031004D487A00436C6F00636B20004E
:1078A000706F6C006172690074793A000D0A2000F3
:1078B000312E200049646C0065206C006F77200039
:1078C0002A646500666175006C740D000A20320040
:1078D0002E204900646C65002068690067684F00CD
:1078E0007574700075742000636C6F00636B20000A
:1078F00065646700653A0D000A2031002E204900BA
:10790000646C650020746F00206163007469760008
:10791000650D0A0020322E00204163007469760054
:10792000652074006F206900646C6500202A640083
:1079300065666100756C7400496E70007574200096
:1079400073616D00706C6500207068006173650084
:107950003A0D0A0020312E00204D690064646C004D
:1079600065202A006465660061756C00740D0A006C
:1079700020322E0020456E0064535000492028001C
:107980007370640020636B00702073006B652000CF
:10799000736D7000206373006C206800697A2900A1
:1079A0003D28200020302E004D616300726F2000C2
:1079B0006D656E00750D0A0020312E00536E690052
:1079C00066662000435320006C6F77000D0A20008C
:1079D000322E53006E696600662061006C6C2000D8
:1079E0007472610066666900632D7000202D660068
:1079F000202A42007974650073206400726F700061
:107A0000706564002A464100494C4500442C200022
:107A10004E4F2000444154004144610074612000F5
:107A200062697400732061006E64200070617200EE
:107A3000697479003A0D0A0020312E0020382C009C
:107A4000204E4F004E4520002A6465006661750097
:107A50006C7420000D0A2000322E2000382C2000EB
:107A6000455645004E200D000A2033002E203800D8
:107A70002C204F00444420000D0A2000342E20000A
:107A8000392C20004E4F4E00455374006F7020007B
:107A900062697400733A0D000A2031002E20310013
:107AA000202A640065666100756C74000D0A200070
:107AB000322E200032526500636569007665200031
:107AC000706F6C006172690074793A000D0A2000D1
:107AD000312E200049646C0065203100202A6400AA
:107AE00065666100756C74000D0A2000322E20005E
:107AF00049646C0065203000554152005420280034
:107B0000737064002062720067206400627020005D
:107B10007362200072787000206869007A293D0045
:107B200028202000302E4D00616372006F206D0010
:107B3000656E75000D0A2000312E540072616E00D2
:107B40007370610072656E00742062007269640077
:107B500067650D000A2032002E204C006976650012
:107B6000206D6F006E6974006F720D000A20330083
:107B70002E427200696467006520770069746800AE
:107B800020666C006F772000636F6E0074726F0068
:107B90006C554100525420006272690064676500B0
:107BA0005265730065742000746F20006578690069
:107BB00074526100772055004152540020696E00D4
:107BC000707574005541520054204C0049564500D0
:107BD0002044490053504C0041592C00207D200086
:107BE000544F200053544F00504C4900564520003C
:107BF00044495300504C410059205300544F500009
:107C000050454400574152004E494E00473A20002B
:107C100070696E0073206E006F7420006F706500D5
:107C20006E206400726169006E20280048695A0065
:107C30002920520045564900443A0D000A496E0079
:107C400076616C006964200063686F006963650099
:107C50002C2074007279200061676100696E6D00EC
:107C600073525300204C4F00572C2000434F4D00BF
:107C70004D414E0044204D004F44450052532000DA
:107C800048494700482C20004441540041204D0001
:107C90004F444500416464007265730073206F00B7
:107CA0006620500043463800353734003F546800A2
:107CB000697320006D6F6400652072006571750046
:107CC00069726500732061006E206100646170005C
:107CD000746572004C4344002074790070653A006A
:107CE0000D0A2000312E200048443400343738007B
:107CF00030202800757369006E67200050434600ED
:107D000038353700342049004F2065007870610015
:107D10006E64650072294C00434420002874790089
:107D2000702061006464720029203D00202820003A
:107D300020302E004D616300726F20006D656E0073
:107D4000750D0A0020312E004C434400205265007E
:107D5000736574000D0A2000322E49006E697400AC
:107D6000204C4300440D0A0020332E00436C650074
:107D7000617220004C4344000D0A2000342E430061
:107D8000757273006F722000706F73006974690000
:107D90006F6E200065783A002834290020300D00ED
:107DA0000A2036002E577200697465002074650041
:107DB000737420006E756D0062657200732065003B
:107DC000783A28003629200038300D000A20370084
:107DD0002E5772006974650020746500737420006A
:107DE00063686100726163007465720073206500EE
:107DF000783A280037292000383044006973700031
:107E00006C617900206C69006E6573003A0D0A00A0
:107E100020312E00203120000D0A2000322E2000BB
:107E20004D756C00746970006C6549004E495400D2
:107E3000434C450041524300555253004F522000DD
:107E4000534554004E6F200041434B002C206300EB
:107E5000686563006B206100646170007465720086
:107E6000434C4B00094D4F0053490900435309004F
:107E70004D4953004F5069006E7374006174650082
:107E8000733A47004E440900332E3300560935003B
:107E90002E30560009414400430956005055090050
:107EA000415558000950090050095000094909007E
:107EB00049092D00094F570044092D00092D2D00B7
:107EC0000954780044092D000952780044534300B6
:107ED0004C095300444109002D092D00504743002F
:107EE0000950470044092D00092D31002E28420079
:107EF00052290900322E28005244290009332E004D
:107F0000284F5200290934002E285900572909000A
:107F1000352E2800474E290009362E0028424C00F5
:107F2000290937002E28500055290900382E28002D
:107F30004752290009392E002857540029093000DA
:107F40002E2842006C6B2900474E440009474E0022
:107F50004409410044430900352E300056093300DE
:107F60002E33560009565000550941005558090056
:107F7000657865006375740065203A002020540020
:107F8000494D45004F55540020302E00204D6100D2
:107F900063726F00206D65006E750D000A20310060
:107FA0002E204C006976650020696E0070757400A3
:107FB000206D6F006E6974006F7249006E707500FD
:107FC00074206D006F6E6900746F7200202A730058
:107FD00074617200746269007420650072726F00CF
:107FE00072202A0070617200697479002065720045
:107FF000726F7200202A7300746F700062697400DF
:1080000020657200726F7200204E4F004E452000B6
:10801000554E4B004E4F57004E20450052524F00D8
:108020005220610075746F0072616E0067652000F8
:108030002B4D48007A292B006B487A0029526100A9
:1080400077207600616C7500652066006F722000F5
:108050004252470020284D00494449003D3132003A
:108060003729570041524E00494E47003A205000F0
:108070006F73730069626C0065206200756666004C
:1080800065726F0076657200666C6F0077416E00F6
:1080900079206B0065792000746F20006578690095
:1080A000745370006163650020746F0020636F007B
:1080B0006E7469006E7565004E756D0062657200C4
:1080C000206F660020626900747320007265610091
:1080D000642F770072697400653A200043533A00B8
:1080E0000D0A2000312E200043530D000A203200DB
:1080F0002E202F00435320002A646500666175001E
:108100006C7450006F73690074696F006E206900B1
:108110006E206400656772006565730053657200C8
:10812000766F2000616374006976650047656E00B4
:10813000657261006C0909000909090050726F003D
:10814000746F63006F6C2000696E7400657261006B
:10815000637469006F6E2D002D2D2D002D2D2D00C7
:108160002D2D2D002D2D2D002D2D2D002D2D2D00F3
:108170002D2D2D002D2D2D002D2D2D002D2D2D00E3
:108180002D2D2D002D2D2D002D2D2D002D2D2D00D3
:108190002D2D2D002D2D2D002D2D2D002D2D2D00C3
:1081A0002D2D2D002D2D2D002D2D2D002D2D2D00B3
:1081B0002D2D2D002D2D2D002D2D3F000954680053
:1081C0006973200068656C00700909000928300097
:1081D00029094C0069737400206375007272650090
:1081E0006E7420006D616300726F73003D582F0044
:1081F0007C580900436F6E0076657200747320002E
:10820000582F72006576650072736500205809006A
:108210000928780029094D00616372006F207800F9
:108220007E095300656C660074657300740909006B
:10823000095B0900537461007274230009526500E0
:108240007365740009090900095D090053746F0022
:10825000702409004A756D00702074006F20620060
:108260006F6F74006C6F61006465720009097B00B8
:1082700009537400617274002077690074682000EB
:108280007265610064262F0025094400656C610059
:1082900079203100207573002F6D730009090900E2
:1082A0007D095300746F7000612F41002F40090059
:1082B0004155580050494E0020286C006F772F0020
:1082C00048492F0052454100442909000922610014
:1082D00062632200095365006E64200073747200AB
:1082E000696E670062095300657420006261750061
:1082F000647261007465090009093100323363005A
:108300002F430900415558002061730073696700CD
:108310006E6D65006E74200028617500782F430033
:10832000532909000930780031323300642F4400AA
:10833000094D65006173750072652000414443007A
:1083400020286F006E6365002F434F004E542E00AF
:10835000290930006231310030095300656E640034
:10836000207661006C75650066094D0065617300DB
:10837000757265002066720065717500656E630038
:10838000790909007209520065616400672F530082
:10839000094765006E6572006174650020505700E2
:1083A0004D2F5300657276006F0909002F094300B5
:1083B0004C4B20006869680009436F006D6D6100D7
:1083C0006E646800697374006F72790009090900AE
:1083D0005C0943004C4B20006C6F69000956650036
:1083E000727369006F6E69006E666F002F737400A0
:1083F0006174750073696E00666F0900095E09009B
:10840000434C4B0020746900636B6C002F4C0900D7
:10841000426974006F72640065722000286D7300F9
:10842000622F4C005342290009092D0009444100E4
:1084300054206800696D0900436861006E6765003B
:10844000206D6F006465090009095F00094441005F
:1084500054206C006F6F090053657400206F750025
:108460007470750074207400797065000909090042
:108470002E094400415420007265610064702F0091
:1084800050095000756C6C007570200072657300A7
:10849000697374006F72730020286F0066662F0086
:1084A0004F4E2900092109004269740020726500BD
:1084B0006164730009536300726970007420650081
:1084C0006E6769006E65090009093A000952650086
:1084D00070656100742065002E672E0020723A00DE
:1084E00031307600095368006F772000766F6C009A
:1084F00074732F00737461007465730009093B0085
:108500000942690074732000746F20007265610075
:10851000642F770072697400652065002E672E0055
:108520002030780035353B0032772F005709500056
:1085300053552000286F6600662F4F004E29090012
:10854000093C78003E2F3C00783D20003E2F3C0047
:10855000303E090055736500726D610063726F00F3
:1085600020782F006173730069676E0020782F00F8
:108570006C697300742061006C6C00000000FA00EC
:1085800080B82000104078000050A00081B8200082
:108590008048780080B92000104078006840600072
:1085A0000004E00002003200CAC2A9000100370046
:1085B000CAC2A80080B9200010407800684060005E
:1085C0000004E00003003200F0C2B3008872020031
:1085D00000000000A100200060AB2000629C0200AF
:1085E000000000000080FA00000006000000FA0011
:1085F00080B82000104078000050A10081B8200011
:108600008048780080B92000104078006840600001
:108610000004E00002003200CAC2A90001003700D5
:10862000CAC2A80080B920001040780068406000ED
:108630000004E00003003200F0C2B30088720200C0
:1086400000000000A100200060AB2000629C02003E
:10865000000000000080FA00000006000000FA00A0
:1086600080B9200010407800684060000004E000FD
:1086700002003200CAC2A80001003700CAC2A90025
:1086800080B9200010407800684060000004E000DD
:1086900003003200F0C2B300887202000000000044
:1086A000B100200000AC2000629C0200000000002D
:1086B0000080FA00000006000000FA0000C0EB0095
:1086C000820207000080FB000080FA000000060024
:1086D0000600FA00100798001E0090007B020700B9
:1086E000004F780080B82000104078000042B200AF
:1086F0000004E000030032001E80FB002007980009
:1087000001003700010037002E0090000080FA00C1
:10871000000006000000FA0001022000D0C920007D
:10872000D89B02000000000060B7200010407800D5
:108730000040E800C47002000000000000C2B30066
:10874000887202000000000080B92000104078000C
:1087500061406000C47002000000000000C2B3006D
:10876000887202000000000080B9200010407800EC
:108770000080FB000000D10061406000C470020076
:108780000000000000C2B300887202000000000078
:1087900080B92000104078000080FB004200DE001D
:1087A00061406000C47002000000000000C2B3001D
:1087B000887202000000000080B92000104078009C
:1087C0000080FB004300DE0061406000C4700200D6
:1087D0000000000000C2B300887202000000000028
:1087E00080B82000104078000080FB004300DE00CD
:1087F00061406000C47002000000000000C2B300CD
:10880000887202000000000031002000F0AD20005E
:10881000D89B0200000000000080FA000000060063
:108820000C00FA00A81A020000000000D216020094
:108830000000000050079800A81A02000000000085
:10884000D21602000000000040079800A81A02009B
:1088500000000000D216020000000000300798005F
:10886000A81A020000000000D2160200000000005A
:1088700020079800A81A020000000000D21602008B
:1088800000000000000F7800A81A0200000000009D
:10889000D216020000000000100798005E00900051
:1088A0000000E000090034005E009000E40F50007A
:1088B00006003C005E0090000040E9008040780027
:1088C00060B7200001487800020037000000EB008C
:1088D000500798004E0090000000E0000F003400A8
:1088E0004E009000E20F50000C003C004E00900043
:1088F0000040E900E140600080B9200010407800AD
:1089000061C16000E1CFB30001406000024070002F
:1089100081B9200080487800020037000000EB0099
:10892000500798003E0090000000E0001000340066
:108930003E009000E20F50000D003C003E00900011
:108940000040E9006141600080B92000904078005B
:108950006140610000414000D0CFB30080C06000A2
:1089600082C0700080B92000014878000200370002
:108970000000EB00500798002E0090000000E0007F
:10898000100034002E009000E20F50000D003C005B
:108990002E0090000040E9006141600080B9200095
:1089A00090407800614061004201DD00B0CFB3002B
:1089B00080C0600082C0700080B92000014878004B
:1089C000020037000000EB00500798001E00E00096
:1089D00010003400200020009E0F10000D003C000D
:1089E0001E0078000040E9006141600080B920006D
:1089F00090407800614061004301DD0070CFB3001A
:108A000080C0600082C0700080B9200001487800FA
:108A1000020037000000EB00500798001E00900095
:108A20000000E000100034001E009000E20F500033
:108A30000D003C001E0090000040EA006141600013
:108A400080B8200090407800614061004301DD0063
:108A500070CFB30080C0600082C0700080B820007A
:108A600001487800020037000000EB005007980032
:108A70005E0090000000E00079003A000000EB008A
:108A80006069880071032000D0BB2000629C020056
:108A9000000000008001EB004200200011002000D7
:108AA000100020001E1D0200000000000040E90030
:108AB0008040780060B72000014878005103200012
:108AC00040BF2000629C0200000000008001EB001B
:108AD0002200200011002000100020001E1D0200B6
:108AE000000000000040E900E140600080B9200083
:108AF0001040780061C16000E1CFB3000140600028
:108B00000240700081B920008048780031042000C4
:108B100090C22000629C0200000000008001EB0077
:108B20002200200011002000200020001E1D020055
:108B3000000000000040E9006141600080B92000B1
:108B4000904078006140610000414000D0CFB30008
:108B500080C0600082C0700080B9200001487800A9
:108B600011032000C0C62000629C0200000000002B
:108B70008001EB00220020001100200010002000E6
:108B80001E1D0200000000000040E900614160007D
:108B900080B9200090407800614061004201DD0012
:108BA000B0CFB30080C0600082C0700080B92000E8
:108BB00001487800D101200070222100629C02004F
:108BC000000000008001EB002200200011002000C6
:108BD000200020001E1D0200000000000040E900EF
:108BE0006141600080B920009040780061406100E0
:108BF0004301DD0070CFB30080C0600082C0700010
:108C000080B9200001487800F1042000B0932000D2
:108C1000629C0200000000008001EB0022002000A6
:108C200011002000100020001E1D020000000000A6
:108C30000040EA006141600080B820009040780068
:108C4000614061004301DD0070CFB30080C060006F
:108C500082C0700080B82000014878000100370011
:108C6000ACFE070080B82000104078000050A10042
:108C700081B820008048780060B72000104078005C
:108C80008080FB00E08120000080400010407800E0
:108C9000A600070080B92000104078000080FB008B
:108CA0004300DE0061406000614060004601DD007D
:108CB000A12C200091407800F0CBB30000C06000F0
:108CC00002407000CAE2B7000080FA00000006000F
:108CD0000000FA00E90007000080FA00000006002A
:108CE0000600FA00000F78001E0078006101B8004D
:108CF0001207980023079800F000200001002000D0
:108D00001E019000AE019000800F5100818F59002C
:108D100079003E001E009000AE009000006001004F
:108D20000F003700130037001E00370076003700B1
:108D300071003700700037006F0037006E00370099
:108D40006D0037006C003700220037002700370025
:108D50002C00370031003700360037003B00370069
:108D600041032000D0CB2000629C020000000000E4
:108D7000650037007100200050592000629C0200FD
:108D800000000000F1002000C01E2100629C0200D3
:108D90000000000011C0B3000040EB00D900070044
:108DA000590037007100200050592000629C0200D9
:108DB00000000000F1002000C01E2100629C0200A3
:108DC0000000000011C0B30010C0B300CD000700C8
:108DD0004D00370080B92000104078000000A1004D
:108DE00081B92000804878001D00370080B920003C
:108DF000104078000000A00081B920008048780071
:108E00001700370080B92000104078000010A10042
:108E100081B92000804878001100370080B9200017
:108E2000104078000010A00081B920008048780030
:108E30000B00370080B92000104078000020A1000E
:108E400081B92000804878000500370080B92000F3
:108E5000104078000020A00081B9200080487800F0
:108E600080B92000104078006140600061406000DF
:108E70004601DD002124200091407800F0CBB300B2
:108E800000C060000240700042E2B70080B92000DC
:108E9000104078000080FB000000D10061406000BD
:108EA000614160003124200091407800E0CFB300A0
:108EB00000C060000240700043E2B70080B92000AB
:108EC000104078000080FB004200DE00614060003E
:108ED0006140600000414000312420009140780052
:108EE000D0CFB30000C060000240700043E2B70082
:108EF00008FE07000400370041022000C0202000C7
:108F0000629C0200000000000080FA0000000600E1
:108F10000000FA0001012000A0042100629C020070
:108F2000000000000080FA00000006000200FA00C5
:108F3000004F780041E2A90080B82000104078007E
:108F4000684060000004E00004003200CEE2A800A7
:108F5000CF02A800CEC2A80003003700CEE2A900CD
:108F6000CF02A900CEC2A900816A200091407800FA
:108F700000CEB30000C060007040B300A8E6B700A8
:108F8000916C20009140780000CEB30000C06000DA
:108F90007040B300C9E6B700816C200091407800B2
:108FA00000CEB30000C060000034A000C8E6B700E7
:108FB000CAC2A800C8C2A900C902A900C8E2A80084
:108FC000C922A9001E80FB001012880042A2A8003E
:108FD00080B920001040780061406000614060006E
:108FE0004601DD002124200091407800F0CBB30041
:108FF00000C060000240700042E2B70080B920006B
:10900000104078000080FB000000D100614060004B
:10901000614160003124200091407800E0CFB3002E
:1090200000C060000240700043E2B70080B9200039
:10903000104078000080FB004200DE0061406000CC
:1090400061406000004140003124200091407800E0
:10905000D0CFB30000C060000240700043E2B70010
:109060000000EB00201288000000EB0000128800D6
:1090700041E2A8000080FA00000006000000FA00AB
:1090800041E2A900A8C6BF00F041B300A8E6B700BE
:10909000916C20009140780000CEB30000C06000C9
:1090A000C9E6B700816C20009140780000CEB30083
:1090B00000C06000C8E6B700CEE2A900CF02A90058
:1090C000CEC2A9000080FA00000006000200FA00EB
:1090D000004F78001E80FB004012880085C0BF0052
:1090E000644060000004E000FCFF32004012800099
:1090F000004F78008540A9001E80FB000080FA0028
:10910000000006000400FA0020479800314798004C
:1091100010C0B300004F7800307302000000000060
:10912000D6FF0700850007002E4090000004E000F5
:1091300002003A0042E2A80062E2A8002E4090003D
:10914000E14F500002003E0041E2A80061E2A800A9
:109150001E04E00009003A00CAC2BF000044B20089
:109160000004E00005003200D0C5B30044730200E3
:109170000000000010C0B300004F780040C2BF00E4
:109180000042B2000004E0002F003A0060C2BF00BD
:109190000042B2000004E0002B003A0040128000C0
:1091A0001047980010C0B3009E4F100005003A0011
:1091B000B0C5B30044730200000000000040EB00A3
:1091C000004F78003E4090000004E00005003200AF
:1091D0001E4090000080FB00507102000000000063
:1091E00006003700C0C5B300447302000000000051
:1091F0001E409000447302000000000040138000F5
:10920000104798003E4090000004E0000B00320040
:1092100080C2B30044730200000000001E409000B2
:109220000080FB00507102000000000090C2B300FB
:109230004473020000000000030037001E4090004D
:10924000447302000000000040C2BF000044B200AE
:109250000004E00009003A0060C2BF000044B20010
:109260000004E00005003A00D040800001402000EA
:10927000010060000000E00014003200D0408000D7
:1092800001402000010060000000E00002003A0000
:10929000AC730200000000000000EB000012880028
:1092A0000000EB00001388003E4090000004E00046
:1092B00004003200A09F2800586E02000000000049
:1092C00093FF3700CA82A9001200370023C2BF00F3
:1092D000624060000004E00002003A007A7302007D
:1092E0000000000022C2BF00614060000004E000F6
:1092F00097FF320030118000104798003E409000E8
:109300000004E00003003200B0A02800586E020004
:10931000000000008800070060B7200010407800BF
:109320008080FB00E0812000008040001040780039
:10933000FEFE07000080FA00000006000000FA00B0
:10934000C8C2A800C902A800C8E2A800C922A80093
:10935000A16A20009140780000CEB30000C06000F8
:109360006040B300AAE6B700E16A200091407800AF
:1093700000CEB30000C060006040B300AEE6B700AE
:10938000816A20009140780000CEB30000C06000E8
:109390009040B300A8E6B700916A200091407800A1
:1093A00000CEB30000C060000034A000A9E6B70002
:1093B000C16A20009140780000CEB30000C0600078
:1093C0007040B300ACE6B700D16A2000914078004D
:1093D00000CEB30000C060000034A000ADE6B700CE
:1093E00060B72000104078008080FB00E081200002
:1093F00000804000104078000080FB0010128800C0
:1094000080B9200010407800614060006140600039
:109410004601DD002124200091407800F0CBB3000C
:1094200000C060000240700042E2B70080B9200036
:10943000104078000080FB000000D1006140600017
:10944000614160003124200091407800E0CFB300FA
:1094500000C060000240700043E2B7000000EB0073
:10946000201288000000EB000012880060B7200086
:10947000104078008080FB00E081200000804000E8
:10948000104078000080FB001013880080B9200095
:109490001040780061406000614060004601DD00DE
:1094A0002126200091407800F0CBB30000C060007E
:1094B0000240700062E2B70080B9200010407800DE
:1094C0000080FB000000D10061406000614160004D
:1094D0003126200091407800E0CFB30000C060004A
:1094E0000240700063E2B7000000EB002013880028
:1094F0000000EB00001388000000EB004012880021
:109500000000EB00401388004322A9006322A90059
:109510004362A80042A2A9006362A80062A2A90057
:1095200040C2A90060C2A9004402A8006402A800C9
:109530000080FA00000006000000FA0041E2A900E5
:109540004362A90061E2A9006362A900AAC6BF0044
:10955000F041B300AAE6B700AEC6BF00F041B300C9
:10956000AEE6B700A8C6BF00F041B300A8E6B7005A
:10957000A9C6BF00F041B300A9E6B700ACC6BF0062
:10958000F041B300ACE6B700ADC6BF00F041B30098
:10959000ADE6B7000080FA00000006000000FA0007
:1095A000C0A028002C6E0200000000000080FA001D
:1095B000000006000A00FA00881F780011C0B300FE
:1095C00060B720000148780080B920001040780082
:1095D0000000A10081B920008048780080B92000F7
:1095E000104078000010A00081B920008048780069
:1095F00080B92000104078000020A10081B920002F
:109600008048780080B82000104078000030A0002A
:1096100081B820008048780060B7200010407800B2
:109620008080FB00208220000080400010407800F5
:109630003EFE0700D9FF07000000370022C2BF002E
:10964000614060000004E000FCFF32003011800047
:109650008040780060B920000148780060B920009F
:10966000104078000080FB004400DE00804078005D
:1096700050B920000148780050B92000104078000F
:109680000080FB00400798004E009000E40F50005F
:10969000EF0032004E009000E40F500007003C0045
:1096A0004E0090000000E0000B0032004E009000E1
:1096B000E10F5000C0003200510137004E00900011
:1096C000E60F5000EA0032004E009000E80F500014
:1096D000FC0032004A01370060B9200010407800D9
:1096E0000080FB00300798003E009000E30F500020
:1096F000230032003E009000E30F50000A003C00BF
:109700003E009000E10F5000130032003E00900038
:10971000E10F500012003C003E0090000000E0000D
:109720000B003200A00037003E009000ED0F50000B
:109730001B0032003E009000EE0F50001F00320070
:109740003E009000E40F50002300320096003700E6
:109750004AFE07002E01370090FF0700B7FF3700D1
:1097600060168000F1FB2F00010060006016880089
:1097700010C0B3008872020000000000AFFF370085
:10978000601680000104200001007000601688004F
:1097900010C0B3008872020000000000A7FF37006D
:1097A00010C0B30088720200000000008040EB008F
:1097B00010C0B30053FE0700A0FF370010C0B30075
:1097C00088720200000000008040EB000040EB00C7
:1097D0004CFE070099FF370022C2BF0061406000C5
:1097E0000004E000FCFF32003011800010079800F8
:1097F0001E0090004800DD001007980022C2BF0044
:10980000614060000004E000FCFF32003011800085
:109810009E009000008070001007980022C2BF00D8
:10982000614060000004E000FCFF32003011800065
:10983000000F78001E0078004800DD00000F78005F
:1098400022C2BF00614060000004E000FCFF320063
:10985000301180001E0F70009E009000F0FF20006D
:10986000808F500003003E00F0FF20009E0F10008C
:10987000040036000040EB00887202000000000087
:109880006EFF37000000EB00200798000C00370047
:1098900022C2BF00614060000004E000FCFF320013
:1098A000714080002E0090008080400030118000C8
:1098B000804878002E0090000000E8002007980003
:1098C000AE0090001E009000808F5000F0FF390025
:1098D000CAC2A9000000EB0020079800080037006A
:1098E000714080002E009000008040001040780001
:1098F000F6FD07002E0090000000E8002007980009
:10990000AE0090001E009000808F5000F4FF3900E0
:109910001000200066990200000000000000EB002B
:109920002007980009003700714080002E00900049
:109930000084400000C0EB00E4FD0700004C78000C
:109940002E0090000000E800200798002E009000F4
:109950009E0F5000F4FF3900CAC2A80010C0B30027
:1099600088720200000000000000EB002007980051
:1099700009003700714080002E00900000804000F8
:109980001040780088720200000000002E00900055
:109990000000E800200798002E0090009E0F500065
:1099A000F4FF390025FF37000040EB008872020009
:1099B0000000000021FF370060B9200090407800CF
:1099C000F0C0B30080C0600060B92000014878009A
:1099D00060B92000104078008040E80060B92000A5
:1099E0000148780010C0B300887202000000000037
:1099F0008040EB0040B92000014878000D0037009E
:109A000022C2BF00614060000004E000FCFF3200A1
:109A100030118000ADFD07008872020000000000D8
:109A200040B92000104078008040E80040B9200094
:109A30000148780040B920009040780060B92000CB
:109A40001040780080CF5000EDFF3900FBFE37005A
:109A500060B9200010407800B89E020000000000AD
:109A600010C0B3008872020000000000F3FE37004F
:109A700060B920009040780070C0B30080C06000E2
:109A800060B920000148780060B92000904078005B
:109A900060B720000148780060B7200010407800CF
:109AA0008080FB0020822000008040001040780071
:109AB0001EFD070010C0B300887202000000000005
:109AC000DEFE370080B92000104078000000A100C1
:109AD00081B920008048780080B9200010407800CB
:109AE0000010A10081B920008048780080B92000D2
:109AF000104078000020A10081B920008048780043
:109B000080B82000104078000030A10081B820000B
:109B10008048780060B92000104078000080FB0089
:109B20004200DE00610060000004E0000500320039
:109B300080B92000104078000000A00081B920000A
:109B40008048780060B92000104078000080FB0059
:109B50000000D100610060000004E0000500320058
:109B600080B92000104078000010A00081B92000CA
:109B70008048780060B92000104078000080FB0029
:109B8000610060000004E0000500320080B92000A0
:109B9000104078000020A00081B9200080487800A3
:109BA00060B92000104078000080FB004300DE0018
:109BB0000000A200610060000004E0000500320027
:109BC00080B82000104078000030A00081B820004C
:109BD0008048780060B72000104078008080FB004B
:109BE000208220000080400010407800CFFC070059
:109BF00010C0B30088720200000000008FFE370022
:109C00000040EB0088720200000000008BFE37006D
:109C10004F0478000080FA00000006000400FA00FB
:109C2000169E0200000000000004E0002200320046
:109C300032C2BF00684060000004E000040032004F
:109C40003100200010CF2000D89B0200000000004F
:109C500032C2BF00644060000004E0000400320033
:109C60003100200040CF2000D89B020000000000FF
:109C7000069E020000000000000F780032C2BF0004
:109C8000624060000004E00008003200F1002000A3
:109C900070CF2000D89B02000000000090118000CF
:109CA000D1FF2F0001006000901188001E00780095
:109CB0001007980006003700F100200060D0200057
:109CC000D89B0200000000000000EB001007980085
:109CD0001E0090000080FA00000006000200FA005A
:109CE000000F78001E007800F29D020000000000C6
:109CF0000000EB000080FA00000006000000FA00FF
:109D000001022000C0DB2000D89B02000000000000
:109D100060B7200010407800C4700200000000000E
:109D200000C2B300887202000000000060B720008B
:109D300010407800E94F500007003A00C011800041
:109D4000667002000000000000C2B30088720200CA
:109D5000000000000C00370060B7200010407800C1
:109D60000080FB0080004000A0B020000080400088
:109D700010007800667002000000000000C2B3000E
:109D80008872020000000000A0DD20001040780072
:109D900063406000C47002000000000000C2B30015
:109DA0008872020000000000A0DD20001040780052
:109DB0000080FB004200DE0061406000C4700200D1
:109DC0000000000000C2B300887202000000000022
:109DD000A0DD2000104078000080FB004300DE0082
:109DE00061406000C47002000000000000C2B300C7
:109DF000887202000000000080B820001040780047
:109E00000080FB004300DE0061406000C47002007F
:109E10000000000000C2B3008872020000000000D1
:109E200031002000F0AD2000D89B020000000000AF
:109E30000080FA00000006000C00FA00A81A0200D8
:109E400000000000D2160200000000005007980039
:109E50005E009000EA0F500005003A00A81A0200C8
:109E600000000000D216020000000000000F780081
:109E7000A81A020000000000D21602000000000034
:109E800040079800A81A020000000000D216020045
:109E90000000000030079800A81A0200000000002F
:109EA000D21602000000000020079800A81A020045
:109EB00000000000D2160200000000001007980009
:109EC0005E0090000000E000090034005E00900099
:109ED000EA0F500006003C005E0090000040E900E0
:109EE0008040780060B72000014878000200370009
:109EF0000000EB00500798004E0090000000E000CA
:109F00000F0034004E009000E40F50000C003C00A5
:109F10004E0090000040E900E3406000A0DD20001A
:109F20001040780063C16000C1CFB3000140600001
:109F300002407000A1DD2000804878000200370058
:109F40000000EB00500798003E0090000000E00089
:109F5000100034003E009000E20F50000D003C0065
:109F60003E0090000040E90061416000A0DD20005B
:109F700090407800614061004201DD00B0CFB30045
:109F800080C0600082C07000A0DD20000148780021
:109F9000020037000000EB00500798002E009000F0
:109FA0000000E000100034002E009000E20F50008E
:109FB0000D003C002E0090000040E900614160006F
:109FC000A0DD200090407800614061004301DD0089
:109FD00070CFB30080C0600082C07000A0DD2000A0
:109FE00001487800020037000000EB00500798009D
:109FF0001E0090000000E000100034001E009000E1
:10A00000E20F50000D003C001E0090000040EA00EE
:10A010006141600080B8200090407800614061009C
:10A020004301DD0070CFB30080C0600082C07000CB
:10A0300080B8200001487800020037000000EB00E3
:10A04000500798005E0090000000E00073003A00A6
:10A050000000EB0060698800D108200030872000F4
:10A06000629C0200000000008001EB00A2002000C2
:10A0700011002000100020001E1D02000000000042
:10A080000040E9008040780060B720000148780077
:10A0900060B7200010407800E94F50000B003A00F4
:10A0A000C1012000001B2100629C02000000000092
:10A0B0008001EB00F2FF27001100200020022000A9
:10A0C0001E1D020000000000000F78004105200066
:10A0D00050D12000D89B0200000000008001EB005E
:10A0E0004200200011002000100020001E1D020070
:10A0F000000000000040E900E3406000A0DD200017
:10A100001040780063C16000C1CFB300014060001F
:10A1100002407000A1DD200080487800110220007C
:10A1200090D62000D89B0200000000008001EB00C8
:10A130002200200011002000100020001E1D02003F
:10A14000000000000040E90061416000A0DD200047
:10A1500090407800614061004201DD00B0CFB30063
:10A1600080C0600082C07000A0DD2000014878003F
:10A1700021032000A0D82000D89B0200000000008E
:10A180008001EB00220020001100200010002000C0
:10A190001E1D0200000000000040E9006141600057
:10A1A000A0DD200090407800614061004301DD00A7
:10A1B00070CFB30080C0600082C07000A0DD2000BE
:10A1C00001487800F1042000B0932000629C020056
:10A1D000000000008001EB002200200011002000A0
:10A1E000100020001E1D0200000000000040EA00D8
:10A1F0006141600080B820009040780061406100BB
:10A200004301DD0070CFB30080C0600082C07000E9
:10A2100080B820000148780001003700B7FE070031
:10A2200060B7200010407800E94F50001C003A0051
:10A23000A0DD2000104078000080FB004200DE001E
:10A240006140600080417800A0DD2000104078006F
:10A250006340600080427800A0DD2000104078005C
:10A260000080FB004300DE00614060000041780098
:10A2700080B82000104078000080FB004300DE0022
:10A2800061406000804078001E0078000342780042
:10A2900085417800469D0200000000002200370042
:10A2A000A0DD2000104078000080FB004200DE00AE
:10A2B0006140600000417800A0DD2000104078007F
:10A2C0006340600080417800A0DD200010407800ED
:10A2D0000080FB004300DE006140600080427800A7
:10A2E00080B82000104078000080FB004300DE00B2
:10A2F000614060000043780060B7200010407800A3
:10A300000080FB0080004000A0B0200000804000E2
:10A3100010007800024278000541780086407800FD
:10A32000469D020000000000A0DD200010407800E3
:10A3300063406000E34F500003003A0091C0B30057
:10A3400070B7200001487800CA9D0200000000009C
:10A35000C111800040118000808F50000400310046
:10A3600001022000C01C2100629C020000000000CD
:10A370000080FA00000006000000FA00D69D0200EE
:10A38000000000000080FA00000006000400FA004F
:10A39000000F78001E007800100798001E00900043
:10A3A000E10F50000C0032001E009000E10F500041
:10A3B000040039001E009000E20F50003D00320002
:10A3C0005900370031052000C0DD2000D89B020075
:10A3D0000000000058003700B1002000F0E220002B
:10A3E000629C020000000000D1002000A0E32000D9
:10A3F000629C020000000000089D020000000000B6
:10A400000000E0004C00320090118000D1FF2F00CE
:10A4100001006000901188000000370032C2BF00C8
:10A42000614060000004E0000600320023C2BF006B
:10A43000624060000004E00002003A00B0118000B9
:10A440002011880022C2BF00614060000004E000CB
:10A450000600320033C2BF00624060000004E0002A
:10A4600002003A0030118000A011880032C2BF0003
:10A47000624060000004E00004003A0022C2BF0015
:10A48000624060000004E000E4FF320091118000AF
:10A49000D0FF2F0000806000901188001111800013
:10A4A000D0FF2F000080600010118800CA82A90030
:10A4B000DAFF3700E100200070E42000629C020017
:10A4C00000000000F1002000C01E2100629C02007C
:10A4D0000000000090118000D1FF2F0001006000FB
:10A4E0009011880032C2BF00614060000004E000AB
:10A4F0000600320023C2BF00624060000004E0009A
:10A5000002003A00B01180002011880022C2BF0072
:10A51000614060000004E000F2FF32003011800072
:10A52000000F78000400370041022000C020200006
:10A53000629C0200000000000080FA00000006009B
:10A540000000FA0091118000D0FF2F000080600011
:10A5500090118800A0DD2000104078000040A0008D
:10A56000A1DD20008048780080B8200010407800ED
:10A570000010A00081B8200080487800C1012000B0
:10A5800050E52000629C0200000000000080FA00FC
:10A59000000006000000FA00A0DD20001040780056
:10A5A0000040A100A1DD20008048780080B8200094
:10A5B000104078000010A10081B820008048780089
:10A5C0004101200010E72000629C02000000000012
:10A5D0000080FA00000006000200FA000000EB0014
:10A5E000000F780034003700A0DD20001040780014
:10A5F000704060000004E0002B003200A0A328009F
:10A60000586E020000000000610020006069200018
:10A61000D89B02000000000032C2BF00684060000A
:10A620000004E000040032003100200010CF2000C0
:10A63000D89B02000000000032C2BF0064406000EE
:10A640000004E000040032003100200040CF200070
:10A65000D89B020000000000069E020000000000DF
:10A66000949802000000000032C2BF006240600007
:10A670000004E00008003200F100200070CF20004C
:10A68000D89B02000000000090118000D1FF2F0035
:10A690000100600090118800A0A32800586E0200FD
:10A6A0000000000002003700069E020000000000CB
:10A6B00010002000000F7800169E0200000000002D
:10A6C0000004E000C8FF3A001E0078000080FA0095
:10A6D000000006000000FA00B1002000100921006F
:10A6E000629C0200000000000080FA0000000600EA
:10A6F0000000FA00B0A328002C6E02000000000049
:10A700000080FA00000006000400FA00A0DD20002E
:10A71000104078000000A1000010A100A1DD200081
:10A7200080487800A0DD2000104078000020A100C3
:10A73000A1DD200080487800A0DD200010407800D6
:10A740000030A100A1DD20008048780080B8200002
:10A75000104078000030A00081B8200080487800C8
:10A76000F0588000A06E8800A0DD20001040780026
:10A770000040A100A1DD200080487800A0DD20007D
:10A78000104078000080FB004200DE006140600065
:10A7900080417800A0DD2000104078006340600018
:10A7A00080427800A0DD2000104078000080FB008F
:10A7B0004300DE00614060000041780080B8200066
:10A7C000104078000080FB004300DE006140600024
:10A7D00080407800A06E80000342780085417800B8
:10A7E000469D020000000000CA9D0200000000001B
:10A7F000BFFF070000003700169E020000000000A7
:10A800000004E0000C003200A0DD200010407800C1
:10A81000704060000004E00005003200069E020067
:10A8200000000000887202000000000002003700F3
:10A83000069E02000000000032C2BF0062406000BD
:10A840000004E0000400320090118000D1FF2F00CE
:10A85000010060009011880022C2BF0061406000CA
:10A860000004E000E4FF32003011800080407800F6
:10A8700080DD20000148780080DD20001040780055
:10A880000080FB004400DE008040780070DD200086
:10A890000148780070DD2000104078000080FB0047
:10A8A000100798001E009000E40F5000D000320006
:10A8B0009E009000E48F500007003C001E009000B6
:10A8C0000000E0000F0032009E009000E18F500079
:10A8D0009F0032008A0137001E009000E60F5000F2
:10A8E000CB0032009E009000E68F500084013500BE
:10A8F0009E00900068805000E10F500080013E00F3
:10A90000FB00370080DD2000104078000080FB0055
:10A91000000F78001E007800E20F5000190032008E
:10A920009E007800E28F500007003C001E00780077
:10A930000000E0000E0032009E007800E18F500021
:10A940000E0032007E0037001E007800E70F500036
:10A95000260032009E007800EF8F50005B0032002E
:10A960001E007800E30F500017003200740037001B
:10A97000D69D020000000000650137005CFF070063
:10A980009DFF370010C0B300887202000000000075
:10A9900032C2BF00624060000004E00004003200E8
:10A9A00090118000D1FF2F000100600090118800FD
:10A9B000A0DD2000104078000040A000A1DD2000B4
:10A9C000804878008CFF3700A0DD20001040780020
:10A9D0000040A100A1DD20008048780010C0B30035
:10A9E000887202000000000083FF370010C0B3002F
:10A9F0008872020000000000D69D020000000000E6
:10AA000022C2BF00614060000004E000FCFF320091
:10AA1000301180004800DD00A06E880010C0B30037
:10AA2000887202000000000022C2BF006140600086
:10AA30000004E000FCFF3200A16E800030118000B5
:10AA400000807000A06E8800A0DD2000104078001B
:10AA50000080FB004200DE00614060008041780021
:10AA6000A0DD200010407800634060008042780044
:10AA7000A0DD2000104078000080FB004300DE00D5
:10AA8000614060000041780080B8200010407800EC
:10AA90000080FB004300DE006140600080407800E1
:10AAA000A06E80000342780085417800469D020038
:10AAB00000000000CA9D02000000000010C0B300AA
:10AAC00088720200000000004BFF370010C0B30086
:10AAD000887202000000000090118000D1FF2F005A
:10AAE00001006000901188000000370032C2BF00F2
:10AAF000614060000004E0000600320023C2BF0095
:10AB0000624060000004E00002003A00B0118000E2
:10AB10002011880022C2BF00614060000004E000F4
:10AB2000F2FF320033C2BF00624060000004E00068
:10AB3000EEFF3A0030118000A0118800EBFF3700D3
:10AB40000040EB0088720200000000002AFF37007E
:10AB500080DD200090407800F0C0B30080C060002D
:10AB600080DD20000148780080DD20001040780062
:10AB70008040E80080DD20000148780010C0B3006C
:10AB800088720200000000008040EB0060DD2000C1
:10AB9000014878000F00370022C2BF00614060000A
:10ABA0000004E000FCFF320030118000F29D020042
:10ABB0000000000010C0B300887202000000000016
:10ABC00060DD2000104078008040E80060DD20005B
:10ABD0000148780060DD20009040780080DD200092
:10ABE0001040780080CF5000EBFF390002FF3700A3
:10ABF00080DD200010407800B89E020000000000B8
:10AC000010C0B3008872020000000000FAFE370096
:10AC100080DD200090407800F0C0B30080C060006C
:10AC200080DD20000148780080DD200010407800A1
:10AC3000EA4F500003003600A1C0B30080DD2000C1
:10AC40000148780080DD2000104078000080FB0083
:10AC500080004000E0B1200000804000100078003B
:10AC6000A06E8800D69D020000000000A0DD20003C
:10AC7000104078000080FB004200DE006140600070
:10AC800080417800A0DD2000104078006340600023
:10AC900080427800A0DD2000104078000080FB009A
:10ACA0004300DE00614060000041780080B8200071
:10ACB000104078000080FB004300DE00614060002F
:10ACC00080407800A06E80000342780085417800C3
:10ACD000469D020000000000CA9D02000000000026
:10ACE00010C0B3008872020000000000C2FE3700EE
:10ACF000A0DD2000104078000000A1000010A1009D
:10AD0000A1DD200080487800A0DD20001040780000
:10AD10000020A100A1DD200080487800A0DD2000F7
:10AD2000104078000030A100A1DD200080487800AC
:10AD300080B82000104078000030A10081B82000C9
:10AD40008048780080DD2000104078000080FB0003
:10AD50004300DE00610060000004E0000D003200EE
:10AD6000A0DD200010407800634060000014A000C7
:10AD7000E3406000A0DD20001040780063C1600067
:10AD8000C1CFB3000140600002407000A1DD20008F
:10AD90008048780080DD2000104078000080FB00B3
:10ADA0004200DE00610060000004E0000D0032009F
:10ADB000A0DD200010407800634060000004A00087
:10ADC000E3406000A0DD20001040780063C1600017
:10ADD000C1CFB3000140600002407000A1DD20003F
:10ADE0008048780080DD2000104078000080FB0063
:10ADF0000000D100610060000004E00005003200A6
:10AE0000A0DD2000104078000020A000A1DD20007F
:10AE10008048780080DD2000104078000080FB0032
:10AE2000610060000004E00005003200A0DD2000A9
:10AE3000104078000030A000A1DD2000804878009C
:10AE400080DD2000104078000080FB004400DE0020
:10AE50000000A200610060000004E0000500320074
:10AE600080B82000104078000030A00081B8200099
:10AE700080487800D69D020000000000A0DD200080
:10AE8000104078000080FB004200DE00614060005E
:10AE900080417800A0DD2000104078006340600011
:10AEA00080427800A0DD2000104078000080FB0088
:10AEB0004300DE00614060000041780080B820005F
:10AEC000104078000080FB004300DE00614060001D
:10AED00080407800A06E80000342780085417800B1
:10AEE000469D020000000000CA9D02000000000014
:10AEF00010C0B30088720200000000003EFE370060
:10AF00000040EB0088720200000000003AFE3700AB
:10AF10000080FA00000006000000FA00029B020018
:10AF2000000000000080FB000080FA000000060026
:10AF30000200FA00000F78001E0078006A9A0200F2
:10AF400000000000001020000080FA000000060051
:10AF50000000FA00689B0200000000000080FB0077
:10AF60000080FA00000006000000FA0060BA20002D
:10AF700010407800C89A0200000000000080FA002B
:10AF8000000006000000FA0060BA200010407800BF
:10AF90000080FB000080FA00000006000000FA00BC
:10AFA0008040EB0060BA2000014878004102200098
:10AFB000B0002000629C0200000000000080FA0047
:10AFC000000006000000FA0011C0B30060BA2000C3
:10AFD0000148780041022000B0002000629C02007D
:10AFE000000000000080FA00000006000000FA00E7
:10AFF00080B82000104078000030A00081B8200008
:10B00000804878008040EB0080BB20000148780039
:10B01000C922A800CB22A900E1022000F0022000F2
:10B02000629C0200000000000080FA0000000600A0
:10B030000400FA00881F7800000F78001E00E0006E
:10B0400044003200200320009E0F100041003E000B
:10B050001E0FE90080BB2000104078000080FB003C
:10B060009E0F500005003E0091022000D0052000F8
:10B07000629C02000000000063013700E100200034
:10B0800060082000D89B0200000000001E0078002D
:10B090000040E800C47002000000000000A2280088
:10B0A0002C6E0200000000008040EB0020BB20005E
:10B0B000014878001F0037001E01780020BB2000E7
:10B0C000104078008080FB004310DD0081004000CC
:10B0D00090BB200000804000104078000080FB0002
:10B0E000949802000000000000C2B30088720200C1
:10B0F000000000001E01780020BB200010407800F6
:10B100008080FB004310DD008100400090BB2000E8
:10B1100000804000104078006A9A020000000000A1
:10B1200020BB2000104078008040E80020BB2000B9
:10B130000148780020BB200010407800E74F500005
:10B14000DDFF360030A22800586E0200000000002B
:10B150002D0137001E0078001007980050052000D0
:10B160009E009000808F5000110132005005200099
:10B170009E009000808F500008003E001E0090004E
:10B180000000E00012003200300320009E0090001A
:10B19000808F5000DD00320017013700C00E200004
:10B1A0009E009000808F500063003200000F20004E
:10B1B0009E009000808F50005F003200C00C200085
:10B1C0009E009000808F5000020132000A0137007B
:10B1D000D100200040092000629C02000000000015
:10B1E00071012000100A2000629C02000000000093
:10B1F00080BB2000104078000004E00005003A0009
:10B2000091022000D0052000629C02000000000096
:10B21000440037008040EB0030BB2000014878003C
:10B220003A00370000C2B30088720200000000003C
:10B2300030BB2000104078000040E800C4700200DD
:10B240000000000040A228002C6E02000000000058
:10B250008040EB0020BB200001487800160037003A
:10B2600030BB2000104078000081FB0020BB200094
:10B27000104078008080FB004310DD00810040001A
:10B2800090BB200000804000104078000080FB0050
:10B29000949802000000000000C2B300887202000F
:10B2A0000000000020BB2000104078008040E80033
:10B2B00020BB20000148780020BB2000104078000F
:10B2C000E74F5000E6FF360061002000800B2000B1
:10B2D000D89B02000000000030BB20001040780026
:10B2E0000080FB00C300DD0090BB20000080400018
:10B2F00010407800F700070030BB200010407800B5
:10B300008040E80030BB20000148780080BB20006E
:10B310009040780030BB20001040780080CF500073
:10B32000C0FF3E00310D2000E00B2000629C0200B7
:10B3300000000000B40037001E0078008040780054
:10B34000C083200001487800C00E20009E0F10002E
:10B3500005003A003101200010192000629C020013
:10B360000000000004003700D1002000401A200037
:10B37000629C02000000000071012000100A200001
:10B38000629C0200000000008040EB0020BB200017
:10B39000014878000A0107008040780030BB200097
:10B3A000014878008040EB0080BB20000148780015
:10B3B0004D00370000C2B300887202000000000098
:10B3C00020BB2000104078000040E800C47002005C
:10B3D0000000000040A228002C6E020000000000C7
:10B3E0000000EB00805D88000D003700815D80006B
:10B3F00090C0200000804000104078000080FB00DA
:10B40000949802000000000000C2B300887202009D
:10B4100000000000805D80000000E800805D880082
:10B42000805D8000E70F5000F0FF360061002000D3
:10B43000800B2000D89B02000000000090C020007C
:10B4400010407800A300070020BB200010407800C7
:10B45000E94F50001B003E000000EB00805D8800BB
:10B460001000370080BB2000104078008081FB0076
:10B47000845D8000815D800090C0200000804000DD
:10B48000104178004318DD008400400090BB20008C
:10B490000080400002487800805D80000000E800E5
:10B4A000805D8800805D8000E70F5000EDFF360072
:10B4B00080BB2000104078008040E80080BB200066
:10B4C0000148780020BB2000104078008040E80050
:10B4D00020BB200001487800C700070080407800AA
:10B4E00030BB20000148780030BB200010407800BD
:10B4F0000004E000AFFF3A00B1022000101B200062
:10B50000629C0200000000003F0037004800070076
:10B5100011012000C01D2000D89B02000000000087
:10B5200030C3B3006A9A0200000000000000EB0084
:10B53000805D880014003700885D8000029B020057
:10B54000000000008040780070BA20000000440035
:10B5500001487800815D800070BA200000804000C2
:10B56000104078000080FB0094980200000000006A
:10B5700000C2B3008872020000000000805D8000FD
:10B580000000E800805D8800805D8000E70F5000CB
:10B59000E9FF360030A22800586E020000000000CB
:10B5A00070BA2000104078004A00070016003700EB
:10B5B0001F00070001012000D01E2000629C020035
:10B5C0000000000050C5B3006A9A020000000000AD
:10B5D0000D00370016000700F1002000D01F2000EA
:10B5E000629C020000000000C0CCB3006A9A020016
:10B5F000000000000400370041022000C0202000AD
:10B60000629C0200000000004F0478000080FA00F5
:10B61000000006000000FA009100200080082100D0
:10B62000629C0200000000000080FA00000006009A
:10B630000200FA00E499020000000000004F7800C8
:10B64000A100200000232000D89B02000000000081
:10B650001E04E00005003A003100200050BB20002D
:10B66000629C0200000000001800370091002000DA
:10B67000A0232000D89B0200000000001E80FB00D9
:10B68000610060000004E00004003200510120006D
:10B6900030242000D89B0200000000001E80FB0028
:10B6A0000000D100610060000004E00004003200EE
:10B6B0004101200080252000D89B020000000000EE
:10B6C00030A22800586E0200000000000080FA003E
:10B6D000000006000400FA00004F78001E80FB0006
:10B6E00010079800200220009E009000808F5000DC
:10B6F0001E003200200220009E009000808F50002B
:10B7000007003C001E009000E40F50001C003200B7
:10B710009E009000F08F50000A0032002200370097
:10B72000800220009E009000808F50000A003200AE
:10B73000D00220009E009000808F50001500320043
:10B7400019003700B1012000C0262000629C0200D1
:10B750000000000018003700A10120007028200020
:10B76000629C02000000000013003700510120001D
:10B77000102A2000629C0200000000000E0037002A
:10B7800081012000602B2000629C0200000000006C
:10B790000900370001012000E02C2000629C02001B
:10B7A0000000000004003700E1002000E02D200030
:10B7B000D89B0200000000000080FA000000060094
:10B7C0000000FA008040EB0010C120000148780022
:10B7D0008040EB0030C12000014878008040EB0041
:10B7E00020C1200001487800080007000080FB000D
:10B7F0000080FA00000006000000FA0003000700C5
:10B800000080FB000080FA00000006000A00FA0039
:10B8100010C0B300704798000040EB0060479800EC
:10B820000040EB005047980010C0B300104798004C
:10B830000040EB00404798008040EB0040C12000F2
:10B840000148780030C12000104078000004E0007A
:10B850009C003A00E4990200000000000004E000AF
:10B860000C0032008040EB0010C12000014878003D
:10B870008040EB0030C12000014878008040EB00A0
:10B8800020C12000014878000000EB00400798002C
:10B89000A1003700C0832000104078006A9A02009F
:10B8A00000000000689B0200000000003047980084
:10B8B000689B020000000000204798003E40900076
:10B8C000E14F500003003A002E409000E14F50003D
:10B8D00068003200BE4090002E40900080CF5000A3
:10B8E00003003200BE409000014F78002600370070
:10B8F00010C12000904078007E409000814F5000A1
:10B900000E0031005E4090008080FB0090C020005F
:10B9100000804000904078001E40900080C0600091
:10B920000040EB00004F78000104E0000C00320002
:10B9300010C0B300004F78000900370010C120008C
:10B94000904078000040EB00004F78007E4090006F
:10B95000814F500002003A0010C0B300004F780041
:10B960001E04E00008003A007E4090006047980006
:10B970006E409000E84F500003003E0020C12000C0
:10B98000EE4090000148780010C0B3009E4F1000B8
:10B990000D003A005E4090000081FB005E40900088
:10B9A0008080FB0090C02000008040009040780024
:10B9B0001E40900080C0700090C020000000410038
:10B9C00001487800110037005E4090000082FB00C3
:10B9D0005E4090008080FB0090C02000008040000E
:10B9E00010407800804178001E41900002407800AD
:10B9F0000080EA008180EA0000C061008040780099
:10BA000090C0200000004200014878001E407800ED
:10BA1000C89A0200000000007E4090000040E8004C
:10BA2000704798001E40900000404000104798006A
:10BA30001E4090000004E0000B003A005E409000C1
:10BA40008080FB0090C02000008040001040780003
:10BA5000920007005E4090000040E80050479800C8
:10BA600010C0B300104798005E409000E74F5000B0
:10BA70008CFF3600FE40900000C4B30080CF500021
:10BA80001000360040C12000104078000004E000A3
:10BA90000C003A0010C12000EE40900001487800F0
:10BAA00010C12000104078000004E00003003A00BC
:10BAB00011C0B30030C120000148780010C0B300AD
:10BAC000404798004E4090000004E000040032001F
:10BAD00090C02000104078000004E0000B003A0005
:10BAE0008040EB0010C12000014878008040EB004E
:10BAF00030C12000014878008040EB0020C12000C8
:10BB0000014878000040EB00404798004E4090000C
:10BB10000080FB00400798004E0090000080FA0073
:10BB2000000006000E00FA000040EB0040479800BD
:10BB30000C0037004E4090000081FB004E4090000A
:10BB40008080FB0090C02000008040009040780082
:10BB500065004700017178004E4090000040E80009
:10BB6000404798004E409000E74F5000F1FF3600EC
:10BB700010C12000904078002147980030C120007B
:10BB8000904078001147980020C12000104F7800A5
:10BB900001C4B30010C12000014878008040EB00D0
:10BBA00030C120000148780018FF07000004E000C1
:10BBB0001A00320010C0B300304798000040EB007C
:10BBC00040479800110037004E4090008080FB00F5
:10BBD00065004700614178004E4090008080FB0086
:10BBE00090C020000080400010407800804F51003D
:10BBF000030032000040EB00304798000900370096
:10BC00004E4090000040E800404798004E409000B1
:10BC1000E74F5000ECFF3600020037000040EB0019
:10BC2000304798000040EB00404798000C00370078
:10BC30004E4090000081FB004E4090008080FB0051
:10BC400065004700E140780090C0200000004100FE
:10BC5000014878004E4090000040E80040479800BE
:10BC60004E409000E74F5000F1FF360010C1200019
:10BC7000AE4090000148780030C120009E40900006
:10BC80000148780020C120001E4878003E40900006
:10BC90000080FB000080FA00000006000200FA00AD
:10BCA000004F780040C12000104078001E4068001E
:10BCB0008080FB00D083200000804000904078000E
:10BCC00040C120000148780040C1200010407800A9
:10BCD0000080FB000080FA00000006000000FA006F
:10BCE00060A228002C6E0200000000000080FA0014
:10BCF000000006000400FA00C922A800CB22A90017
:10BD0000C8C2A90080B82000104078000030A00010
:10BD100081B820008048780080B82000104078006A
:10BD20000020A10081B8200080487800EBFF0700C8
:10BD30000000370022C2BF00614060000004E00044
:10BD4000FCFF3200301180008040780070BB200082
:10BD50000148780070BB2000104078000080FB0094
:10BD60004400DE008040780060BB2000014878007D
:10BD700060BB2000104078000080FB001007980096
:10BD80001E009000E10F5000780032009E009000ED
:10BD9000E48F50009D0032001E0090000000E00083
:10BDA00001003200A100370070BB20001040780075
:10BDB0000080FB00000F78009E007800E28F5000AA
:10BDC000170032001E007800E20F500007003C0010
:10BDD0009E0078000100E000980032001E0078000C
:10BDE000E10F50000C0032005C0037009E0078002C
:10BDF000E48F5000130032001E007800E40F500062
:10BE0000560035009E00780068805000E10F500019
:10BE100052003E0010003700B0FF0700C5FF37009A
:10BE2000E4990200000000008040780040BB200040
:10BE30000148780010C0B3008872020000000000C2
:10BE4000BCFF3700029B0200000000008872020065
:10BE500000000000B7FF370010C0B3008872020076
:10BE60000000000070BB200010407800E94F500037
:10BE700004003A00C1CEB300C0832000014878001E
:10BE80000300370001CFB300C083200001487800D1
:10BE90004BFE07008040780040BB2000014878003E
:10BEA000190037008040EB0050BB200001487800AB
:10BEB0000D00370050BB2000104078008080FB0050
:10BEC00090C020000080400010407800887202007E
:10BED0000000000050BB2000104078008040E800C7
:10BEE00050BB20000148780050BB20001040780073
:10BEF000E74F5000EFFF36003FFE0700804078001C
:10BF000040BB20000148780040BB20001040780072
:10BF10000004E000E3FF3A008040EB0050BB20004B
:10BF2000014878000800370000C0EB00887202006A
:10BF30000000000050BB2000104078008040E80066
:10BF400050BB20000148780050BB20001040780012
:10BF5000E74F5000F4FF360076FF37000040EB005B
:10BF6000887202000000000072FF370070BB2000E2
:10BF700090407800F0C0B30080C0600070BB20002B
:10BF80000148780070BB2000104078008040E80035
:10BF900070BB20000148780010C0B3008872020016
:10BFA000000000008040EB0050BB200001487800FA
:10BFB0000F00370022C2BF00614060000004E000B3
:10BFC000FCFF3200301180006A9A0200000000007D
:10BFD00010C0B300887202000000000050BB2000B7
:10BFE000104078008040E80050BB200001487800F5
:10BFF00050BB20009040780070BB200010407800BB
:10C0000080CF5000EBFF39004AFF370070BB2000A3
:10C0100010407800B89E02000000000010C0B3007D
:10C02000887202000000000042FF37000040EB0071
:10C0300088720200000000003EFF37000080FA0016
:10C04000000006000000FA0060A428002C6E020028
:10C05000000000000080FA00000006000000FA0066
:10C060000040EB0074830200000000000040EB0081
:10C0700074830200000000000040EB0074830200A3
:10C08000000000000040EB0074830200000000008C
:10C090000000EB00B0820200000000000000EB0096
:10C0A000B0820200000000000000EB00B08202003D
:10C0B000000000000080FA00000006000C00FA00FA
:10C0C00080B82000104078000030A00081B8200027
:10C0D0008048780080B82000104078000020A1003F
:10C0E00081B820008048780011C0B30060B72000FC
:10C0F0000148780081C0B30070B720000148780083
:10C1000021C0B300D0DE20000148780080C0EB00E1
:10C1100020C0B3005081020000000000C922A90025
:10C12000C902A900C8E2A80010C0B300E083020061
:10C1300000000000C3FF07000000370022C2BF005C
:10C14000614060000004E000FCFF3200301180001C
:10C150008040780010DF20000148780010DF2000C8
:10C16000104078000080FB004400DE008040780032
:10C1700000DF20000148780000DF20001040780038
:10C180000080FB00300798003E009000E30F500055
:10C1900017013200BE009000E38F50000A003C00FF
:10C1A0003E019000E10F5100A5003200BE01900059
:10C1B000E18F5100FB003C003E0090000000E000D9
:10C1C00012003200E8023700BE009000E68F5000F7
:10C1D000910232003E019000E60F510004003C0045
:10C1E000BE019000E48F510083023200DE0237006E
:10C1F0003E009000E80F50009E023200BE0090000A
:10C20000EA8F500034013200D702370010DF2000DF
:10C21000104078000080FB006101B90042079800DF
:10C2200053079800D0002000010020004E0190002C
:10C23000DE019000800F5100818F59007C003E008C
:10C240004E009000DE00900000600100CA0237003E
:10C250000C0037000D0037001200370017003700C0
:10C260001D00370023003700440037004800370026
:10C270004C00370052003700580037005E0037008E
:10C28000640037006FFF0700ACFF3700DE8102005B
:10C290000000000010C0B30088720200000000001F
:10C2A000A6FF37001E8202000000000010C0B3008D
:10C2B0008872020000000000A0FF37000040EB0081
:10C2C000E08302000000000010C0B300887202008A
:10C2D0000000000099FF370010C0B300E0830200A7
:10C2E0000000000010C0B3008872020000000000CF
:10C2F00092FF3700D0DE200010407800E24F50005F
:10C3000006003A000483020000000000804078002C
:10C31000F0DE20000148780006003700F00F200012
:10C320003E8202000000000080407800F0DE200025
:10C330000148780080B82000104078006440600018
:10C340000004E00008003200F0DE20001040780019
:10C350000080FB009C9902000000000080407800F3
:10C36000F0DE200001487800F0DE20001040780068
:10C37000887202000000000070FF37005283020044
:10C380000000000088720200000000006BFF370010
:10C39000F28302000000000088720200000000002A
:10C3A00066FF370010C0B300968302000000000053
:10C3B00010C0B30088720200000000005FFF370069
:10C3C0000040EB00CE8302000000000010C0B3006C
:10C3D000887202000000000058FF370010C0B30050
:10C3E000CE8302000000000010C0B300887202007B
:10C3F0000000000051FF37000040EB00BC8302004A
:10C400000000000010C0B3008872020000000000AD
:10C410004AFF370010C0B300BC83020000000000D8
:10C4200010C0B300887202000000000043FF370014
:10C430000040EB0088720200000000003FFF370060
:10C4400010DF200090407800F0C0B30080C0600092
:10C4500010DF20000148780010DF20001040780035
:10C460008040E80010DF20000148780010C0B300D1
:10C4700088720200000000008040EB00F0DE200027
:10C48000014878004000370022C2BF0061406000D0
:10C490000004E000FCFF3200301180008040780092
:10C4A000E0DE20000148780080B8200010407800CD
:10C4B000644060000004E00008003200E0DE20007C
:10C4C000104078000080FB009C99020000000000F2
:10C4D00080407800E0DE200001487800D0DE2000B7
:10C4E00010407800E24F500009003A00E0DE2000E2
:10C4F000104078000080FB00B082020000000000C5
:10C5000010C0B3008872020000000000190037005C
:10C51000E0DE2000104078000080FB003E82020038
:10C520000000000080407800E0DE20000148780034
:10C5300080B8200010407800644060000004E000F3
:10C5400008003200E0DE2000104078000080FB0090
:10C550009C9902000000000080407800E0DE20008E
:10C5600001487800E0DE2000104078008872020068
:10C5700000000000F0DE2000104078008040E8005D
:10C58000F0DE200001487800F0DE200090407800C6
:10C5900010DF20001040780080CF5000BAFF390033
:10C5A000E6FE370010DF200090407800F0C0B300B6
:10C5B00080C0600010DF20000148780010DF2000FC
:10C5C000104078008040E80010DF2000014878002B
:10C5D00010DF200010407800968302000000000069
:10C5E00010C0B3008872020000000000D3FE3700C4
:10C5F00010DF200090407800F0C0B30080C06000E1
:10C6000010DF20000148780010DF20001040780083
:10C610008040E80010DF20000148780010C0B3001F
:10C62000887202000000000022C2BF00614060006A
:10C630000004E000FCFF32003011800080407800F0
:10C6400000DF2000014878008040EB00F0DE200091
:10C65000014878001600370000DF20001040780005
:10C660000004E00004003D0010C0B3007483020029
:10C6700000000000030037000040EB00748302005C
:10C680000000000000DF2000104078000040400063
:10C690008040780000DF200001487800F0DE2000B4
:10C6A000104078008040E800F0DE2000014878006B
:10C6B000F0DE20009040780010DF2000104078006D
:10C6C00080CF5000E4FF390010C0B3008872020030
:10C6D0000000000099FE370010DF200010407800B5
:10C6E0000080FB0020079800400A2000AE00900068
:10C6F000808F500015003200500A20002E0190005B
:10C70000800F5100C5003200000A2000AE019000E9
:10C71000808F5100010032003301370022C2BF0078
:10C72000614060000004E000FCFF32003011800036
:10C7300080407800C0DE20000148780010C0B300BF
:10C7400088720200000000007CFE3700C0DE20007E
:10C75000104078000080FB00100798001E00900039
:10C76000E10F5000040032009E009000E28F500064
:10C770003B003200A500370022C2BF0061406000CC
:10C780000004E000FCFF320030118000506F880090
:10C79000506F80006300B900506F88000000EB000C
:10C7A000406F88000C00370022C2BF00614060006B
:10C7B0000004E000FCFF320071408000406F800008
:10C7C000808040003011800080487800406F8000F9
:10C7D0000000E800406F8800416F8000506F8000CB
:10C7E000808F5000F0FF39000000EB00406F8800A0
:10C7F0001300370071408000406F800000804000CF
:10C800000080E8001041780071408000406F800097
:10C81000008040000000E8009041780071408000F6
:10C82000406F800000804000104078008340780016
:10C8300053010700406F800063004000406F880094
:10C84000416F8000506F8000808F5000E9FF3900F9
:10C8500010C0B300887202000000000037FE3700ED
:10C8600022C2BF00614060000004E000FCFF320013
:10C8700030118000506F8800506F80004200DD0052
:10C88000506F88000000EB00406F88000C003700FC
:10C8900022C2BF00614060000004E000FCFF3200E3
:10C8A00071408000406F8000808040003011800027
:10C8B00080487800406F80000000E800406F8800EA
:10C8C000416F8000506F8000808F5000F0FF390072
:10C8D0000000EB00406F8800440037000040EB0090
:10C8E00074830200000000000040EB00748302002B
:10C8F000000000000040EB00748302000000000014
:10C900000040EB00748302000000000071408000D2
:10C91000406F800000804000104078000080FB00E5
:10C92000B08202000000000071408000406F800073
:10C93000008040000000E800104078000080FB000C
:10C94000B08202000000000071408000406F800053
:10C95000008040000080E800104078000080FB006C
:10C96000B08202000000000071408000406F800033
:10C97000008040006301400071408000406F8000F3
:10C980000080400063004000104078006F4060006D
:10C99000004978008040EB00F0DE2000014878007C
:10C9A00006003700ADFD0700F0DE200010407800E3
:10C9B0008040E800F0DE20000148780071408000EF
:10C9C000406F80000080400063004000904078008D
:10C9D000F0DE20001040780080CF5000F1FF3E00D4
:10C9E000406F800064004000406F8800416F80000D
:10C9F000506F8000808F5000B8FF390010C0B30026
:10CA00008872020000000000CCFD37000040EB00FF
:10CA10008872020000000000C8FD3700C0DE200060
:10CA2000104078000080FB00000F78001E017800A5
:10CA3000E10F5100040032009E017800E28F5100A6
:10CA400045003200BDFD370022C2BF0061406000DA
:10CA50000004E000FCFF320030118000506F8800BD
:10CA600022C2BF00614060000004E000FCFF320011
:10CA7000301180008040780000DF200001487800FD
:10CA80000000EB00406F88002E00370000DF200020
:10CA900090407800E0DE2000014878008040EB0004
:10CAA000F0DE20000148780019003700E0DE2000A9
:10CAB000104078000080FB00610060000004E0008E
:10CAC0000400320010C0B3007483020000000000B4
:10CAD000030037000040EB007483020000000000F8
:10CAE000E0DE2000104078000080FB000000D10054
:10CAF00080407800E0DE200001487800F0DE200071
:10CB0000104078008040E800F0DE20000148780006
:10CB1000F0DE200010407800E34F5000E3FF3600C5
:10CB200004830200000000000483020000000000F3
:10CB30008872020000000000406F80000000E800E2
:10CB4000406F8800416F8000506F8000808F5000E0
:10CB5000CEFF390079FD370022C2BF00614060007E
:10CB60000004E000FCFF320030118000506F8800AC
:10CB70000000EB00406F88001600370022C0B300B1
:10CB800060B92000A10B2000B7000700EA000700F1
:10CB900022C0B30060BB2D00A10B2000B200070033
:10CBA00022C0B300603D2D00A10B2000AE000700A5
:10CBB000E100070022C0B30060BB2000A10B2000F1
:10CBC000A9000700DC000700406F80000000E800BB
:10CBD000406F8800416F8000506F8000808F500050
:10CBE000E6FF390055FD37000040EB008872020077
:10CBF0000000000051FD370010DF200010407800D9
:10CC0000B89E02000000000010C0B300887202004D
:10CC10000000000049FD370010DF20009040780040
:10CC200030C0B30080C0600010DF200001487800F1
:10CC300010DF20009040780060B7200001487800A5
:10CC400060B7200090407800D0DE200010407800CF
:10CC5000508102000000000010C0B300E083020019
:10CC60000000000010C0B300887202000000000045
:10CC700032FD370080B82000104078000030A1005D
:10CC800081B820008048780010DF20001040780034
:10CC90000080FB004300DE000000A2006100600095
:10CCA0000004E0000500320080B820001040780049
:10CCB0000030A00081B820008048780021C0B30077
:10CCC000D0DE20000148780010DF200010407800FE
:10CCD0000080FB004200DE00610060000004E00014
:10CCE0000300320031C0B300D0DE200001487800DC
:10CCF00080B82000104078000020A10081B82000FA
:10CD00008048780010DF2000104078000080FB0091
:10CD10000000D100610060000004E0000500320066
:10CD200080B82000104078000020A00081B82000CA
:10CD30008048780060B7200090407800D0DE200066
:10CD400010407800508102000000000010C0B300C5
:10CD5000E08302000000000010C0B30088720200EF
:10CD600000000000F5FC37000040EB008872020074
:10CD700000000000F1FC37000080FA00000006000F
:10CD80000600FA0020479800314798004247980073
:10CD90002E4090000080FB004600DE00004F78002F
:10CDA0000040EB0010479800220037001E40900022
:10CDB000E34F50000C003A001E04E0000A0032006D
:10CDC00010C0B300CE830200000000001E80FB00F4
:10CDD0003A990200000000000040EB00CE83020000
:10CDE00000000000100037002E4090000080FB0083
:10CDF000610060000004E0000400320010C0B300D5
:10CE00007483020000000000030037000040EB00C4
:10CE100074830200000000002E4090000080FB00A0
:10CE20000000D100204798001E4090000040E8001C
:10CE3000104798001E409000E34F5000DBFF360083
:10CE40003E4090000080FB00B08202000000000025
:10CE50004E4090000080FB00B08202000000000005
:10CE60000080FA00000006000800FA001007980091
:10CE700021079800624798000040EB00748302008D
:10CE8000000000000040EB0074830200000000007E
:10CE90000040EB0074830200000000000040EB0043
:10CEA00074830200000000001E0090009C990200A4
:10CEB00000000000B0820200000000001E00900090
:10CEC000AE0090004809DD004800DE00000071005F
:10CED000C808DE009C99020000000000B082020039
:10CEE000000000001E009000AE0090004008DE0030
:10CEF000010020009C99020000000000B0820200A6
:10CF0000000000006E4090006F4060006047980095
:10CF10000040EB00004F7800020037004FFC070094
:10CF20001E4FE8006E4090009E4F1000FBFF39003E
:10CF30000080FA00000006000000FA0010C0B300F4
:10CF400074830200000000000040EB0074830200C4
:10CF5000000000000040EB007483020000000000AD
:10CF60000040EB0074830200000000000000EB00B2
:10CF7000B0820200000000000483020000000000F4
:10CF8000887202000000000004830200000000001C
:10CF9000887202000000000030FC07002FFC070030
:10CFA0000080FA00000006000200FA00005D800028
:10CFB0000000E0001200320000C2B30088720200DC
:10CFC000000000003100200010442000D89B020027
:10CFD0000000000000C2B3008872020000000000E0
:10CFE000F05C80000000E00003003A000040EB002D
:10CFF00074830200000000000000EB00005D880068
:10D00000F05C80000000E00003003A0004830200AE
:10D0100000000000004F780010002000005D880034
:10D020001E80FB000080FA00000006000400FA00E9
:10D03000000F7800005D80000000E0001200320068
:10D0400000C2B3008872020000000000310020001E
:10D0500010442000D89B02000000000000C2B30072
:10D060008872020000000000F05C80000000E00018
:10D0700003003A000040EB0074830200000000004F
:10D080000000EB00005D8800F05C80000000E00024
:10D0900007003A001E007800B08202000000000085
:10D0A00052830200000000000080FB00000F7800A7
:10D0B00000C2B30088720200000000001E00E00001
:10D0C00007003A003100200010442000D89B0200E5
:10D0D0000000000000302000100798000600370014
:10D0E0004100200040442000D89B020000000000C6
:10D0F00000102000100798001E0090000080FA0029
:10D10000000006000000FA00005D80000000E00062
:10D110000F0032004100200040442000D89B020054
:10D120000000000020A12800586E0200000000004E
:10D13000F05C80000000E00003003A0010C0B30083
:10D1400074830200000000000000EB00005D880016
:10D15000F05C80000000E0000F003A00DE81020079
:10D16000000000000000E0000B00320091002000F1
:10D17000A0232000D89B02000000000051012000E5
:10D1800030242000D89B02000000000020A12800CD
:10D19000586E020000000000D100200080442000F2
:10D1A000629C0200000000000080FA0000000600FF
:10D1B0000000FA00005D80000000E0000F00320077
:10D1C0004100200040442000D89B020000000000E5
:10D1D00020A12800586E020000000000F05C8000D2
:10D1E0000000E00003003A0010C0B30074830200A6
:10D1F000000000000000EB00005D8800F05C800093
:10D200000000E00002003A001E8202000000000060
:10D21000C100200050452000629C02000000000078
:10D220000080FA00000006000000FA000101200062
:10D2300020522000D89B0200000000000040EB00BC
:10D24000C47002000000000000C2B3008872020037
:10D250000000000060B7200010407800C470020099
:10D260000000000000C2B30088720200000000004D
:10D2700030A12800586E0200000000000080FA0073
:10D28000000006000400FA000000EB001007980000
:10D290000000EB00F05C8800A81A0200000000000B
:10D2A000D216020000000000000F78001E00E0000F
:10D2B00009003400400020009E0F100006003C00D2
:10D2C0001E0078000040E9008040780060B7200030
:10D2D00001487800020037000000EB00000F7800E2
:10D2E0001E00E0002D003A000000EB00606988009D
:10D2F0000000EB00F05C8800F05C80000000E000C3
:10D300000F003A00B103200060482000629C020038
:10D31000000000008001EB0042002000110020000E
:10D32000100020001E1D0200000000000040E90067
:10D330008040780060B72000014878002200370064
:10D34000C140800030002300808F500004003E0068
:10D3500051032000104C2000D89B02000000000068
:10D36000C1022000604F2000D89B02000000000096
:10D370008001EB003200200011002000100020008E
:10D380001E1D0200000000000040E90080407800FF
:10D3900060B72000014878000B003700C1408000D2
:10D3A00030002300808F500004003E005103200015
:10D3B000104C2000D89B0200000000009AFF0700DC
:10D3C0000000EB00005D880080B82000104078006D
:10D3D0000030A00081B8200080487800F05C800018
:10D3E0000000E00009003A00C922A800C902A80014
:10D3F000CB02A900CB22A90060B7200090407800A2
:10D4000020C0B30050810200000000000080FA003C
:10D41000000006000000FA000000EB00005D88003C
:10D42000F05C8000E10F500001003A0007E2A90023
:10D430000080FA00000006000600FA0010079800BD
:10D440001E009000200798002E009000E10F500071
:10D450000C0032002E009000E10F50000400390053
:10D460002E009000E20F500065003200730037007C
:10D470005103200020532000D89B02000000000030
:10D48000720037008040EB0000302000FE83020075
:10D4900000000000E102200070562000629C0200A3
:10D4A00000000000CBC2BF00614060000004E0004B
:10D4B00004003200CBC2BF00624060000004E00004
:10D4C0000C003A0091002000A0232000D89B02000D
:10D4D000000000005101200030242000D89B0200F1
:10D4E0000000000020A12800586E0200000000008B
:10D4F000560037000000EB00000F780039003700BD
:10D50000F05C80000000E00009003A00DE810200CB
:10D51000000000001E007800B08202000000000041
:10D5200052830200000000000080FB0010079800FA
:10D530001E0090000000E00024003A001E00780069
:10D54000949802000000000080C2B30088720200BC
:10D55000000000001E0078000080D10094980200B6
:10D56000000000001E0078000000A20061006000C2
:10D570000004E0000400320050A128002C6E0200DC
:10D58000000000000B003700F05C80000000E000AD
:10D5900005003A00048302000000000010C0B30040
:10D5A000748302000000000080A128002C6E02009D
:10D5B0000000000030A128002C6E020000000000D6
:10D5C00000C2B3008872020000000000F05C80001E
:10D5D0000000E00002003A001E820200000000008D
:10D5E0001E0FE800F00F20009E0F1000C4FF340053
:10D5F00020A12800586E0200000000001300370030
:10D60000F05C8000E10F500001003A0007E2A90041
:10D610007100200050592000629C020000000000B0
:10D62000F1002000C01E2100629C020000000000EA
:10D6300010C0B3000E0007000400370041022000B4
:10D64000C0202000629C0200000000000080FA0060
:10D65000000006000000FA00B1002000C00921000F
:10D66000629C0200000000000080FA00000006003A
:10D670000A00FA00004F98000040EB002047980095
:10D680000040EB00104798000040EB00004F78008E
:10D690003073020000000000C922A800C902A800DF
:10D6A000CB02A900CB22A90062A0A80062C0A800FA
:10D6B0008660A900CBC2BF000080FB000000D10043
:10D6C00061406000604798006E40900050479800AD
:10D6D000CBC2BF0061406000604798006E40900080
:10D6E000304798000000370086C0BF0068406000E7
:10D6F0000004E00012003A0023C2BF006240600054
:10D700000004E0000E003A007A73020000000000FE
:10D7100022C2BF00614060000004E000F2FF32005E
:10D7200030118000004F780062A0A90062C0A900FB
:10D730000E4890000004E00061003A0063003700EA
:10D740008660A900CBC2BF000080FB000000D100B2
:10D750006140600060479800CBC2BF00614060003C
:10D76000404798002E4090000004E0002E00320058
:10D770003E4090000004E0002B003A004E40900034
:10D780000004E000280032001E409000E74F5000E7
:10D790000B003E001E40780000404000004F780023
:10D7A0006E4090000004E000010032001E04A00062
:10D7B0001E4090000040E800104798003B003700F2
:10D7C0000E4890000004E000040032001E80FB00C0
:10D7D000507102000000000006003700C0C5B30011
:10D7E00044730200000000001E40780044730200F1
:10D7F000000000006E4090000004E00004003200D1
:10D80000D0C2B300447302000000000003003700E0
:10D81000B0C2B30044730200000000000040EB00FF
:10D8200010479800210037003E4090000004E000BF
:10D830001E0032004E4090000004E0001B00320049
:10D840005E4090000004E0000B0032006E4090004B
:10D850000004E00008003A0010C0B3002047980020
:10D860000040EB0010479800B0C5B30044730200BD
:10D87000000000000D0037005E4090000004E00052
:10D880000A003A006E4090000004E00007003200F9
:10D890000040EB00204798000040EB001047980044
:10D8A000D0C5B30044730200000000006E40900039
:10D8B000504798004E409000304798008AFF37004C
:10D8C00020A12800586E0200000000000080FA002D
:10D8D000000006000000FA00B0A128002C6E020033
:10D8E000000000000080FA00000006000400FA00BA
:10D8F000C922A800C902A800CB02A900CB22A90016
:10D90000C8C2A90080B82000104078000030A000F4
:10D9100081B820008048780080B82000104078004E
:10D920000020A10081B820008048780080C0EB0072
:10D9300020C0B3005081020000000000E5FF070096
:10D940000000370022C2BF00614060000004E00018
:10D95000FCFF32003011800080407800C0B9200008
:10D9600001487800C0B92000104078000080FB001A
:10D970004400DE0080407800B0B920000148780003
:10D98000B0B92000104078000080FB00100798001C
:10D990001E009000E10F50005E0032001E0090005B
:10D9A000E10F500004003C001E0090000000E00069
:10D9B00008003200970037001E009000E40F50006E
:10D9C0008C0032001E009000E60F50007A003200FA
:10D9D00090003700C0B92000104078000080FB00A4
:10D9E000000F78001E007800E30F50002600320080
:10D9F0001E007800E30F50000A003C001E00780073
:10DA0000E10F5000180032001E007800E10F5000B6
:10DA100017003C001E0078000000E000810032008A
:10DA2000380037001E007800E60F50002100320059
:10DA30001E007800E60F500004003C001E00780035
:10DA4000E40F5000160032002E0037001E00780050
:10DA5000E70F50001E0032001E007800EF0F50004C
:10DA600022003200270037009AFF0700B5FF370079
:10DA7000DE8102000000000010C0B30088720200C6
:10DA800000000000AFFF37001E820200000000000F
:10DA900010C0B3008872020000000000A9FF370028
:10DAA00004830200000000008872020000000000F1
:10DAB000A4FF37000040EB00748302000000000068
:10DAC00010C0B30088720200000000009DFF370004
:10DAD00010C0B300748302000000000010C0B30047
:10DAE000887202000000000096FF37000040EB0043
:10DAF000DFFE070010C0B3008872020000000000C3
:10DB000090FF37000040EB00887202000000000028
:10DB10008CFF3700C0B9200090407800F0C0B300FF
:10DB200080C06000C0B9200001487800C0B9200062
:10DB3000104078008040E800C0B92000014878001B
:10DB400010C0B30088720200000000008040EB00AB
:10DB5000A0B92000014878001000370022C2BF00A1
:10DB6000614060000004E000FCFF320030118000E2
:10DB7000B08202000000000052830200000000009A
:10DB80008872020000000000A0B920001040780058
:10DB90008040E800A0B9200001487800A0B920002A
:10DBA00090407800C0B920001040780080CF50002D
:10DBB000EAFF390063FF3700C0B9200090407800C9
:10DBC00030C0B30080C06000C0B9200001487800B8
:10DBD000C0B920009040780020C0B30050810200FE
:10DBE0000000000010C0B3008872020000000000B6
:10DBF00054FF3700C0B9200010407800B89E0200E2
:10DC00000000000010C0B300887202000000000095
:10DC10004CFF37000040EB0088720200000000005B
:10DC200048FF37000080FA00000006000200FA00FA
:10DC3000000F78001E00E0000300320010C3B300A4
:10DC4000330207000200370000C3B30030020700B0
:10DC50000080FA00000006000600FA001007980095
:10DC6000020037001E407800290207001E009000C5
:10DC7000104F78001E407800404798004E409000BA
:10DC80000004E0000200320010C0B30040479800DA
:10DC90004E4090009E0090008100E800110798001F
:10DCA0000004E000EFFF3A000080FA0000000600E8
:10DCB0000600FA0010079800020037001E407800A6
:10DCC000130207001E009000104F78001E407800DD
:10DCD000404798004E4090000004E00002003200EF
:10DCE00010C0B300404798004E4090009E00900046
:10DCF0008100E800110798000004E000EFFF3A00FF
:10DD0000D0C0B30002020700A0C0B30000020700A9
:10DD10000080FA00000006000400FA002047980086
:10DD200000C8B300004F7800C09D2800CAFF07005C
:10DD30000040EB00104798000F0037002E40900085
:10DD40001E4060000004E0000300320010C3B30076
:10DD5000EF0107000200370000C3B300EC01070029
:10DD60001E80FB000000D100004F78001E40900094
:10DD70000040E800104798001E409000E74F500018
:10DD8000EEFF36000080FA00000006000E00FA00E8
:10DD900050079800610798000040EB00004F7800A2
:10DDA00000102E00515F20003007980041079800B6
:10DDB0000040EB0010479800320037003E01900011
:10DDC000CE0190005E009000EE0090003006020050
:10DDD0000000000010079800210798001E04E000D2
:10DDE00005003A001E009000AE009000E00F5000C9
:10DDF000E08F5800180032001E0090000043B00071
:10DE0000C30107009E0090003E009000000AB80089
:10DE10009E0090004E0090000088B9000501780037
:10DE200000014100BE0090002E0090000088B90063
:10DE300000014100820278005E009000EE00900038
:10DE40000400500085805800500798006107980032
:10DE500010C0B300004F78003E009000CE0090004C
:10DE6000A200200003002000300602000000000095
:10DE700030079800410798001E4090000040E800DD
:10DE8000104798001E409000E74F5000CBFF36002F
:10DE90005E0090000043B0009D0107000080FA0082
:10DEA000000006000C00FA00400798005107980097
:10DEB0000000EB00100798000000EB00000F780056
:10DEC0006000B80020079800310798004E019000CC
:10DED000DE019000F0232400F1002000800F5100AB
:10DEE000818F5900210036004E009000DE00900026
:10DEF00002242400F300200030060200000000008D
:10DF000020079800310798002E0090006F0007004E
:10DF1000C0C2B3007E0107004E009000DE009000FA
:10DF200002242400F300200050060200000000003C
:10DF300040079800510798004E019000DE019000C4
:10DF4000703E200001002000800F5100818F590099
:10DF500002003E00F09D28003FFF07001000200057
:10DF60001007980010002000000F78004E0190006C
:10DF7000DE019000703E200001002000800F510063
:10DF8000818F5900320036004E009000DE00900074
:10DF9000823E200003002000300602000000000046
:10DFA00020079800310798002E019000BE019000D4
:10DFB0004006200001002000800F5100818F590091
:10DFC000030036002E0090004000070014003700C8
:10DFD0001E0090000000E0000F0032002E019000B3
:10DFE000BE019000A000200001002000800F510021
:10DFF000818F59000300360000C3B30044010700BD
:10E0000002003700409E280013FF07002E009000FA
:10E010002E000700020037002E0090002B000700A2
:10E02000C0C2B3003A0107004E009000DE0090002D
:10E03000823E200003002000500602000000000085
:10E04000400798005107980010002000000F78004A
:10E050004E019000DE0190004006200001002000EB
:10E06000800F5100818F5900030036004E00900050
:10E0700016000700130037001E00E0000F003200FA
:10E080004E019000DE019000A00020000100200061
:10E09000800F5100818F59000300360000C3B30088
:10E0A0001B01070002003700409E2800EAFE07001F
:10E0B0004E00900005000700020037004E0090005F
:10E0C000020007000080FA00000006000800FA00C5
:10E0D000300798000040EB00004F780000712200EC
:10E0E000200798000040EB00104798001E00370002
:10E0F0003E0090002E019000110009000280D8001F
:10E10000100798001E04E00003003A001E00900073
:10E110000000E0000C0032001E0090000043B00040
:10E12000FB0007009E0090002E0090000088B900C0
:10E13000800078003E0090000100500030079800F9
:10E1400010C0B300004F78002E009000A200200005
:10E15000110009000280D800200798001E4090009E
:10E160000040E800104798001E409000E34F500028
:10E17000DFFF36003E0090000043B000E4000700DF
:10E180000080FA00000006000600FA0040479800F0
:10E190000040EB00004F780040C6B30030479800C5
:10E1A0000040EB0020479800200037004E409000D0
:10E1B0008080FB003E4090000081FB0011000900C0
:10E1C0008280D800104798001E04E00003003A0047
:10E1D0001E4090000004E0000B0032001E40900042
:10E1E0000043B000CA0007004E4190009E409000DE
:10E1F0003E4090000088B900004051004047980020
:10E2000010C0B300004F78003E4090000080FB003B
:10E21000A2002000110009000280D80030479800B9
:10E220002E4090000040E800204798002E409000CB
:10E23000E14F5000DDFF36004E4090000043B0003B
:10E24000B30007000080FA00000006000400FA0096
:10E2500010079800709F28007FFE07001E009000A6
:10E260004400DE006F0F60009E007800709E280062
:10E270000080400010407800A50007001E009000BC
:10E280006F0F60009E007800709E280000804000A4
:10E29000104078009E0007000080FA000000060091
:10E2A0000400FA001007980000C3B300F60007004E
:10E2B00080C7B300F40007001E0090004400DE0099
:10E2C0006F0F60009E007800709E28000080400064
:10E2D00010407800EC0007001E0090006F0F6000F7
:10E2E0009E007800709E280000804000104078005A
:10E2F000E50007000080FA00000006000400FA00B4
:10E3000010079800709F280053FE07001E00900021
:10E310004C00DE006F0F60009E007800709E2800A9
:10E320000080400010407800790007001E00900037
:10E330004800DE006F0F60009E007800709E28008D
:10E340000080400010407800710007001E0090001F
:10E350004400DE006F0F60009E007800709E280071
:10E360000080400010407800690007001E00900007
:10E370006F0F60009E007800709E280000804000B3
:10E3800010407800620007000080FA0000000600DC
:10E390000800FA00300798003E009000CF80DE00B1
:10E3A000F403020000000000926C2200B33124004C
:10E3B0005204020000000000100798002107980096
:10E3C0001E009000AE009000560602000000000003
:10E3D000004F78001E4078006BFF0700E0C2B300DA
:10E3E0004B0007001E009000AE0090005606020091
:10E3F00000000000CF80DE00F403020000000000F7
:10E400000001BE001E009000AE009000D604020085
:10E41000000000001007980021079800020020006B
:10E42000031224001E009000AE009000920502002E
:10E430000000000010079800210798001E009000BF
:10E44000AE0090005606020000000000004F780069
:10E450001E4078004CFF07001E009000AE009000A8
:10E460005606020000000000CF80DE00F403020028
:10E47000000000000001BE001E009000AE009000F1
:10E48000D604020000000000100798002107980041
:10E4900002002000031224001E009000AE00900035
:10E4A0009205020000000000100798002107980064
:10E4B0001E009000AE009000560602000000000012
:10E4C000004F78001E4078002FFF07000080FA0000
:10E4D000000006000000FA0022C2BF006140600098
:10E4E0000080FB000080FA00000006000000FA0037
:10E4F00022C2BF00614060000004E000FCFF320067
:10E50000301180000080FB000080FA00000006004F
:10E510000200FA00004F7800D04080000110200077
:10E52000010060000000E00006003A0023C2BF00C6
:10E53000624060000004E000FCFF3A001E00FB00A7
:10E54000201188000080FA00000006000200FA0096
:10E55000004F78001E80FB00401188000080FA0008
:10E56000000006000000FA0095C0BF007040600087
:10E570000004E00010003A0051408000404080005C
:10E58000808F50000C00320023C2BF006240600048
:10E590000004E000FCFF3A008580A9009580A800F7
:10E5A00031408000404080000080400010407800F2
:10E5B0000080FB00201188000080FA0000000600A7
:10E5C000809FBE000000FA000140800020408000D3
:10E5D000808040003011800080487800204080001A
:10E5E0000000E800204088002140800010408000AA
:10E5F000808F500001003A009560A9008560A90055
:10E600000080FA004F00BE0000400600809FBE0060
:10E610000000FA00404080000000E8004040880010
:10E620004140800050408000808F500002003A003E
:10E630009580A900060037003140800040408000EE
:10E6400000804000104078000080FB00201188000E
:10E650008580A9000080FA004F00BE00004006003F
:10E660000000FA000000EB00906E8800100020000F
:10E67000806E8800D040800000A0A100D0408800BB
:10E680000080FA00000006000200FA00004F780047
:10E69000816E8000906E8000808F500005003A00EF
:10E6A000CA82A900D040800000A0A000D04088000D
:10E6B0000E00370071408000806E80008080400036
:10E6C0001E40780080487800806E80000000E800DE
:10E6D000806E8800816E800000002100808F5000D5
:10E6E00002003A000000EB00806E88000080FA0013
:10E6F000000006000200FA00906E8000000FE800A3
:10E70000000021009E0F100002003A000000EB0004
:10E71000000F7800806E80009E0F10000C00320009
:10E7200023C2BF00624060000004E00008003A001D
:10E730001E007800906E880071408000906E80000E
:10E7400000804000104078000080FB00201188000D
:10E750000080FA00000006000200FA000000370006
:10E76000906E8000000FE800000021009E0F100056
:10E7700002003A000000EB00000F7800806E80007D
:10E780009E0F10000D00320023C2BF0062406000E7
:10E790000004E000F2FF3A001E007800906E88004E
:10E7A00071408000906E8000008040001040780032
:10E7B0000080FB0020118800E9FF37000080FA008C
:10E7C000000006000400FA00000F7800110798000E
:10E7D0001E007800900188001E0090001080BA0092
:10E7E000C800DD001E0090001000BA00008070001C
:10E7F0000080FA00000006000600FA000000EB00AE
:10E80000800888000000EB00F00888000000EB00A2
:10E81000E00C8800206180000000E00008003A0061
:10E82000A16C20009140780000CEB30000C06000D1
:10E83000CAE6B7000000EB00B06088003D0037007A
:10E8400020618000E30F500005003C00E003200041
:10E85000000F780010A1A8001081A8001500370053
:10E8600020618000FE0F500005003C00A00F20003A
:10E87000000F780010A1A8001081A9000D0037003A
:10E8800021618000400F2000808F500005003C0077
:10E89000007D2000000F780010A1A9001081A800C1
:10E8A0000400370000E82300000F780010A1A90041
:10E8B0001081A90020618000000178001E0078000E
:10E8C000110009000280D8000000E900200798002C
:10E8D0002E00900060088800306180008000780081
:10E8E0002E0090000088B9004206200011000900A7
:10E8F0000280D80010079800A16C20009140780099
:10E9000000CEB30000C060006041B300CAE6B700AB
:10E910001E009000D00C88001E009000C00C8800E3
:10E9200060002000E00C880011E1A8002000200019
:10E93000B06088000080FA00000006001200FA00B3
:10E940000000EB00800888000000EB00F008880061
:10E950000000EB00E00C8800B0608000E20F500087
:10E9600014003A00A16C20009140780000CEB30062
:10E9700000C06000CAE6B700C1002000C02E200021
:10E98000629C0200000000000000EB00B060880004
:10E99000506980008000E800F00F20008080600057
:10E9A00080C2200000804000104078000004E00099
:10E9B000AE0032000000EB00200798005069800094
:10E9C0000000E8005069880051698000F00F2000C5
:10E9D0000080600050698800A81A02000000000052
:10E9E000D21602000000000040079800A81A02009A
:10E9F00000000000D216020000000000CF80DE0000
:10EA0000F403020000000000008FBE004E009000E2
:10EA10000000E00007003200CE009000F0F9200076
:10EA2000808F500003003E002E0090000000E800A0
:10EA3000200798006011B8001E00BE004A040200C2
:10EA4000000000000000E00001003C000B00370067
:10EA500002002000832C24001E00BE004E04020091
:10EA6000000000000000E000010035000300370056
:10EA70002E0090000000E800200798002E00900073
:10EA8000E20F5000110032000000EB0060698800C6
:10EA900011012000802F2000629C02000000000075
:10EAA0001101200090302000D89B020000000000DF
:10EAB0008001EB0002FA200011002000200320005A
:10EAC0001E1D020000000000400798004E0090004C
:10EAD000E30F500005003E00E003200030079800DF
:10EAE00010A1A8001081A800150037004E0090006A
:10EAF000FE0F500005003E00A00F200030079800D8
:10EB000010A1A8001081A9000D003700CE009000D0
:10EB1000400F2000808F500005003E00007D200047
:10EB20003007980010A1A9001081A8000400370048
:10EB300000E823003007980010A1A9001081A90067
:10EB40003E0090004E019000110009000280D800A4
:10EB50000000E900600798002E009000E20F5000CE
:10EB60000E0032000101200070322000D89B02000C
:10EB7000000000008001EB00320620008000EB0066
:10EB8000200320001E1D020000000000CF80DE00D8
:10EB9000F403020000000000008FBE00020020000D
:10EBA000832C24001E00BE0052040200000000005E
:10EBB000008FBE006E009000CF80DE00F4030200E4
:10EBC0000000000070079800010F98006E00900090
:10EBD0000000E00008003D0002002000037824004F
:10EBE0007E0090008E089000D80402000000000013
:10EBF00070079800010F98001E01BE007E00900073
:10EC00008E0890009205020000000000FA05020044
:10EC10000000000050079800A16C2000914078008F
:10EC200000CEB30000C060006041B300CAE6B70088
:10EC30005E009000D00C88005E009000C00C880040
:10EC400060002000E00C88006E00900060088800E2
:10EC500011E1A800A100200070332000629C020096
:10EC60000000000020002000B06088000080FA0052
:10EC7000000006000000FA00B0608000E20F5000C3
:10EC800005003A00F101200010342000629C0200CF
:10EC9000000000003E003700F10020000036200098
:10ECA000D89B0200000000000000EB00F008880084
:10ECB0000000EB0080088800C942A80061682000BD
:10ECC0009140780000CEB30000C06000A040B300C7
:10ECD00086E6B700A0032000800888002E00070009
:10ECE000C0608800D1608800C2608000D36080006E
:10ECF000F00F200001002000800F5100818F59008B
:10ED000009003600C0608000D1608000C808DD00C6
:10ED10000080FD00804078000040EB00C06088006B
:10ED2000D160880009003700B1002000B01921002F
:10ED3000D89B020000000000A0002000800888008E
:10ED400015000700C0608800D1608800C0608000A6
:10ED5000D1608000526F02000000000040A3280034
:10ED60002C6E02000000000080A32800586E0200F4
:10ED70000000000086C6BF00F041B30086E6B70081
:10ED80000000EB00F00888000000EB00800888001D
:10ED90000080FA00000006000000FA000080EB008E
:10EDA000700888000080EB00600888000000EB001D
:10EDB000400888000000EB00300888000000EB00ED
:10EDC000B00888000000EB00A00888008000200048
:10EDD000F0088800400F2000E00888000040220072
:10EDE000D00888008780A9001FE1A80011E1A800D1
:10EDF00087C0BF00704060000004E000FCFF3200EC
:10EE000011E1A9001FE1A90030088000106188000D
:10EE1000400880000061880000618000010020003F
:10EE2000E0608800F1608800E0608000F1608000B0
:10EE3000C000DD0000002000E0608800F160880074
:10EE4000106180006101B800E0608000F160800026
:10EE50000200400083804800E0608800F160880084
:10EE6000E0608000F16080000080FA000000060091
:10EE70000000FA0080B82000104078006140600077
:10EE80000004E00002003A00C942A8000100370077
:10EE9000C8C2A800E1002000F0362000D89B020084
:10EEA000000000000080FA00000006000000FA00E8
:10EEB00080B8200010407800614060000004E0004D
:10EEC00003003A00C942A900CB42A8000200370063
:10EED000C8C2A900CAC2A80081002000D037200003
:10EEE000629C0200000000000080FA0000000600A2
:10EEF0000000FA0080B820001040780061406000F7
:10EF00000004E00003003A00C942A900CB42A90076
:10EF100002003700C8C2A900CAC2A90071002000BF
:10EF200050382000629C0200000000000080FA00BF
:10EF3000000006000200FA0080B8200010407800AF
:10EF4000614060000004E00009003A00C942A800E6
:10EF50000000000000000000CBC2BF000080FB00EA
:10EF60004200DE0061406000004F7800080037007A
:10EF7000C8C2A8000000000000000000CAC2BF0014
:10EF80000080FB004600DE0061406000004F78001A
:10EF90001E80FB000080FA00000006000C00FA0052
:10EFA0000000EB00800888000000EB00F0088800FB
:10EFB0000000EB00E00C8800B0608000E20F500021
:10EFC00014003A00A16C20009140780000CEB300FC
:10EFD00000C06000CAE6B700C1002000C02E2000BB
:10EFE000629C0200000000000000EB00B06088009E
:10EFF000506980008000E800F00F200080806000F1
:10F0000080C2200000804000104078000004E00032
:10F0100066003200506980000000E80050698800F6
:10F0200051698000F00F2000008060005069880066
:10F03000A81A020000000000D21602000000000022
:10F04000CF80DE00F403020000000000008FBE004D
:10F05000606980000000E00008003A000200200023
:10F06000433324001E00BE004A04020000000000DA
:10F070000000E00001003C00100037000000EB0041
:10F08000606988003101200040242100629C020058
:10F09000000000008001EB00420B20008000EB002C
:10F0A000A00520001E1D020000000000CF80DE0031
:10F0B000F403020000000000008FBE0010A1A800B1
:10F0C0001081A800204E20003007980002002C007C
:10F0D000A35524001E00BE005204020000000000E0
:10F0E000008FBE003E009000CF80DE00F4030200DF
:10F0F0000000000040079800510798003E00900073
:10F100000000E00008003D00020020000378240019
:10F110004E009000DE009000D804020000000000C5
:10F1200040079800510798001E01BE004E00900055
:10F13000DE009000920502000000000002002000A6
:10F1400083272400D804020000000000FA05020012
:10F150000000000020079800A16C2000914078007A
:10F1600000CEB30000C060006041B300CAE6B70043
:10F170002E009000D00C88002E009000C00C88005B
:10F1800060002000E00C88003E00900060088800CD
:10F1900011E1A800C100200070252100629C02003E
:10F1A0000000000020002000B06088000080FA000D
:10F1B000000006000000FA0000A428002C6E0200E7
:10F1C000000000000080FA00000006000200FA00C3
:10F1D000CA82A800FC000700F6FF07000000370005
:10F1E000F00007008040780060DE200001487800D1
:10F1F00060DE2000104078000004E000E3003500ED
:10F2000060DE2000104078000004E00002003A00B8
:10F21000E8FF0700F2FF370060DE200010407800B2
:10F22000E14F500006003A00E7000700DA4A02000A
:10F2300000000000E4000700DEFF0700E8FF3700E1
:10F2400060DE200010407800E24F500006003A00D7
:10F25000DD000700766C020000000000DA00070005
:10F26000D4FF0700DEFF370060DE2000104078008A
:10F27000E34F500006003A00D30007008453020019
:10F2800000000000D0000700CAFF0700D4FF3700CD
:10F2900060DE200010407800E44F500006003A0085
:10F2A000C90007007A5E020000000000C6000700E7
:10F2B000C0FF0700CAFF370060DE20001040780062
:10F2C000E54F500006003A00BF0007005E600200F4
:10F2D00000000000BC000700B6FF0700C0FF3700B9
:10F2E00060DE200010407800E64F500006003A0033
:10F2F000B5000700AE8E020000000000B20007005B
:10F30000ACFF0700B6FF370060DE20001040780039
:10F31000E74F500004003A00AB000700AA000700C6
:10F32000A4FF0700AEFF370060DE20001040780029
:10F33000EF4F50000A003A0010C0B300887202007C
:10F3400000000000CA82A90023C2BF006140600023
:10F350000004E000FCFF32000000FE00A0FF3700C8
:10F3600060DE200010407800F24F500035003A0077
:10F370000000EB00800888000000EB00F008880027
:10F380000000EB00E00C8800A16C200091407800A8
:10F3900000CEB30000C060006041B300CAE6B70011
:10F3A000800007000080FB00000F78001E0078003E
:10F3B0000000D100610060000004E00001003200A4
:10F3C00010A1A8009E007800618060000004E000A9
:10F3D000010032001081A800720007000080FB00CD
:10F3E0004800DD00000F78006E0007000080FB0081
:10F3F0001E0F70001E007800D00C88009E00780060
:10F40000C10C880060002000E00C88006500070047
:10F410000080FB004800DD00000F7800610007005D
:10F420000080FB001E0F70001E007800600888003E
:10F4300011E1A80010C0B3008872020000000000B3
:10F4400067FF370060DE200010407800F34F500067
:10F450000D003A000000EB00800888000000EB007F
:10F46000E00C8800A16C20009140780000CEB30031
:10F4700000C06000CAE6B70010C0B3008872020086
:10F480000000000056FF370060DE200010407800CA
:10F49000F44F50000E003A0021E3A800C0C0B300B2
:10F4A000DC97020000000000000F780021E3A900B3
:10F4B0001E0078004800DE00887202000000000094
:10F4C0001E007800887202000000000044FF370030
:10F4D00060DE200010407800F54F500018003A0020
:10F4E00021E3A800C0C0B300DC97020000000000C8
:10F4F000000F780023C2BF00614060000004E000FC
:10F50000FCFF32001E0078004800DE008872020016
:10F51000000000001E007800887202000000000059
:10F5200022C2BF00614060000004E000EDFF320035
:10F5300031118000010F780021E3A90028FF370076
:10F5400060DE2000104078000080FB004500DE00F7
:10F550000080FB000000D100610060000004E000BA
:10F560000600320060DE2000104078001F00070017
:10F57000887202000000000019FF37000040EB0015
:10F58000887202000000000015FF370060DE2000D6
:10F5900010407800A50007008872020000000000FB
:10F5A0000FFF37000000FA0022C2BF006140600078
:10F5B0000004E000FCFF3200301180000080FB00FE
:10F5C0000080FA00000006000000FA0000C0EB0016
:10F5D000060007000040EB0094000700C962A90084
:10F5E000CB62A9000080FA00000006000400FA00C7
:10F5F000204798000040EB00004F78002E4090001C
:10F600000080FB004400DE00610060000004E000B8
:10F610000200320010C0B300004F78009E40780016
:10F6200061C06000614060004201DD00912C20005B
:10F6300091407800B0CFB30000C06000024070007D
:10F64000C9E2B7000040EB00004F78002E40900068
:10F650000080FB004300DE00610060000004E00069
:10F660000200320010C0B300004F78009E407800C6
:10F6700061C060006140600000414000912C2000AA
:10F6800091407800D0CFB30000C06000024070000D
:10F69000C9E2B7000040EB00004F78002E40900018
:10F6A0000080FB004200DE00610060000004E0001A
:10F6B0000200320010C0B300004F78009E40780076
:10F6C00061C0600061416000912C20009140780091
:10F6D000E0CFB30000C0600002407000C9E2B70094
:10F6E0000040EB00004F78002E4090000080FB00AF
:10F6F0000000D100610060000004E0000200320060
:10F7000010C0B300004F78009E40780061C06000D8
:10F71000C700DD00C8C2BF000074A1000140700036
:10F72000C8E2B7000040EB00004F78002E40900088
:10F730000080FB00610060000004E0000200320075
:10F7400010C0B300004F78009E40780061C0600098
:10F75000614060004601DD00812C2000914078006E
:10F76000F0CBB30000C0600002407000C8E2B700F8
:10F77000500020006699020000000000AE4090009A
:10F7800000CEB30000C0600020479800CBC2BF008D
:10F79000644060000004E000030032002E4090004E
:10F7A0000044A00020479800CBC2BF006240600028
:10F7B0000004E000030032002E4090000034A0005E
:10F7C00020479800CBC2BF00614060000004E00009
:10F7D000030032002E4090000024A0002047980033
:10F7E000CAC2BF0001C8B300014060000004E000CD
:10F7F000030032002E4090000014A0002047980023
:10F80000CAC2BF000044B2000004E000030032009E
:10F810002E4090000004A000204798002E40900049
:10F820000080FB000080FA00000006000400FA00DF
:10F83000204798002E4090000080FB004600DE002C
:10F84000610060000004E00005003200C082A900F1
:10F85000C282A800C8A2A900CAA2A800040037005A
:10F86000C082A900C282A900C8A2A900CAA2A90098
:10F870000040EB00004F78002E4090000080FB001D
:10F880004400DE00610060000004E000020032007D
:10F8900010C0B300004F78009E40780061C0600047
:10F8A000614060004201DD00B12C200091407800F1
:10F8B000B0CFB30000C0600002407000CBE2B700E0
:10F8C0000040EB00004F78002E4090000080FB00CD
:10F8D0004300DE00610060000004E000020032002E
:10F8E00010C0B300004F78009E40780061C06000F7
:10F8F0006140600000414000B12C20009140780040
:10F90000D0CFB30000C0600002407000CBE2B7006F
:10F910000040EB00004F78002E4090000080FB007C
:10F920004200DE00610060000004E00002003200DE
:10F9300010C0B300004F78009E40780061C06000A6
:10F9400061416000B12C200091407800E0CFB3000D
:10F9500000C0600002407000CBE2B7000040EB0046
:10F96000004F78002E4090000080FB000000D10086
:10F97000610060000004E0000200320010C0B3002B
:10F98000004F78009E40780061C06000C700DD0035
:10F99000CAC2BF000074A10001407000CAE2B700F3
:10F9A0000040EB00004F78002E4090000080FB00EC
:10F9B000610060000004E0000200320010C0B300EB
:10F9C000004F78009E40780061C060006140600098
:10F9D0004601DD00A12C200091407800F0CBB3005F
:10F9E00000C0600002407000CAE2B7005000200072
:10F9F0006699020000000000AE40900000CEB30007
:10FA000000C0600020479800CBC2BF006440600087
:10FA10000004E000030032002E4090000044A000EB
:10FA200020479800CBC2BF00624060000004E000A5
:10FA3000030032002E4090000034A00020479800C0
:10FA4000CBC2BF00614060000004E0000300320050
:10FA50002E4090000024A00020479800CAC2BF009A
:10FA600001C8B300014060000004E0000300320060
:10FA70002E4090000014A00020479800CAC2BF008A
:10FA80000044B2000004E000030032002E40900069
:10FA90000004A000204798002E4090000080FB004A
:10FAA0000080FA00000006000000FA0080B8200084
:10FAB000104078000030A00081B820008048780015
:10FAC000960007000080FA00000006000000FA001F
:10FAD0003C01070053000700302721001040780048
:10FAE0000080FB000080FA00000006000400FA001D
:10FAF000100798001E00900071010700004F780069
:10FB00001E04E00005003A003100200010442000EF
:10FB1000D89B0200000000000C00370010C0B300AA
:10FB20009E4F100005003A00410020004044200094
:10FB3000D89B020000000000040037008100200074
:10FB400000122100D89B02000000000000102000DD
:10FB50000080FA00000006000400FA00000F7800A0
:10FB60001E007800100798001E0090000000E000C2
:10FB7000040032001E009000E10F50000600320029
:10FB8000220037006102200080122100629C0200E6
:10FB90000000000021003700D1002000E014210007
:10FBA000629C020000000000F1002000C01E210045
:10FBB000629C020000000000020107000004E00057
:10FBC00008003A0030272100104078000080FB0038
:10FBD000949802000000000000C2B3008872020086
:10FBE0000000000022C2BF00614060000004E0008D
:10FBF000F1FF320030118000000F780020A62800AD
:10FC0000586E02000000000004003700410220008E
:10FC1000C0202000629C0200000000000080FA006A
:10FC2000000006000400FA00004F78001E80FB0070
:10FC3000100798009E009000E28F50001A003200DA
:10FC40001E009000E20F500007003C009E00900054
:10FC50000100E0002F0032001E009000E10F500074
:10FC60000C003200270037009E009000E48F500007
:10FC7000170032001E009000E40F50000F00350006
:10FC8000F00F20009E009000808F5000180032007E
:10FC90001C00370001012000B0152100629C020009
:10FCA000000000001B003700E1002000B01621001A
:10FCB000629C02000000000016003700F1002000E6
:10FCC00090172100629C0200000000001100370024
:10FCD00000C2B30088720200000000008100200012
:10FCE00000122100D89B020000000000090037002C
:10FCF0005100200080182100629C020000000000DA
:10FD000004003700E1002000D0182100629C0200AE
:10FD1000000000000080FA00000006000000FA0069
:10FD2000C922A800C902A900CB02A900CB22A900C0
:10FD30000080FA00000006000400FA000040EB001A
:10FD4000410107000004E000030032002000200011
:10FD5000100798000E003700CBC2BF000080FB00E8
:10FD60000000D10061406000004F780010C0B30077
:10FD7000350107000004E0000300320020002000ED
:10FD800010079800020037001E80FB001007980043
:10FD90001E0090000080FA00000006000600FA0035
:10FDA0000040EB00204798000040EB00104798000F
:10FDB000CBC2BF000080FB000000D100E14060002A
:10FDC000202721001040780061C16000E1CFB3001E
:10FDD0000140600002407000212721008048780027
:10FDE0002027210010407800614060000004E000FE
:10FDF0000300320010002000200798006E0037003A
:10FE000010C0B300100107000004E000030032003E
:10FE10004100200021079800670037000040EB00F8
:10FE200030479800190037001E4090000080FB000A
:10FE30000000D10010479800BFFF0700004F780076
:10FE400020C0B3009E4F100003003A004100200084
:10FE5000210798005800370010C0B3009E4F1000D3
:10FE600007003A009E40900000C8B30000C0400068
:10FE7000104798002E4090000004A20020479800F0
:10FE80003E4090000040E800304798003E4090001F
:10FE9000E74F5000E4FF3600302721009E409000DD
:10FEA00001487800A4FF0700004F780020C0B3008D
:10FEB0009E4F100003003A004100200021079800E7
:10FEC0003D0037001E407800E140600040272100DF
:10FED0001040780061C16000E1CFB30001406000D4
:10FEE000024070004127210080487800402721000F
:10FEF00010407800614060008080FB002E40900040
:10FF00000080FB00808F500008003A00402721004D
:10FF1000104078000020A000412721008048780090
:10FF200021002000210798002300370040272100EE
:10FF3000104078000020A10041272100804878006F
:10FF40007DFF0700004F780020C0B3009E4F1000D7
:10FF500003003A00410020002107980016003700F6
:10FF60001E407800614160004027210090407800E9
:10FF70006140610000414000D0CFB30080C060000C
:10FF800082C070004027210001487800C902A90002
:10FF90004027210010407800624060000004E0002B
:10FFA00003003A00310020002107980002003700CA
:10FFB0000000EB00200798002E0090000080FA005F
:10FFC000000006000200FA0000C0EB00004F7800BD
:10FFD000C922A800C902A8000040EB001047980001
:10FFE00011003700CBC2BF00614060000004E00098
:10FFF00007003A0069FF0700004F78001E04E00088
:020000040001F9
:100000000C00320040C0B3009E4F100009003200C7
:100010005000200066990200000000001E40900081
:100020000040E800104798001E409000E14F40005B
:10003000ECFF3A00C902A9001E80FB000080FA0014
:10004000000006000400FA00004F780010C0B30062
:100050007D0007000004E0000300320020002000C3
:1000600010079800130037009E40780061C06000C0
:100070006140600000414000912C200091407800D8
:10008000D0CFB30000C0600002407000C9E2B700EA
:100090000040EB006C0007000004E00003003200A9
:1000A0002000200010079800020037008000EB00BD
:1000B000110798001E0090000080FA000000060062
:1000C0000800FA00404798000040EB0020479800E5
:1000D000C902A900CB02A900C00320006699020052
:1000E00000000000CB22A900C922A900C902A80073
:1000F0001000200066990200000000000040EB00A4
:10010000510007000004E00003003200400020001E
:1001100030079800490037000000EB00000F78001E
:100120001C0037004E4090000080FB006100600022
:100130000004E0000B00320010C0B300C1FF070054
:100140000004E00003003200400020003007980067
:100150003A0037002E4090000004A200204798008B
:10016000070037000040EB00B6FF07000004E00086
:100170000300320040002000300798002F003700B5
:100180004E4090000080FB000000D10040479800E6
:100190001E0FE800700020009E0F1000E1FF3600E7
:1001A0002E4090000004A200204798002E409000AE
:1001B000A4FF07000004E00003003200400020001C
:1001C000300798001D003700C922A800CB22A900E3
:1001D00010C0B3001C0007000004E0000300320060
:1001E000400020003007980014003700D2FE0700BE
:1001F000E24F500003003A00400020003007980012
:100200000E003700CCFE07000080FB00000F7800D6
:10021000200020009E0F100003003A004000200044
:100220003007980005003700C902A900CB02A900D9
:100230001E0078000080FB00300798003E00900010
:100240000080FA00000006000600FA00204798002F
:100250000080EB00000F7800CBC2BF00614060005F
:100260008080FB002E4090000080FB00808F5000BB
:1002700003003A000000EB0020079800050037005B
:100280001E0FE9001E00E000F3FF3A0010002000FE
:10029000200798002E0090000080FA000000060061
:1002A0000400FA00004F780011479800C0DD2000DC
:1002B0001E48780030C0B3009E4F100005003A0081
:1002C00000202000F06E880000082000006F8800E9
:1002D0000400370000202000F06E8800002020007D
:1002E000006F88001E4090000080FB0010079800FF
:1002F0001E009000E10F5000110032001E0090001F
:10030000E20F5000180032001E0090000000E000D4
:10031000010032001E00370041C1B30020DE200082
:100320000148780041C6B30030DE20000148780063
:1003300021C3B30040DE2000014878001D003700D3
:1003400021C0B30020DE200001487800A1C0B30026
:1003500030DE20000148780051C0B30040DE2000AC
:10036000014878001300370011C0B30020DE2000E0
:100370000148780051C0B30030DE20000148780009
:1003800021C0B30040DE200001487800090037009A
:100390008040EB0020DE2000014878008040EB0028
:1003A00030DE2000014878008040EB0040DE200075
:1003B000014878000080FA00000006000200FA0000
:1003C0000000EB00000F780030DE20009040780045
:1003D0000030200009010700CBC2BF00614060006F
:1003E0000004E00004003200CBC2BF0062406000A5
:1003F0000004E00002003A0010002000000F780026
:1004000030DE200090407800002020001701070017
:1004100030DE20009040780000102000130107001B
:1004200030DE20009040780000202000F30007001C
:100430001E0078000080FA00000006000000FA00AC
:1004400030DE2000904078000030200007010700D7
:1004500030DE20009040780000102000E700070008
:1004600030DE20009040780000202000E3000700EC
:100470000000EB000080FA00000006000C00FA000B
:10048000500798000000EB00000F780070B72000C4
:10049000104078000080FB008000E9001000200080
:1004A0000100DD00300798005E00900020079800F2
:1004B0000000EB00400798002000370020DE2000FD
:1004C00010417800AE0090003E0090000080600077
:1004D00001202000FC00070030DE20009040780062
:1004E00000102000C50007000008200026010700BA
:1004F0000080FB001007980030DE2000904078005C
:1005000000102000D90007002E00900000004000DD
:10051000200798001E00780000004000000F7800BF
:100520001E0090000000E000010032001E0FE800F5
:100530004E0090000000E8004007980070B72000CF
:10054000104078008080FB004E009000808F5000AB
:10055000DAFF3E001E0078000080FA00000006006E
:100560000800FA003007980070B7200010407800AB
:100570000080FB008000E900100020000100DD0089
:10058000100798003E009000000F78000000EB007C
:10059000200798001400370020DE2000104178006A
:1005A0001E0090001E00600001202000C600070011
:1005B00030DE200090407800001020008F000700FF
:1005C00030DE20009040780000102000A7000700D7
:1005D0001E00780000004000000F78002E00900000
:1005E0000000E8002007980070B720001040780055
:1005F0008080FB002E009000808F5000E6FF3E00C0
:100600000080FA00000006000600FA000000EB007F
:10061000000F780000202000DB0007000000EB0046
:10062000200798001600370030DE20009040780048
:10063000001020007100070000202000D2000700F9
:100640000080FB001007980030DE2000904078000A
:1006500000102000850007001E0078000000400008
:10066000000F78001E0090000000E0000100320042
:100670001E0FE8002E0090000000E8002007980000
:1006800070B72000104078008080FB002E009000A2
:10069000808F5000E4FF3E001E0078000080FA00CA
:1006A000000006000200FA00006F8000B60007009C
:1006B00030DE200090407800001020004F0007003E
:1006C000006F8000B0000700004F780030DE20008F
:1006D0009040780000102000640007001E80FB009E
:1006E0000080FA00000006000200FA00004F7800C7
:1006F00020DE200010417800F16E80001E80FB009B
:100700007100070030DE20009040780000102000CB
:100710003A00070030DE20009040780000102000F2
:10072000520007000080FA00000006000400FA00F2
:10073000204798000040EB00004F78000900370088
:1007400030DE200090407800001020002B000700D1
:1007500030DE2000904078000010200043000700A9
:100760001E4FE8002E4090009E4F1000F4FF39000D
:100770000080FA00000006000200FA00004F780036
:1007800020DE200010417800F16E80001E80FB000A
:100790004D0007000080FA00000006000200FA0089
:1007A000004F780020DE2000104178001E80FB0002
:1007B00001102000440007000080FA00000006003D
:1007C0000200FA00004F780020DE2000104178007F
:1007D0001E80FB00010420003B0007000080FA009F
:1007E000000006000000FA00006F800066000700AD
:1007F0000080FB000080FA00000006000400FA0000
:10080000000F78002147980080B820001040780041
:10081000684060000004E0000B003A0060168000B1
:100820001E007000601688001E0078000080EA003C
:100830008180EA008000780040168000008060001F
:100840004016880003003700401680001E0070002C
:10085000401688002E4090000080FB006699020040
:10086000000000000080FA00000006000400FA000A
:10087000000F7800214798001E0078000080EA00F1
:100880008180EA00800078006016800000806000AF
:10089000601688001E0078000080EA008180EA006F
:1008A00080007800401680000080600040168800BC
:1008B0002E4090000080FB006699020000000000BE
:1008C0000080FA00000006000600FA00000F780021
:1008D00011079800424798001E00E0000F003A0000
:1008E0001E0090000080EA008180EA00800078000D
:1008F0006016800000806000601688001E00900076
:100900000080EA008180EA008000780040168000C4
:1009100000806000401688001500370080B8200075
:1009200010407800684060000004E0000C003A00CD
:10093000611680001E009000008070006016880024
:100940001E0090000080EA008180EA0080007800AC
:1009500040168000008060004016880004003700C8
:10096000401680009E009000010070004016880034
:100970004E4090000080FB006699020000000000DD
:100980000080FA00000006000400FA00000F780062
:10099000401680001E007000401688000000000015
:1009A0000000000000000000501680001E006000E3
:1009B0000000E00003003200100020001007980043
:1009C000020037000000EB00100798001E009000A6
:1009D0000080FA00000006000000FA000483020014
:1009E000000000000080FA00000006000200FA008B
:1009F000000F78001E007800B082020000000000A6
:100A0000001020000080FA00000006000000FA003C
:100A1000DE8102000000000081002000D092200052
:100A2000D89B020000000000D1002000804420007C
:100A3000629C0200000000000080FA000000060036
:100A40000000FA001E820200000000006100200089
:100A500050932000D89B020000000000C10020003D
:100A600050452000629C0200000000000080FA0057
:100A7000000006000000FA0052830200000000009F
:100A80000080FB000080FA00000006000000FA0071
:100A9000F2830200000000000080FB000080FA00EA
:100AA000000006000000FA000040EB00CE830200C8
:100AB000000000000080FA00000006000000FA00BC
:100AC00010C0B300CE830200000000000080FA00D6
:100AD000000006000000FA0010C0B3009683020078
:100AE000000000000080FA00000006000000FA008C
:100AF0000040EB00BC830200000000000080FA0010
:100B0000000006000000FA0010C0B300BC83020021
:100B1000000000000080FA00000006000000FA005B
:100B200001012000A0982000D89B020000000000D6
:100B300060B7200010407800C47002000000000080
:100B400000C2B300887202000000000080B82000DC
:100B5000104078000080FB004300DE006140600030
:100B6000C47002000000000000C2B30088720200DE
:100B70000000000031002000F0AD2000D89B0200F2
:100B8000000000000080FA00000006000400FA00E7
:100B9000A81A020000000000D216020000000000A7
:100BA00010079800A81A020000000000D2160200E8
:100BB00000000000000F78001E0090000000E00020
:100BC000090034001E009000E40F500006003C00B5
:100BD0001E0090000040E9008040780060B72000CF
:100BE00001487800020037000000EB001007980071
:100BF0001E00E00010003400200020009E0F1000B6
:100C00000D003C001E0078000040EA0061416000D9
:100C100080B8200090407800614061004301DD0011
:100C200070CFB30080C0600082C0700080B8200028
:100C300001487800020037000000EB001007980020
:100C40001E0090000000E00026003A000000EB00CB
:100C500060698800B103200060482000629C0200A7
:100C6000000000008001EB00420020001100200085
:100C7000100020001E1D0200000000000040E900DE
:100C80008040780060B7200001487800F10420001F
:100C9000B0932000629C0200000000008001EB0085
:100CA0002200200011002000100020001E1D020064
:100CB000000000000040EA006141600080B82000B0
:100CC00090407800614061004301DD0070CFB300C7
:100CD00080C0600082C0700080B8200001487800A9
:100CE000010037008DFF0700CB02A900CB22A9002D
:100CF000C922A800C902A90060B72000904078006E
:100D000020C0B30050810200000000000080FA0003
:100D1000000006000400FA00000F78001E007800B2
:100D2000100798001E009000E10F50000C003200E8
:100D30001E009000E10F5000040039001E009000DA
:100D4000E20F500007003200080037008103200046
:100D5000A0992000D89B0200000000000700370087
:100D600010000700250007000400370041022000A2
:100D7000C0202000629C0200000000000080FA00F9
:100D8000000006000200FA00000F7800B100200009
:100D9000C0092100629C0200000000000080FA00EF
:100DA000000006000000FA00F1032000209D200052
:100DB000629C0200000000000040EB00E0830200A3
:100DC00000000000F00F2000669902000000000003
:100DD00010C0B300E08302000000000010C0B300A8
:100DE00096830200000000000040EB00E083020058
:100DF000000000000080FA00000006000A00FA006F
:100E0000881F7800D102200010A12000D89B02008A
:100E1000000000000000EB00000F78001000370019
:100E20001E04780004830200000000008040780067
:100E300063004700017478009E007800630047005B
:100E4000614078000080FB00267102000000000075
:100E500000C2B30088720200000000001E0FE8000C
:100E6000300020009E0F1000EDFF3600A0A52800E6
:100E7000586E020000000000A1002000E0A3200046
:100E8000D89B02000000000063004700104078007B
:100E90000080FB004400DE000080FB00400798005B
:100EA0004E009000E90F5000130032004E009000F9
:100EB000E90F500004003C004E009000E80F500085
:100EC000080032001B0037004E009000EA0F50006F
:100ED0000E0032004E009000EF0F50001000320064
:100EE000140037006100200080A42000D89B02007D
:100EF000000000001300370061002000E0A4200083
:100F0000D89B0200000000000E00370061002000A6
:100F100040A52000D89B0200000000000900370017
:100F200031002000A0A52000D89B02000000000096
:100F30000400370071002000D0A52000D89B0200DB
:100F400000000000A0A52800586E0200000000006C
:100F5000B100200040A62000D89B02000000000045
:100F600063004700104090000080FB004700DE0057
:100F70000004E00005003A0061002000F0A6200017
:100F8000D89B02000000000004003700F1002000A0
:100F900050A72000D89B020000000000A0A5280058
:100FA000586E020000000000C100200040A8200090
:100FB000D89B020000000000630047001040900032
:100FC0008080FB0080F72F00008060004380DE00FF
:100FD000204798002E4090000004E00005003A00F1
:100FE000D100200000A92000D89B020000000000D2
:100FF0001E0037002E409000EF4F500005003A00D1
:1010000031002000A0A52000D89B020000000000B5
:101010001600370000042000000F7800E3004700AE
:101020000040EB0080487800080037001E00780080
:1010300000004000000F7800630047001040780077
:101040008040E800630047000148780063004700E3
:10105000904078002E40900080CF5000F3FF390080
:101060001E0078006670020000000000A0A52800A5
:10107000586E02000000000091012000D0A920005D
:10108000D89B0200000000006300470090409000E1
:1010900070C0B30000C0600020479800100020001E
:1010A000000F7800E30047000040EB008048780024
:1010B000080037001E00780000004000000F780094
:1010C00063004700104078008040E800630047005C
:1010D0000148780063004700904078002E4090005F
:1010E00080CF5000F3FF39001E007800C47002006A
:1010F00000000000A0A52800586E020000000000BB
:101100004F0478000080FA00000006000000FA009A
:1011100040168000017C200001007000401688000D
:101120001100070020C0B3002D0007006A72020002
:10113000000000000004E0000500320076720200AA
:1011400000000000260007000004E00004003A0050
:10115000360107000004E00001003A00F3FF370009
:101160000080FA00000006000000FA00CA82A90010
:101170000000EB00400388000000EB0050038800F3
:101180000000EB00000388000000EB001003880063
:101190000000EB00F0088800D10A200091407800A0
:1011A000F0C8B30000C06000ADE0B7000000EB0085
:1011B000E008880000642000D008880000002100BA
:1011C000307088008040EB0040E02000014878004B
:1011D0000000EB00906F88000080FA00000006001D
:1011E0000A00FA00004F7800E06F80004007980086
:1011F000CE009000E18F5000440032004E0190007C
:10120000E10F5100040039004E009000E20F500041
:101210004F003200000137009E80FB00310798002C
:101220003E019000E20F5100150032003E00900098
:10123000E20F500007003C00BE0090000100E000FB
:101240000B0032003E019000E10F5100100032000F
:10125000230037003E009000F10F5000EE003200F6
:10126000BE009000F38F5000EB0032001C003700EE
:10127000BDFF07001200200022079800E800370099
:10128000C0A428002C6E020000000000E20037001D
:10129000CA82A8000000EB00F00888000000EB0004
:1012A000B00888000000EB00A00888008000200043
:1012B000F00888008660A9009660A900D10A200085
:1012C00091407800F0C8B30000C060000044A00066
:1012D000ADE0B70010002000906F8800CE0037000E
:1012E00040DF20001E48780041C0B30090DF20009E
:1012F000014878008040EB00A0DF20000148780022
:1013000010002000E06F8800C3003700A0DF20003D
:10131000104078008040E800A0DF200001487800FD
:10132000A0DF2000104078008080FB0040DF20001C
:10133000008040001E487800A0DF20009040780028
:1013400090DF20001040780080CF5000B2003900BC
:1013500040DF2000104078000080FB00100798005C
:10136000100820009E009000808F50003E00320048
:10137000000C20001E019000800F5100050032007B
:10138000000820009E009000808F50004E00320028
:101390009F00370050DF2000104078000080FB00E5
:1013A0004400DE00610060000004E0000300320041
:1013B000100380000000A0001003880050DF200010
:1013C000104078000080FB004300DE0061006000F8
:1013D0000004E0000400320010038000010220003D
:1013E000010070001003880050DF200010407800DA
:1013F0000080FB004200DE00610060000004E000AD
:10140000040032001003800001042000010070007D
:101410001003880050DF2000104078000080FB009F
:101420000000D100610060000004E0000400320010
:1014300010038000010820000100700010038800E4
:1014400050DF2000104078000080FB006100600049
:101450000004E000040032001003800001102000AE
:10146000010070001003880060DF20001040780049
:101470000080FB0030708800307080004800DD0084
:101480003070880050DF2000104078008080FB0022
:1014900030708000008070003070880030708000F4
:1014A0004200DD0064004000307088003170800030
:1014B00000002100808F5000550036000000210000
:1014C000307088005200370070DF20001040780034
:1014D0000080FB0001002000F06F88000170880090
:1014E000F06F800001708000C808DD000080FD0002
:1014F000804078000040EB00F06F880001708800A9
:1015000060DF2000104078000081FB000300200015
:10151000F06F800001708000000071008180710018
:10152000F06F880001708800F06F8000017080000B
:10153000C808DD000080FD00804078000040EB001E
:10154000F06F88000170880050DF200010407800A4
:101550000081FB0003002000F06F8000017080001C
:101560000000710081807100F06F880001708800B8
:10157000F06F8000017080004209DD00CE00DE00C7
:10158000810071004200DD0064004000E0804800FE
:10159000920120000300200030060200000000003D
:1015A000F06F880001708800F26F80000370800087
:1015B0000001200001002000800F5100818F5900A0
:1015C00007003600F06F800001708000700050004E
:1015D000E0805800F06F8800017088000400370038
:1015E0001000200001002000F06F880001708800CA
:1015F000F06F8000017080004008DE0001002000D4
:10160000E0088800F06F800001708000D00888003A
:101610000000EB00E06F88000000EB00200798005E
:101620002E0090000080FA00000006000200FA0080
:10163000906F8000E10F500001003200360037004B
:1016400086C0BF00684060000004E00003003A006C
:10165000100380000000E0002F003A001FE1A80006
:101660008780A9000000EB00107088000E00370092
:101670007140800010708000808040005016800013
:101680004600DE008048780087C0BF0070406000E0
:101690000004E000FCFF32008780A9001070800089
:1016A0000000E80010708800117080003070800029
:1016B000808F5000EEFF39000000EB00100388001F
:1016C0000000EB00F0088800307080001070880087
:1016D0000A003700714080001070800000804000D8
:1016E0000000E9001040780088720200000000004D
:1016F000107080000000E9001070880010708000F9
:101700000000E000F3FF3A0097FE07001000200001
:10171000000F7800020037000000EB00000F780097
:101720001E0078000080FA00000006000200FA00A7
:10173000000F78001E00780080407800002721000C
:10174000104078000080FB000000D1006140600084
:1017500046010700001020000080FA00000006008B
:101760000000FA0000272100104078000010A100BE
:10177000012721008048780041012000B0EC2000C2
:10178000629C0200000000000080FA0000000600D9
:101790000000FA0000272100104078000010A0008F
:1017A000012721008048780021012000F0ED200071
:1017B000629C0200000000000080FA0000000600A9
:1017C0000000FA0080B82000104078000030A0002F
:1017D00081B8200080487800002721001040780060
:1017E0000010A0000127210080487800816A2000B5
:1017F0009140780000CEB30000C060007040B3009C
:10180000A8E6B700916C20009140780000CEB300AC
:1018100000C060007040B300C9E6B700816C2000D2
:101820009140780000CEB30000C060000034A000FA
:10183000C8E6B700CAC2A900C8C2A900C902A90067
:10184000C8E2A800C922A900D01320001012880005
:101850000000EB00201288000000EB00001288005E
:1018600041E2A800D101200040F02000629C02006B
:10187000000000000080FA00000006000800FA00E6
:1018800020079800506980000000E8005069880037
:1018900051698000F00F20000080600050698800CE
:1018A000A81A020000000000D2160200000000008A
:1018B000100798000000EB00606988002E0090007F
:1018C000300798003E009000E30F50003C003200CB
:1018D0003E009000E30F500004003E003E009000E8
:1018E0000000E0000B0032000F0037003E009000C7
:1018F000E60F5000480032003E009000E70F500015
:101900006A0032003E009000E40F500037003200C1
:101910008B0037008109200060F62000629C0200E5
:10192000000000008A0037005100200030632000D2
:10193000629C020000000000AC0007002E00900036
:10194000E10F5000820032001E0090000000E00015
:10195000030034001E009000E20F5000130034001A
:1019600041022000E0FF2000629C02000000000015
:101970008001EB0022002000110020002000200048
:101980001E1D020000000000100798001E009000BD
:10199000E10F500003003A000040EB007500070023
:1019A0000200370080C0B300720007004100200031
:1019B00020022100629C0200000000006400370049
:1019C00011C0B3000040EB00A8000700F0002000A9
:1019D0003A9902000000000051002000600221003E
:1019E000629C020000000000590037001E009000B9
:1019F0008040780000C8B30080C070000040EB0059
:101A00009A000700A1002000B0022100629C0200A1
:101A1000000000004E00370011C0B3000040EB0092
:101A200092000700F00020003A9902000000000038
:101A300000032000200798001E0090000000E00036
:101A400002003A0000052000100798000000EB009B
:101A5000000F780011003700AE00900090032000C6
:101A6000808F5000020036000003200020079800FD
:101A70002E0090008040780010C0B3007B0007006B
:101A80002E00900088720200000000002E009000DE
:101A90000000E800200798001E0FE8001E009000DC
:101AA0009E0F1000ECFF35002900370011C0B30075
:101AB0000040EB006D000700F00020003A990200A2
:101AC0000000000010022000200798001E00900077
:101AD0000000E00002003A00000520001007980016
:101AE0000000EB00000F780011003700AE009000FE
:101AF000F0072000808F5000020036001002200006
:101B0000200798002E0090008040780010C0B3009D
:101B1000560007002E0090008872020000000000AE
:101B20002E0090000000E800200798001E0FE8003B
:101B30001E0090009E0F1000ECFF350004003700DF
:101B400041022000C0202000629C02000000000032
:101B50000080FA00000006000000FA00B10020003A
:101B6000C0092100629C0200000000000080FA0011
:101B7000000006000200FA00004F78001E407800C6
:101B80000042B000804078000040EB0037000700C2
:101B9000F00020003A9902000000000081C0B3006C
:101BA0000040EB0031000700F00020003A990200ED
:101BB0000000000011C0B3000040EB002B00070044
:101BC000F00020003A99020000000000E1C0B300DC
:101BD0000040EB0025000700F00020003A990200C9
:101BE000000000000080FA00000006000000FA007B
:101BF0000040EB004A000700F00020003A99020084
:101C00000000000031C0B3000040EB0026000700D8
:101C1000500020003A9902000000000031C0B300DB
:101C20000040EB0020000700000A20006699020037
:101C30000000000031C0B3000040EB001A000700B4
:101C4000000A2000669902000000000021C0B300D5
:101C50000040EB0014000700000A20006699020013
:101C6000000000000080FA00000006000200FA00F8
:101C7000004F7800114798001E4090000080FB0044
:101C80004400DE00804078001E4078000600070017
:101C90001E409000EF4060001E40780002000700E8
:101CA0000080FA00000006000200FA00004F7800F1
:101CB000114798001E4090004400DD001047980036
:101CC0001E4090000004A0001047980010C0B30010
:101CD0009E4F100003003A001E4090000014A00028
:101CE000104798001E4090000D0007001E40900015
:101CF0000034A000104798001E4090000800070024
:101D00009E40900070CFB30000C060001047980064
:101D10001E409000020007000080FA00000006004C
:101D20000200FA00004F78001E407800664802006A
:101D300000000000CAC2A800CAC2A9000080FA00C0
:101D4000000006000000FA0020A528002C6E02000A
:101D5000000000000080FA00000006000A00FA00FF
:101D6000704080003007980010002000B093880079
:101D7000F4FF070000003700767202000000000048
:101D8000104798001E4090000080FB00400798001C
:101D9000CE009000E38F5000200032004E009000F3
:101DA000E30F50000A003C00CE009000E18F50008D
:101DB0005B0032004E009000E10F50005E003C00DE
:101DC000CE0090000100E000E7003200DB003700A9
:101DD0004E009000E60F50000E003200CE00900042
:101DE000E68F500004003C004E009000E50F5000CC
:101DF00095003200D1003700CE009000E78F5000F0
:101E0000640032004E009000E80F50005400320091
:101E1000CA003700CBFF0700D7FF3700BE00900095
:101E200030C0B300804878003E0090008000E80099
:101E300080C0B3008048780021E3A800C0C0B30090
:101E4000DC97020000000000200798003E00900090
:101E50008080E8002E0090004800DE008048780076
:101E60003E009000E30040002E0090008048780083
:101E7000B0C0B300DC97020000000000200798000B
